:020000040800F2
:1000000000070020F1010008BD2400087524000845
:100010009D2400087524000895240008F3010008B9
:10002000F3010008F3010008F30100085935000846
:10003000F3010008F3010008F3010008F3010008D0
:10004000F3010008F3010008F3010008F3010008C0
:10005000F3010008F30100082143000849430008A8
:100060007143000899430008C1430008F3010008E8
:10007000F3010008F3010008F3010008F301000890
:10008000F3010008F3010008F30100082924000827
:100090005524000865240008F3010008E94300081E
:1000A000F3010008F3010008F3010008F301000860
:1000B000E5440008F3010008F3010008F30100081B
:1000C000F3010008F3010008F3010008F301000840
:1000D000F3010008BD440008D1440008F301000802
:1000E0004D440008F3010008F3010008F301000883
:1000F000F3010008F3010008F3010008F301000810
:10010000F3010008F3010008F3010008F3010008FF
:10011000F3010008F3010008F3010008F3010008EF
:10012000F3010008F3010008F3010008F3010008DF
:10013000F3010008F3010008F3010008F3010008CF
:10014000F3010008F3010008F3010008F3010008BF
:10015000F3010008F3010008F3010008F3010008AF
:10016000F3010008F3010008F3010008F30100089F
:10017000F3010008F3010008F3010008F30100088F
:10018000F3010008F3010008F3010008F30100087F
:10019000F3010008F3010008F3010008F30100086F
:1001A000F3010008F3010008F3010008F30100085F
:1001B000F3010008F3010008F3010008F30100084F
:1001C000F3010008F3010008F3010008F30100083F
:1001D000F3010008F3010008F3010008F30100082F
:1001E000C10F000800000000000000000000000037
:1001F00002E000F000F8FEE772B6374880F30888A6
:10020000364880F3098836483649086040F20000D5
:10021000CCF200004EF63471CEF200010860BFF35C
:100220004F8FBFF36F8F40F20000C0F2F0004EF628
:100230008851CEF200010860BFF34F8FBFF36F8F7C
:100240004FF00000E1EE100A4EF63C71CEF20001D4
:100250000860062080F31488BFF36F8F03F06AFEF6
:1002600003F0FCFE4FF055301F491B4A91423CBF42
:1002700041F8040BFAE71D49184A91423CBF41F886
:10028000040BFAE71A491B4A1B4B9A423EBF51F82E
:10029000040B42F8040BF8E700201849184A914271
:1002A0003CBF41F8040BFAE703F048FE03F024FFDB
:1002B000144C154DAC4203DA54F8041B8847F9E797
:1002C00000F042F8114C124DAC4203DA54F8041B12
:1002D0008847F9E703F030BE000700200023002024
:1002E0000000000808ED00E00001002000070020E9
:1002F000384D0008002300208023002080230020A8
:1003000030520020E0010008E4010008E401000888
:10031000E40100082DE9F04F2DED108AC1F80CD052
:10032000C3689D46BDEC108ABDE8F08F002383F3BF
:1003300011882846A047002003F06AFAFEE703F080
:10034000F3F900DFFEE70000F8B500F04BFE03F024
:100350008BFD074603F0DAFD064600283DD12B4B06
:100360009F423AD001339F423AD0294B27F0FF02F7
:100370009A4238D1F8B200F03FFC354642F2107490
:1003800000F040FC08B10024254601F055F970B397
:10039000032000F043F80024254636B11D4B9F4250
:1003A00003D003F0ABFD00242546002003F066FDDA
:1003B000194B1B691B071FD40DB100F045F800F065
:1003C0008FFC02F083F80546C4B102F07FF8401BB1
:1003D000A04213D900F038F8F3E735460024CFE700
:1003E00004460125CCE705464FF47A74C8E7B4F516
:1003F0007A7F08BF0125D0E70024E0E700F0B8FCD1
:100400004FF47A7003F00AFADEE700BF010007B08C
:10041000000008B0263A09B000040240084B1870EA
:1004200003280CD8DFE800F008050208022000F0DD
:1004300037BE022000F02ABE024B00225A607047ED
:10044000802300208423002010B501F0F5F830B19E
:10045000204B03221A70204B00225A6010BD1F4B04
:100460001F4A1C4619680131F8D004339342F9D170
:1004700062681C4B9A42F1D91B4B9B6803F10063E5
:1004800003F580339A42E9D203F00CFD03F01EFD20
:10049000002000F0C1FD0220FFF7C0FF134B1A6CD3
:1004A00000221A64196E1A66196E596C5A64596ED4
:1004B0005A665B6E72B64FF0E0233021C3F8084DE8
:1004C000D4E9003281F311889D4683F308881047F0
:1004D000C4E700BF8023002084230020000001081F
:1004E00020000108FFFF0008002300200038024020
:1004F000094A136849F2690099B21B0C00FB0133E9
:100500001360064B186844F2506182B2000C01FB84
:100510000200186080B270471823002014230020C6
:1005200010B500211022044600F0D6FD034B03CB8A
:10053000206061601868A06010BD00BF107AFF1FC6
:10054000F0B5ADF54F7D6CAC4FF4C47207460D4667
:100550002046002100F0C0FD01F0B8FF264B4FF40B
:100560007A72B0FBF2F0186093E80700022384E887
:1005700007000DF5E9702382FFF7D2FF4EF6031353
:100580001E49238407A804F0E1FA162384F83231C7
:100590000DF2E32207AB0DF12C0C1E4603CE66458F
:1005A00010605160334602F10802F6D130681060E5
:1005B000B38893800DAE31460122204600F0D8FD6D
:1005C00000230393AB7E029305F11903019380B2DC
:1005D0000123CDE904600093E97E05A3D3E900235C
:1005E000384602F089FB0DF54F7DF0BDAFF300807A
:1005F0009E6AC421818A46EE8C2300205C4B000851
:100600002DE9F0412C4C237ADAB080460D465BBBD5
:1006100027A9284600F0D2FE0746002842D19DF8BF
:100620009D60C82E3ED801464FF4A662204600F0D9
:1006300053FD4FF48073C4F8F8314FF40073C4F8DD
:100640000C334FF44073C4F8203432460DF19E0150
:1006500004F1090000F02EFD26449DF89C307772CD
:1006600023720BB9EB7E23728122002106AC27A8EE
:1006700000F032FD0122214627A800F0E5FE00230C
:100680000393AB7E029305F1190380B201932823F3
:10069000CDE904400093E97E05A3D3E90023404659
:1006A00002F02AFB5AB0BDE8F08100BFAFF3008032
:1006B00026417272DF25D7B7D4330020F0B5254E1E
:1006C0004FF48A7505FB0065F1B096F8D83085F8CF
:1006D000DC300024D822214685F8E8403AA800F012
:1006E000FBFC06F1090000F0EFFCD5F8E4308DF8D2
:1006F000F000C2B206AF06F109010DF1F100CDE93B
:100700003A3400F0D7FC394601223AA800F0D2FE74
:1007100080B2CDE9047008230127CDE9023706F144
:10072000D803019330230093317A0B4807A3D3E910
:10073000002302F0E1FAA04206DD01F0C7FEC5F891
:10074000E000384671B0F0BD2046FBE778F6339FF5
:1007500093CACD8DD4330020A43300202DE9F0417D
:100760001D4D1E4E1E4F86B0284602F0F1FA03467C
:1007700058B30024CDE90344ADF81440027B8DF852
:10078000142099684068029403AA03C21B68DFF82A
:10079000548043F00043029301F09AFE821941F124
:1007A0000003009402A9384601F02EF9A04205DDAD
:1007B000284602F0D1FA88F80040D5E798F80030D2
:1007C000072B05D8013388F8003006B0BDE8F0816A
:1007D000014802F0C1FAF8E7A433002040420F00BC
:1007E000103900200939002070B50D4614461E4608
:1007F00002F0DEF950B9022E10D1012C0ED112A355
:10080000D3E90023C5E90023012007E0282C10D0FC
:1008100005D8012C09D0052C0FD0002070BD302C3C
:10082000FBD10BA3D3E90023ECE70BA3D3E900230F
:10083000E8E70BA3D3E90023E4E70BA3D3E9002304
:10084000E0E700BFAFF30080401DA12026812A0B06
:1008500078F6339F93CACD8D9E6AC421818A46EE75
:1008600026417272DF25D7B7F017304A39059E56F8
:1008700038B505460E4C0021013500F0EFFBA4F819
:100880002C55B4F82C0500F0D1FB78B1B4F82C0548
:1008900000F0DCFB014648B9B4F82C0500F0DEFBA3
:1008A000B4F82C350133A4F82C35EAE738BD00BF85
:1008B000D433002010B50A4B0A4A1A6003F580535E
:1008C00093F870203AB9DC6E2CB1204600F032FF6C
:1008D000204601F06FF8BDE81040034800F02ABF41
:1008E00010390020B04B0008684900202DE9F04F76
:1008F0008FB000AF05460C4602F05AF900284BD1E4
:10090000237E022B1BD1E38A012B18D101F0DEFDDF
:100910000646FFF7EDFD03464FF4C870DFF8D482BA
:10092000B3FBF0F206F5167602FB103316FA83F3EA
:10093000C8F80030E37E33B9A74B00221A703C3769
:10094000BD46BDE8F08F07F12401204600F0EAFC27
:100950000028F4D107F11400FFF7E2FD97F82640D4
:1009600007F11401224607F1270004F0BDF8002822
:10097000E2D10F2C08D8984B1C70D8F80030A3F5A2
:100980001673C8F80030DAE797F824100029D6D09B
:10099000284602F005F9D2E7E38A282B33D010D895
:1009A000012B2BD0052BCAD1BFF34F8F8B498C4B1A
:1009B000CA6802F4E0621343CB60BFF34F8F00BFFD
:1009C000FDE7302BBBD1874EE17E327A9142B6D122
:1009D000607E3146002291F8DC50854200F0AD8007
:1009E0000132042A01F58A71F5D1326840F6B83136
:1009F000FA328A4294BF32603160A0E7214628462D
:100A0000FFF79EFD9BE721462846FFF7F9FD96E795
:100A1000B2F8EC507B6005F103094FEA99094FEAFF
:100A20008902D11DC908A8EBC1039D46EB460021F0
:100A3000584600F051FB04F1EE012A463144584675
:100A400000F038FB7B6813B9012000F0E5FA96F856
:100A5000D20000F0EBFA044630B9307200F006FB29
:100A6000204600F0D9FAB0E0D6F8D4203AB996F88A
:100A7000D200B6F82C25824201D8FFF7F9FED6F84D
:100A8000D4202A44944208D296F8D200B6F82C25F5
:100A90000130824201D8FFF7EBFE70685FFA89F2FD
:100AA000594600F021FB08B9C54679E0726896F80E
:100AB000D2002A447260D6F8D42005EB0209C6F8A9
:100AC000D49000F0B3FA814509D396F8D220D6F835
:100AD000D4000132001B86F8D220C6F8D400FF2DC6
:100AE0000FD80024347200F0C1FA204600F094FAC6
:100AF00000F0A2FD3C4B188108B9FFF7A5FCC546E4
:100B00001DE7BB6896F8D9000AFB0362FB68D2F8C0
:100B1000E41082F8E83001F58061C2F8E030C2F8F4
:100B2000E410FFF7CBFDFFF719FE96F8D92001324C
:100B300002F0030286F8D920B6E74FF48A7A0AFB5E
:100B400002F505F1EA013144204600F0E7FCF860C7
:100B500000287FF4F4AE3544012285F8E82001F046
:100B6000B5FCD5F8E020D6ED007ADFED206A801ADA
:100B7000192838BF192040F6B832904228BF1046D5
:100B8000B8EE677A07EE900AF8EEE77A67EEA67A93
:100B9000DFED176AE7EE267AFCEEE77AC6ED007A1B
:100BA00096F8D9307168BB600AFB03F4321992F8E9
:100BB000E8505DB1D2F8E4308B42E8463FF428AF0C
:100BC000002182F8E810C2F8E010C5467368064AB2
:100BD0009B0A01331381B2E69D33002000ED00E053
:100BE0000400FA05D43300208C230020CDCCCC3D6A
:100BF0006666663FA0330020014B1870704700BF47
:100C00009823002030B54FF000542C4B22689A42B4
:100C100085B023D1637D0BB3294A2A481370237D05
:100C200003724FF48073C0F8F8314FF40073C0F8CA
:100C30000C3300254FF44073C0F820342249C0F82B
:100C4000E450C922093000F035FA2046E022294656
:100C500000F042FA0124204605B030BD03F060F9EF
:100C6000044608B90024F6E7184A194D136C43F0FE
:100C700000731364AA6D174B9A42F3D12B6E013B9C
:100C80007E2BEFD8144A07CA01AB83E80700184649
:100C9000032100F09FFC6B6D83424FF00003E1D114
:100CA0002A6D8A4201BFAB65054B2A6E1A7003BFDD
:100CB0000A4BEA6D1A601C46CDE700BF9AAD44C5E9
:100CC00098230020D4330020160000200038024072
:100CD000006600405041A0B058660040102300203C
:100CE00037B51A4D00F0A8FC02236B71184B288110
:100CF00019681848012201F083FA00230193164B6A
:100D0000164900931648174B4FF4805201F020FF0C
:100D1000154B197811B1124801F042FF01F0D6FBD2
:100D20000446FFF7E5FB4FF4C873B0FBF3F202FB98
:100D3000130304F5167010FA83F00C4B186003F0DF
:100D4000E5F808B10F232B8103B030BD8C230020C0
:100D50001023002010390020E90700089C23002000
:100D6000A4330020ED08000898230020A0330020C1
:100D70002DE9F04F2DED028B0FF23829D9E90089CA
:100D8000834C93B00BAE9FED7E8BFFF7E7FC814F5A
:100D9000DFF828A200230A93ADF834300B93736078
:100DA0004FF0000B5B468DED008B01250DF11D0210
:100DB00007A938468DF81C508DF81DB001F0CEF90A
:100DC0009DF81C30002B40F0A580204601F0F0FE7D
:100DD0000646002845D1704F01F078FB3B689842E9
:100DE0003FD301F073FB8246FFF782FB4FF4C873D9
:100DF000B0FBF3F202FB13030AF5167010FA83F04E
:100E00003860664F97F800B0CBF1100ABBF1000FC5
:100E100014BF33462B465FFA8AFA0EA88DF82830A5
:100E2000FFF77EFBBAF1060F28BF4FF0060A0EABA4
:100E300003EB0B0152460DF1290000F03BF90AAB20
:100E40000393182302930AF10102554BD2B2CDE964
:100E50000053049220464CA3D3E9002301F0EEFE98
:100E60003E7001F033FB4F4A4F4D1368C31AB3F580
:100E70007A7F2ED3106001F02BFB02460B462046F2
:100E800001F074FF204601F093FE10B32B7A474E19
:100E9000002B14BF03230223737101F017FB0EAF65
:100EA0004FF47A730122B0FBF3F0394630603046DC
:100EB00000F010FA182302933D4B019380B240F2E8
:100EC0005513CDE90370009342464B46204601F08E
:100ED000B5FE2B7A93B101F0F9FA002607464FF4DC
:100EE0008A7A95F8D900304400F003000AFB0053D9
:100EF00093F8E82092B30136042EF2D1C82002F014
:100F00008DFC2B7A002B7FF43DAF13B0BDEC028B30
:100F1000BDE8F08FDAF8143083F48053CAF8143047
:100F2000594610220EA800F0D7F80DF11E0308AAAA
:100F30000AA9384600F06EFE96E803000FAB83E87E
:100F400003009DF834308DF844300A9B0E930EA9AF
:100F5000DDE90823204602F0DDF821E7D3F8E020A0
:100F600042B12B68FA2B38BFFA23BA1A0533B2EB19
:100F7000430FC0D3FFF7A2FB0028BCD1BEE700BFE0
:100F80000000000000000000401DA12026812A0B67
:100F9000A433002010390020A03300209D3300200E
:100FA0009C33002004390020D43300208C230020FF
:100FB00008390020F1C6A7C1D068080F000402401C
:100FC00008B5054800F0C4FEBDE80840034A0449DE
:100FD000002003F065BD00BF10390020304A00201A
:100FE000B508000870B502F0EDFD094E094D3080DE
:100FF000002428683388834208D902F0DDFD2B687D
:1010000004440133B4F5803F2B60F2D370BD00BFC0
:10101000244A0020F849002002F084BE00F100605C
:10102000920000F5803002F013BE0000054B1A68F4
:10103000054B1B889B1A834202D9104402F0BCBDA9
:1010400000207047F8490020244A0020024B1B680A
:10105000184402F0B9BD00BFF8490020024B1B68DC
:10106000184402F0C9BD00BFF8490020064991F8B4
:10107000243033B10023086A81F824300822FFF7B6
:10108000CDBF0120704700BFFC490020022802BFED
:10109000024B4FF480529A61704700BF0004024037
:1010A000022802BF024B4FF080529A61704700BF86
:1010B0000004024010B50023934203D0CC5CC4541A
:1010C0000133F9E710BD000003460246D01A12F9B9
:1010D000011B0029FAD1704702440346934202D013
:1010E00003F8011BFAE770472DE9F8431F4D14463A
:1010F00095F824200746884652BBDFF870909CB3D1
:1011000095F824302BB92022FF2148462F62FFF7A3
:10111000E3FF95F82400C0F10802A24228BF22464E
:10112000D6B24146920005EB8000FFF7C3FF95F869
:101130002430A41B1E44F6B2082E17449044E4B297
:1011400085F82460DBD1FFF791FF0028D7D108E0B4
:101150002B6A03EB82038342CFD0FFF787FF00287F
:10116000CBD10020BDE8F8830120FBE7FC4900203B
:101170002DE9F3470D46044600219046284640F2EB
:101180007912FFF7A9FF234620220021284601F00B
:1011900063FF231D02222021284601F05DFF631D0D
:1011A00003222221284601F057FFA31D03222521F7
:1011B000284601F051FF04F1080310222821284697
:1011C00001F04AFF04F1100308223821284601F0FB
:1011D00043FF04F1110308224021284601F03CFF9F
:1011E00004F1120308224821284601F035FF04F1DA
:1011F000140320225021284601F02EFF04F1180389
:1012000040227021284601F027FF04F12003082224
:10121000B021284601F020FF04F121030822B82163
:10122000284601F019FF04F12207C0263B4631464B
:1012300008222846083601F00FFFB6F5A07F07F117
:101240000107F3D194F832308DF8073031460DF1B3
:1012500007030822284601F0FFFE002604F1330AA6
:101260009DF807304FEAC6099E4209F5A47720D3BE
:1012700094F83231502B28BF50238DF80730B8F145
:10128000000F08D139460DF107030722284601F067
:10129000E3FE09F24F17002604F233149DF80730DD
:1012A0009E4207EBC6010DD30731C80802B0BDE866
:1012B000F0870AEB060308223946284601F0CCFEE7
:1012C0000136CDE7A3190822284601F0C5FE0136F4
:1012D000E4E7000013B504460846002101602346F8
:1012E000C0F803102022019001F0B6FE0198231DE2
:1012F0000222202101F0B0FE0198631D0322222169
:1013000001F0AAFE0198A31D0322252101F0A4FEED
:10131000019804F108031022282101F09DFE072006
:1013200002B010BDF7B5047F05460E462CB1838A86
:10133000122B02D9012003B0F0BD00231946072269
:101340000096284601F04CFD731C009301220023F7
:101350000721284601F044FDD4B9B31C00930522AF
:1013600023460821284601F03BFD0D24B378102BBD
:10137000E0D83746B278BB1B934210D32B7FA88AA4
:101380000734E408B3B9844294BF00200120D2E7B7
:10139000AB8ADB00083BDB08B3700824E6E7FB1CE4
:1013A0000093214600230822284601F019FD083445
:1013B0000137DFE7201A18BF0120BCE7F7B5047F2B
:1013C00005460E462CB1838ACA2B02D9012003B0F0
:1013D000F0BD0023194600960822284601F000FDC2
:1013E000731CD4B90822009311462346284601F005
:1013F000F7FC10247378C82BE8D8012372785F1C9F
:10140000013B934210D32B7FA88A0734E408B3B979
:10141000844294BF00200120D9E7AB8ADB00083B5F
:10142000DB0873700824E5E7F319009321460023D5
:101430000822284601F0D4FC08343B46DEE7201A97
:1014400018BF0120C3E70000F7B50D460446002190
:10145000164628468122FFF73FFE23460822002138
:10146000284601F0F9FD94F901206378002AB8BFFD
:101470007F238DF807309EB90DF10703072208215D
:10148000284601F0E9FD0F27002602349DF80730B9
:101490009E4207EBC60105D30731C80803B0F0BD73
:1014A0000827F1E7A3190822284601F0D5FD0136E7
:1014B000ECE70000F7B50E4605460021144630461D
:1014C000CE22FFF709FE2B4628220021304601F0EC
:1014D000C3FD2B7AC82B28BFC8238DF807308CB9E1
:1014E0000DF1070308222821304601F0B5FD302414
:1014F0002F469DF807207B1B934205D3E01DC008B3
:1015000003B0F0BD2824F3E707F1090321460822C0
:10151000304601F0A1FD08340137EAE7F7B5047F52
:1015200005460E4634B1838AB3F5827F02D9012085
:1015300003B0F0BD0096012310220021284601F0DF
:101540004FFCDCB9B31C0093092223461021284626
:1015500001F046FC19247388B3F5807FE7D837463D
:101560007288BB1B934210D32B7FA88A0734E408F0
:10157000B3B9844294BF00200120D9E7AB8ADB00D5
:10158000103BDB0873801024E5E73B1D00932146E8
:1015900000230822284601F023FC08340137DFE746
:1015A000201A18BF0120C3E730B5094D0A44914203
:1015B0000DD011F8013B5840082340F30004013BD3
:1015C0002C4013F0FF0384EA5000F6D1EFE730BD62
:1015D0002083B8EDF7B54FF0FF33DFF854C0DFF8E4
:1015E00054E000EB81011A4688421CD050F8044BAD
:1015F000019401AF042417F8015B82EA0562082513
:10160000DB18164605F1FF355241002EBCBF83EAB8
:101610000C0382EA0E0215F0FF05F1D1013C14F033
:10162000FF04E8D1E0E7D843D14303B0F0BD00BFE9
:101630009336EAA9EBE1F042F7B5384A10685168F1
:101640006B4603C36A4636493648082303F05CFA02
:101650000446002833D10A25334A106851686B4686
:1016600003C36A4631492F48082303F04DFA044664
:10167000002849D00369B3F5E02F45D8B0F86610CB
:1016800040F2E93291423FD1294A024402F15C0121
:101690008B4239D35C3B234900209E1AFFF784FF1D
:1016A0003246074604F164010020FFF77DFFA3687E
:1016B0009F4229D1E368984208BF002524E00369CE
:1016C000B3F5E02F27D8418B40F2E932914220D187
:1016D000174A024402F110018B4218D3103B114902
:1016E00000209D1AFFF760FF2A46064604F1180104
:1016F0000020FFF759FFA3689E4202D1E368984299
:1017000001D00D25A8E70025284603B0F0BD10251F
:10171000A2E70C25A0E70B259EE700BF744B00084D
:10172000DCFF0600000001087D4B000890FF06006A
:101730000800FFF710B5037C044613B9006803F0F6
:10174000CBF9204610BD00000023BFF35B8FC360C0
:10175000BFF35B8FBFF35B8F8360BFF35B8F70471B
:10176000BFF35B8F0068BFF35B8F704770B50546B2
:101770000C30FFF7F5FF05F1080604463046FFF789
:10178000EFFFA04206D930466D68FFF7E9FF254418
:10179000281A70BD3046FFF7E3FF201AF9E7000072
:1017A00070B50546406898B105F10800FFF7D8FF0D
:1017B00005F10C0604463046FFF7D2FF844230465E
:1017C00094BF6D680025FFF7CBFF013C2C44201A25
:1017D00070BD000038B50C460546FFF7C7FFA042B4
:1017E00010D305F10800FFF7BBFF04446868B4FBA1
:1017F000F0F100FB1144BFF35B8F0120AC60BFF33D
:101800005B8F38BD0020FCE72DE9F0411446074608
:101810000D46FFF7C5FF844228BF0446D4B1B84641
:1018200058F80C6B4046FFF79BFF30442860404659
:101830007E68FFF795FF331A9C4203D86C60012045
:10184000BDE8F0816B60A41B3B68AB602044E8609E
:101850000220F5E72046F3E738B50C460546FFF7CA
:101860009FFFA04210D305F10C00FFF779FF04445D
:101870006868B4FBF0F100FB1144BFF35B8F0120FB
:10188000EC60BFF35B8F38BD0020FCE72DE9FF4122
:10189000884669460746FFF7B7FF6C4606B204EB79
:1018A000C6060025B44209D06268206808EB05012D
:1018B000FFF700FC636808341D44F3E72946384607
:1018C000FFF7CAFF284604B0BDE8F081F8B5054629
:1018D0000C300F46FFF744FF05F10806044630467A
:1018E000FFF73EFFA042304688BF6C68FFF738FF25
:1018F000201A386020B130462C68FFF731FF2044B1
:10190000F8BD000073B5144606460D46FFF72EFFDE
:10191000844228BF04460190DCB101A93046FFF79C
:10192000D5FF019B33B93268C5E90233C5E900240C
:1019300001200CE09C4238BF019428600198686047
:101940008442F5D93368AB60241AEC60022002B0FF
:1019500070BD2046FBE700002DE9FF410F466946B8
:10196000FFF7D0FF6C4600B204EBC0050026AC4286
:1019700009D0D4F8048054F8081BB8194246FFF780
:1019800099FB4644F3E7304604B0BDE8F08100001F
:1019900038B50546FFF7E0FF044601462846FFF745
:1019A00019FF204638BD00000121884238BF084693
:1019B00003F07CB808B103F08FB8704710B4026828
:1019C00054681A4623465DF8044B184700207047B8
:1019D0000020704770470000002070470E207047BD
:1019E00000F5805090F8D800C0F340007047000028
:1019F00000F5805090F9E0007047000000F580503D
:101A0000C0F8DC1001207047F7B50C68BDF82070F5
:101A100014F0005473D10D7B082D70D8302585F358
:101A20001188456AAE6876010CD4AC68240108D4EC
:101A3000AC6814F0805460D184F31188204603B060
:101A4000F0BD01240E6804F1180C002EB8BFF6009A
:101A50004FEA0C1CB4BF46F00406760545F80C604E
:101A60000E680FFA84FC16F0804F18BF05EB0C1EB1
:101A700005EB0C1C1EBFDEF8806146F00206CEF8B6
:101A800080610E7BCCF8846105EB04158E68C5F887
:101A90008C614E68C5F88861DCF8805145F001051D
:101AA000CCF8805141F2780500EB441C660105EB4F
:101AB0004414AC440444CCE900230D46083401F13D
:101AC0000C0C55F804EB44F804EB6545F9D12D886E
:101AD0002580841904F5805407F0030594F8946078
:101AE00026F00B06354384F89450002484F31188C3
:101AF000009700F035FD0120A1E70224A2E74FF096
:101B0000FF309CE713B500F580540191E06EFFF7BC
:101B100047FE1F280AD90199E06E2022FFF7B6FE82
:101B2000A0F120035842584102B010BD0020FBE74D
:101B300008B5302383F3118800F58050C06EFFF79D
:101B400003FE002383F3118808BD00000022026019
:101B5000828142608260704710B500220023C0E994
:101B600000230023044603810C30FFF7EFFF2046DB
:101B700010BD0000F0B5054600F580500C4690F809
:101B8000D83013F0040FC3F3800108BF114661F38E
:101B9000820380F8D83005EB441303F584531033E7
:101BA00089B01B79D8074FEA44162FD582B319079D
:101BB0002ED46846FFF7D0FF05EB441303F584539A
:101BC00003AA03F1080718685968144603C40833C8
:101BD000BB422246F7D1186820609B88A380DDE9CC
:101BE0000E23CDE900230123ADF808302B686946A8
:101BF0001B6C28469847354405F5845510352B79DC
:101C00001A075CBF43F008032B7101E0002AF2D1F0
:101C100009B0F0BD2DE9F0479A4688B007468846DE
:101C20009146302383F3118807F580546846FFF707
:101C300093FFE06EFFF79AFD1F282AD9E06E20225D
:101C40006946FFF7A5FE202823D103AD444605AB26
:101C50002E4603CE9E4220606160354604F10804A2
:101C6000F6D130682060B388A380DDE90023C9E99C
:101C70000023BDF80830AAF80030002383F3118850
:101C800053464A464146384608B0BDE8F04700F0A2
:101C90002BBC002080F3118808B0BDE8F08700005D
:101CA0002DE9F84F182204460F4604300021FFF7B3
:101CB00013FA2046234B40F8283BFFF747FF04F177
:101CC0003800FFF749FF04F1580804F582554646ED
:101CD000183530462036FFF73FFFAE42F9D104F504
:101CE00080554FF480534FF00009C5E91739C5F806
:101CF00058800123EE6604F5875804F58456C5F82C
:101D0000649085F8683085F87030183608F1180846
:101D10004FF0000A4FF0000B46E908ABA6F118009F
:101D2000FFF714FF203646F8289C4645F4D185F885
:101D3000E07017B1044800F0C3FB044B6362204617
:101D4000BDE8F88FB04B0008884B000800640040E5
:101D500010B5044B197804464A1C1A70FFF7A0FF0F
:101D6000204610BD2C4A00202DE9F047002950D014
:101D7000294B2A4FB7FBF1F599428CBF0A23112357
:101D8000581EB5FBF3FC03FB1C53C4B22BB1022855
:101D90000346F5D80020BDE8F0870CF1FF36B6F514
:101DA000806FF7D2C4EBC40E0EF103034FEAE309D0
:101DB000C3F3C703A4EB030809F1010A4FF47A75D2
:101DC0005FFA88F009FB05555AFA88F8B5FBF8F573
:101DD000B5F5617FC1BF0EF1FF33C3F3C703E01A4E
:101DE000C0B25C1C50FA84F40CFB04F4B7FBF4F4AE
:101DF000A142CFD1013BDBB20F2BCBD80138C0B20F
:101E00000728C7D80021107116809170D370012067
:101E1000C1E70846BFE700BF3F420F0040787D01A1
:101E200070B505460E464FF47A746B6A5B6803F032
:101E30000103B34207D04FF47A7001F0EFFC013C8C
:101E4000F3D1204670BD0120FCE7000070B5426A66
:101E5000936913F0700F17D000230C4D936141F27A
:101E6000900400EB4312224411794E0709D58907EB
:101E700007D5416A55F823608E60117941F004015D
:101E800011710133032BECD170BD00BF9C4B0008D6
:101E900073B51D46436A16469A68D207044609D5AB
:101EA0009A6801219960C2F34002CDE900650021E2
:101EB000FFF760FE636A9A68D1050BD59A684FF404
:101EC00080719960C2F34022CDE90065012120466E
:101ED000FFF750FE636A9A68D2030BD59A684FF4F5
:101EE00080319960C2F34042CDE90065022120466D
:101EF000FFF740FE04F58053D3F8DC0010B103680F
:101F00001B699847204602B0BDE87040FFF79EBFAE
:101F1000F8B50446466A002977D106F10C073868FF
:101F2000800775D006EB01153868D5F8B00110F0C0
:101F3000040FD5F8B0011ABFC00840F00040400DB2
:101F4000A062D5F8B0C11CF0020F1CBF40F0804069
:101F5000A062D5F8B40106EB011100F00F0084F87F
:101F60003400D1F8B80184F82C00D1F8B801000A87
:101F700084F82D00D1F8B801000C84F82E00D1F8B7
:101F8000B801000E84F82F00D1F8BC0184F83000AD
:101F9000D1F8BC01000A84F83100D1F8BC01000C72
:101FA00084F83200D1F8BC11090E84F833103821BE
:101FB000396004F1440004F1280104F1340551F8BA
:101FC000046B40F8046BA942F9D109880180C4E987
:101FD0000E2321460023A4F8403051F8383B204618
:101FE0001B6C984704F5805393F8D820D3F8DC0095
:101FF00042F0040283F8D82010B103681B699847A7
:102000002046BDE8F840FFF721BF06F1100786E73C
:10201000F8BD000010B5044600F05AFA02460B461F
:1020200052EA030102D0013A63F10003044908684F
:1020300020B12146BDE81040FFF76ABF10BD00BFC8
:10204000284A0020F0B5302181F31188DFF848E0FC
:1020500000F583511831002441F2900C00EB441537
:1020600065442E7977070ED4F6060CD5D1E90076B3
:1020700097429E4107D2466A5EF82470B7602E7977
:1020800046F004062E710134032C01F12001E5D144
:10209000002383F31188F0BD9C4B000808B5302362
:1020A00083F31188FFF7D2FE002383F3118808BD64
:1020B0002DE9F041436A0446986800F0E050B0F121
:1020C000E05F0E4622D0F8B1302383F3118800255B
:1020D00004F5845741F2900804EB451343441B79FF
:1020E0001A0706D50135032D07F12007F4D1012089
:1020F00007E05B07F6D43946304600F083FA002843
:10210000F0D1002383F31188BDE8F0810120FBE7C3
:1021100008B5302383F3118800F58050C06EFFF7B7
:1021200025FB002383F3118843090CBF0120002005
:1021300008BD0000F8B51D46002313700F46064683
:102140001446FFF7E5FF80F00100387025B12946FD
:102150003046FFF7ADFF2070F8BD00002DE9B84113
:102160000C4615461F46804600F0B2F90B46217812
:10217000024609B9287850B14046FFF763FFFFF7E0
:102180008DFF3B462A462146FFF7D4FF0120BDE8DC
:10219000B881000070B5302686F31188174B1A6C91
:1021A00042F000721A641A6A42F000721A621A6AE5
:1021B00022F000721A62002383F3118800F5805424
:1021C00094F8D83013F0010516D1A9B186F311881F
:1021D0000321132001F01EFA0321142001F01AFA42
:1021E0000321152001F016FA94F8D83043F00103CA
:1021F00084F8D83085F3118870BD00BF00380240E4
:102200002DE9F04700F5805588B095F8E030012BB6
:1022100004468846164600F28280824F57F82320F3
:102220000AB947F82300D7F800A0C4F81C8084F846
:102230002060BAF1000F64D095F8E030012B70D027
:1022400001212046FFF7A6FF302383F31188626A3D
:10225000136823F002031360626A136843F00103FA
:102260001360636A00275F6187F3118801212046AC
:10227000FFF7D6FD002800F09580E86EFFF764FABE
:1022800004F58359BA4609F118092022002168464D
:10229000FEF722FF02A8FFF759FCCDF818A06A4606
:1022A00009EB07030DF1180E9446BCE80300F44552
:1022B00018605960624603F10803F5D1DCF80000AC
:1022C000186020379CF804201A71602FDDD195F832
:1022D000D8306FF38203002785F8D8306A4641462C
:1022E0002046ADF80070ADF802708DF80470FFF76D
:1022F0003BFD636A48BB4FF400421A6008B0BDE87A
:10230000F08741F2E800FFF74FFB814610B15146DC
:10231000FFF7C6FCC7F80090B9F1000F8CD1002080
:10232000ECE7386803681B6B98470146002887D1A3
:102330003868FFF72FFF3868036832465B6841460C
:10234000984700287FF47CAFE9E761221A609DF886
:1023500002309DF803201B06120402F4702203F0E1
:1023600040731343BDF80020C2F3090213439DF8E4
:1023700004201205022E02F4E0020CBF4FF00041CF
:1023800000211343626A0B43D361636A13225A61CB
:10239000626A136823F00103136039462046FFF791
:1023A0003FFD08B9636AA6E795F8E03093BB616A20
:1023B000D1F8002242F00102C1F80022616AD1F88E
:1023C000002222F47C5222F00E02C1F80022616A3F
:1023D000D1F8002242F46062C1F80022626AC2F8B9
:1023E0001432626AC2F80432626A41F6FF71C2F8BE
:1023F0000C12626AC2F84032626AC2F84432636AFE
:102400000122C3F81C22626AD2F8003223F00103D1
:10241000C2F8003295F8D83043F0020385F8D8307E
:102420006CE700BF284A002008B500F051F850EAD8
:102430000103024602D0421E61F10001044B1868FC
:1024400010B10B46FFF724FDBDE8084001F0B8B815
:10245000284A002008B50020FFF7DCFDBDE8084051
:1024600001F0AEB808B50120FFF7D4FDBDE8084083
:1024700001F0A6B800B59BB0EFF309816822684669
:10248000FEF718FEEFF30583014B9B6BFEE700BFE1
:1024900000ED00E008B5FFF7EDFF000000B59BB0D0
:1024A000EFF3098168226846FEF704FEEFF3058327
:1024B000014B5B6BFEE700BF00ED00E0FEE70000B4
:1024C0000FB408B5029801F059F9FEE701F06ABCB3
:1024D00001F04CBC0139C9B202299EBF00EBC1001A
:1024E0000023C0E901337047F8B51B885B07054638
:1024F0000E4615D4044600F11807BC4210D063689C
:1025000053B12B682846DB6B9847A368C1B23246AB
:10251000606898470834F0E7A368002BF1D1F9E729
:102520000120F8BD73B56C4684E806000146002220
:102530004E68D5B26EB98E685EB900EBC200021D5E
:1025400094E80300013582E803001D70012002B009
:1025500070BD0132032A01F10801E9D10020F6E73C
:102560002DE9F04F89B00446BDF848700E46054687
:1025700000F118084FF0000907F004074FF0000AB7
:102580004FF0000BA84538D06B680BB9AB684BB166
:1025900057B923682046DB6B9847AB68C1B2324617
:1025A000686898470835EDE7B9F1000FFAD1CDE931
:1025B00000ABADF80890334603AA06F1080E186880
:1025C00059689446ACE80300083373456246F6D177
:1025D0001868CCF800009B88ACF80430FFF778FF4F
:1025E0000423ADF808302368CDE900011B6C69466F
:1025F000204698474FF00109D4E7012009B0BDE813
:10260000F08F000030B503680968DD0FB5EBD17FAE
:1026100023F0604421F060424FEAD1700BD0002BD0
:10262000B8BFA40C0029B8BF920C944202D034BFAA
:102630000120002030BD944205D1C1F38070C3F366
:1026400080738342F6D194422CBF00200120F1E731
:102650002DE9F041456A15B94162BDE8F0814B684A
:1026600023F06047C3F38A464FEAD37EC3F38078F2
:1026700016EA230638BF3E46AC462B465A68BEEBE8
:10268000D27F22F060440AD0002A18DAA40CB442A7
:1026900017D19D420FD10D60DEE71346EEE7A7424A
:1026A00007D102F08044C2F3807242450BD054B18E
:1026B000EFE708D2EDE7CCF800100B60CDE7B442AD
:1026C00001D0B442E5D81A689C46002AE5D11960C9
:1026D000C3E700002DE9F047089D01F007044FEA29
:1026E000D508224405F0070500EBD1004FF47F49DF
:1026F000944201D1BDE8F08704F0070705F0070A0E
:1027000057453E4638BF5646C6F10806111B8E4255
:1027100028BF0E46E10808EBD50E415C13F80EC049
:10272000B94029FA06F721FA0AF1FFB28CEA010151
:1027300047FA0AF739408CEA010C03F80EC034441A
:102740003544D5E780EA0120082341F2210201B295
:102750004000002980B203F1FF33B8BF504013F0AE
:10276000FF03F4D17047000038B50C468D18A54220
:1027700000D138BD14F8011BFFF7E4FFF7E70000B4
:1027800042684AB1136843604389818901339BB22F
:102790009942438138BF83811046704770B588B035
:1027A000202204460D4668460021FEF795FC20468F
:1027B0000495FFF7E5FF024658B16B46054608AEA3
:1027C0001C4603CCB44228606960234605F1080525
:1027D000F6D1104608B070BD082817D909280CD0CA
:1027E0000A280CD00B280CD00C280CD00D280CD0AB
:1027F0000E2814BF4020302070470C207047102056
:102800007047142070471820704720207047000040
:10281000082817D90C280CD910280CD914280CD941
:1028200018280CD920280CD930288CBF0F200E2056
:102830007047092070470A2070470B2070470C2012
:1028400070470D20704700002DE9F843078C072FD3
:1028500004461ED9D0E9029800254FF6FF73C5F152
:102860002006A5F1200029FA05F108FA06F628FA53
:1028700000F031430143C9B21846FFF763FF083542
:10288000402D0346EBD1E1693A46BDE8F843FFF736
:102890006BBF4FF6FF70BDE8F883000010B54B68C2
:1028A00023B9CA8A63F30902CA8210BD04691A688F
:1028B0001C600361C38A013BC3824A60EFE70000EA
:1028C0002DE9F84F1D46CB8A0F46C3F309010529B0
:1028D000814692460B4630D00020AAB207F11A0476
:1028E0009EB2042E1FFA80F80FD8904503F1010321
:1028F00006D3FB8A0A4462F30903FB8201201AE033
:102900001AF80060E6540130EAE79045F1D2A1F1EF
:10291000050B1C237C68BBFBF3F203FB12BB1FFA05
:102920008BF6002C45D14846FFF72AFF044638B9FC
:1029300078606FF00200BDE8F88F4FF00008E6E71E
:10294000002606607860ADB24FF0000B454510D907
:102950000AEB0803221D13F8011B9155B1B208F1CF
:1029600001081B291FFA88F82BD0454506F10106FE
:10297000F1D8FB8AC3F30902154465F30903BCE7E8
:10298000013292B21C462368002BF9D16B1F0B4415
:102990001C21B3FBF1F301339BB29A42D3D2BBF1BA
:1029A000000FD0D14846FFF7EBFE20B9C4F800B0C5
:1029B000BFE70122E7E7C0F800B05E4620600446AA
:1029C000C1E74545D5D94846FFF7DAFE08B920608A
:1029D000AFE7C0F800B0002620600446B6E700006C
:1029E0002DE9F04F2DED028B1C4683B05B690192FF
:1029F00007468846002B00F0A780238C2BB1E269A4
:102A0000002A00F0A180072B35D807F10C00FFF752
:102A1000B7FE054638B96FF00205284603B0BDEC95
:102A2000028BBDE8F08F14220021FEF755FB228CAB
:102A3000E16905F10800FEF73DFB208C013080B212
:102A4000FFF7E6FEFFF7C8FE013880B220840130B0
:102A500028746369228C1B782A4403F01F0363F0F7
:102A60003F0348F000411372384669602946FFF77A
:102A7000EFFD0125D1E702339BB20722C18A06335D
:102A8000B3FBF2F3828A521A9BB292B29342C2D83B
:102A900000F10C034FF0000908EE103A4FF0800AE5
:102AA0004E464D4618EE100AFFF76AFE8346002890
:102AB000B1D014220021FEF70FFB002E3AD1019B6A
:102AC000ABF8083002220BF1080E1FFA82FC0CF161
:102AD0000100BCF1060F218C80B201D88E422BD3AD
:102AE000FFF796FEFFF778FE62691278013802F070
:102AF0001F028E4208BF4FF0400A42EA49121BFAF9
:102B000080F14AEA020A013048F0004281F808A048
:102B10008BF81000CBF8042059463846FFF798FD93
:102B2000238C0135B3422DB289F001094FF0000A20
:102B3000B8D172E70022C6E7E169895D0EF802109C
:102B40000136B6B20132C0E76FF0010565E700005B
:102B5000F8B515460E463022002104461F46FEF702
:102B6000BBFA069B6360B5F5001F079BA76034BFE7
:102B70006A094FF6FF72A36297B2E66104F1100092
:102B800000239A4206D800230360A782E3822383AE
:102B9000E360F8BD0660013330462036F1E70000FF
:102BA00003781BB94BB2002BC8BF017070470000FF
:102BB00000787047F8B50C46C969074611B9238CEF
:102BC000002B37D1257E1F2D34D8387828BB228C96
:102BD000072A2CD8268A36F003032BD14FF6FF7034
:102BE000FFF7C2FD20F001003102400441EA056117
:102BF000400C41EA40254FF6FF72234629463846ED
:102C0000FFF7EEFE002807DD626913780133DBB2BF
:102C10001F2B88BF00231370F8BD218A2D0645EABB
:102C2000012505432046FFF70FFE0246E5E76FF05A
:102C30000300F1E76FF00100EEE7000070B58AB025
:102C4000044616460021282268461D46FEF744FA2F
:102C5000BDF83830ADF810300F9B05939DF840302B
:102C60008DF81830119B07936946BDF84830ADF8D0
:102C700020302046CDE90265FFF79CFF0AB070BD09
:102C80002DE9F041D36905460C4616460BB9138C65
:102C90005BBB377E1F2F28D895F80080B8F1000F56
:102CA00026D03046FFF7D0FD3378210241EAC33108
:102CB00041EA0801338A41EA076141EA03410246D9
:102CC000334641F080012846FFF78AFE00280ADDDE
:102CD0003378012B07D1726913780133DBB21F2BD4
:102CE00088BF00231370BDE8F0816FF00100FAE7A0
:102CF0006FF00300F7E70000F0B58BB004460D4617
:102D000017460021282268461E46FEF7E5F99DF881
:102D10004C305A1E534253418DF800309DF84030DC
:102D2000ADF81030119B05939DF848308DF81830A0
:102D3000149B07936A46BDF85430ADF820302946FD
:102D40002046CDE90276FFF79BFF0BB0F0BD0000F7
:102D5000406A00B104307047436A1A6842620269EF
:102D60001A600361C38A013BC38270472DE9F041B9
:102D7000D0F82080194E14461D464146002709B957
:102D8000BDE8F081D1E90223A21A65EB0303964264
:102D900077EB03031ED2036A8B420DD1FFF77EFD52
:102DA000036A1B68036203690B60C38A0161016ADD
:102DB000013BC3828846E2E7FFF770FD0B68C8F865
:102DC000003003690B60C38A0161013BC382D8F8FC
:102DD0000010D4E788460968D1E700BF80841E0050
:102DE0002DE9F04F8BB00D46DDF8509014469B4610
:102DF0008046002800F01981B9F1000F00F015811C
:102E0000531E3F2B00F21181012A03D1BBF1000FA9
:102E100040F00B810023CDE90833B8F81430B5EB4E
:102E2000C30F4FEAC30703D300200BB0BDE8F08FF8
:102E30002B199F42D8F80C303ABF7F1BFFB22746B0
:102E40001BB9D8F81030002B7AD0272D4ED8C5F1F9
:102E50002806B7424FF000032CBFF6B23E4600935F
:102E60002946D8F8080008AB3246FFF733FCA7EB39
:102E7000060A35445FFA8AFAB8F8143003F10053B1
:102E8000053BDB000493D8F80C3003932821039B07
:102E900013B1BAF1000F2CD1D8F8100040B1BAF13B
:102EA000000F05D0009608AB5246691AFFF712FCD6
:102EB00038B2002FB8D066070AD00AAB03EBD401B2
:102EC000624211F8083C02F00702134101F8083C85
:102ED000082C3CD9102C40F2B580202C40F2B78051
:102EE000BBF1000F00F09C80082334E0BA460026B6
:102EF000C2E7049BE02B28BFE02306930B44AB42C0
:102F0000059314D95A1B03980096924534BF524634
:102F1000D2B2691A08AB04300792FFF7DBFB079ABD
:102F20001644AAEB020A1544F6B25FFA8AFA049B29
:102F3000069A05999B1A0493039B1B680393A6E7C3
:102F40000093D8F8080008AB3A462946AEE7BBF133
:102F5000000F13D00123B4EBC30F6CD0082C12D890
:102F60009DF82030621E23FA02F2D50706D54FF0F5
:102F7000FF3202FA04F423438DF820309DF820300C
:102F800089F8003051E7102C12D8BDF82030621EAD
:102F900023FA02F2D10706D54FF0FF3202FA04F409
:102FA0002343ADF82030BDF82030A9F800303CE7CD
:102FB000202C0FD80899631E21FA03F3DA0705D5F0
:102FC0004FF0FF3202FA04F40C430894089BC9F84E
:102FD00000302AE7402C2BD0DDE90865611EC4F1E2
:102FE0002102A4F1210326FA01F105FA02F225FAE1
:102FF00003F311431943CB0712D50122A4F1200397
:10300000C4F1200102FA03F322FA01F1A240524274
:1030100043EA010363EB430332432B43CDE9082327
:10302000DDE90823C9E90023FFE66FF00100FCE6B3
:103030006FF00800F9E6082CA0D9102CB3D9202C89
:10304000EED8C3E7BBF1000FADD0022383E7BBF19D
:10305000000FBBD004237EE730B5012A144638BFE9
:103060000124402C85B028BF40240025012ACDE949
:10307000025518D81B788DF8083063070AD004ABC6
:1030800003EBD405624215F8083C02F007029340B6
:1030900005F8083C009103462246002102A8FFF7EC
:1030A00019FB05B030BD082AE4D9102A03D81B88C3
:1030B000ADF80830E1E7202A8DBFD3E900231B6873
:1030C0000293CDE90223D8E710B5CB681BB98B601A
:1030D0000B618B8210BD04691A681C600361C38A8E
:1030E000013BC382CA60F0E703064CBFC0F3C030A7
:1030F0000220704708B50246FFF7F6FF022806D106
:103100005306C2F30F2001D100F0030008BDC2F343
:103110000740FBE72DE9F04F93B0CDE903230A68A0
:1031200004461046FFF7E0FF022814BFC2F306264C
:103130000026002A0D46824680F2F78112F0C0492F
:1031400040F0F381097B002900F0EF81022803D0D1
:103150002378B34240F0EC81C2F304630693104637
:1031600002F07F030593FFF7C5FF059B29444FEA53
:10317000834848EA0A4848EA4668CE780023002295
:10318000CDE90823F309834648EA0008029367D093
:10319000059B009302466768534608A92046B84736
:1031A000002800F0C881276A4FB9414604F10C009D
:1031B000FFF7F4FA074690B96FF0020054E03B695C
:1031C00098450DD03F68002FF9D1414604F10C001D
:1031D000FFF7E4FA07460028EED0236A3B60276237
:1031E00097F817C006F01F08CCF3840CACEB08006E
:1031F0001FFA80FE0028B8BF0EF12000A8EB0C03D8
:103200001FFA83FED7E90221B8BF00B2002B079353
:10321000BEBF0EF120031BB2079352EA010338D060
:10322000039BDFF824E39A1A049B4FF0000C63EB36
:10323000010196457CEB01032BD36B7B97F81AE0D9
:10324000734519D1029B002B78D0012821DC7868C6
:10325000F8B9DFF8F0C2944570EB010316D337E0FC
:10326000276A27B96FF00C0013B0BDE8F08F3B69F7
:103270009845B5D03F68F4E7B24890427CEB010333
:1032800001D30020F0E7029B002BFAD0079B0F2B05
:1032900017DCFA7DB30002F0030203F07C03134352
:1032A000FB7539462046FFF7F9FA6B7BBB76029B2C
:1032B0003BB9FB7DC3F38402013262F38603FB75E5
:1032C000D0E76A7BBB7E9A42DBD1029B002B35D0D4
:1032D000B309022B32D0039BBB60049BFB6014221A
:1032E00000210DA8FDF7F8FE039B0A93049B0B93A6
:1032F0002B1D0C932B7BADF83EB0013BDBB2ADF840
:103300003C30069B8DF84230059B8DF8433094F895
:103310002C308DF840A083F001038DF844308DF8F7
:103320004180A3680AA920469847FB7DC3F3840324
:10333000013303F01F039B02FB82A2E7FB7DC6F370
:103340004012B2EBD31F40F0F980C3F3840343452E
:1033500040F0FC80029A2B7BB609002A52D016F06E
:10336000010661D1032B40F2F480039BBB60049BF8
:10337000FB60FB8A66F30903FB822B7BAE1D033BDC
:10338000DBB23246394604F10C00FFF799FA002807
:103390000CDA39462046FFF781FAFB7DC3F384033C
:1033A000013303F01F039B02FB8205E7DDE908847C
:1033B000AB883B834FF6FF73C9F12000A9F12002CF
:1033C00028FA09F104FA00F0014324FA02F2114349
:1033D0001846C9B2FFF7B6F909F10809B9F1400F6B
:1033E0000346E9D1B8822A7B033AD2B23146FFF7CD
:1033F000BBF9FB7DB882DA43C2F3C01262F3C71394
:10340000FB753EE786B92E1D013BDBB232463946DD
:1034100004F10C00FFF754FA0028BADB2A7BB88AC3
:10342000013AD2B23146E2E7F98AC1F30901013B20
:103430000429DAB25BD8281D002307F11B069A4243
:1034400008D910F801CB06F801C001310133052974
:10345000DBB2F4D103990A9104990B91934207F1DD
:103460001B010C9138BF043379680D9134BF55FAB4
:1034700083F300230E93FB8AADF83EB0C3F3090338
:103480001A44069B8DF84230059B8DF8433094F822
:103490002C30ADF83C2083F001038DF8443000233C
:1034A0008DF840A08DF841807B602A7BB88A013A74
:1034B000291DFFF759F93B8BB882834203D1A368DA
:1034C0000AA92046984720460AA9FFF7FDFDFB7D83
:1034D000BA8AC3F38403013303F01F039B02FB8208
:1034E0003B8B9A420CBF00206FF01000BCE67B685B
:1034F000002BAFD0052001E01C3033461E68002EA3
:10350000FAD1091A081D2E1D184401EB090CBCF153
:103510001B0F5FFA89F39DD89A429BD916F8013B9D
:1035200000F8013B09F10109EFE76FF009009BE6A4
:103530006FF00A0098E66FF00B0095E66FF00D0053
:1035400092E600BF40420F0080841E006FF00E0024
:103550008AE66FF00F0087E6EFF3098305494A6BAF
:1035600022F001024A63683383F30988002383F35E
:103570001188704700EF00E0302080F3118862B6B8
:103580000C4B0D4AD96821F4E0610904090C0A4387
:10359000DA60D3F8FC20094942F08072C3F8FC20BD
:1035A0000A6842F001020A602022DA7783F82200DA
:1035B000704700BF00ED00E00003FA05001000E0D6
:1035C00010B5302383F311880E4B5B6813F400634E
:1035D00014D0F1EE103AEFF30984683C4FF0807399
:1035E000E361094BDB6B236684F3098800F090F8F4
:1035F00010B1064BA36110BD054BFBE783F31188A7
:10360000F9E700BF00ED00E000EF00E03F03000835
:103610004203000800F1604303F561430901C9B2A8
:1036200083F80013012200F01F039A4043099B0016
:1036300003F1604303F56143C3F880211A607047CA
:1036400000230375826803691B6899689142FBD265
:103650005A68036042601060586070470023037529
:10366000826803691B6899689142FBD85A680360B5
:10367000426010605860704708B50846302383F3F5
:1036800011880B7D032B05D0042B0DD02BB983F3B0
:10369000118808BD8B6900221A604FF0FF338361E7
:1036A000FFF7CEFF0023F2E7D1E9003213605A6042
:1036B000F3E70000FFF7C4BF054BD9680875186829
:1036C00002681A60536001220275D860FCF722BEBE
:1036D000384A002030B50C4BDD684B1C87B00446DF
:1036E0000FD02B46094A684600F046F92046FFF7FE
:1036F000E3FF009B13B1684600F048F9A86907B0E2
:1037000030BDFFF7D9FFF9E7384A002079360008C5
:10371000044B1A68DB6890689B68984294BF00204D
:1037200001207047384A0020084B10B51C68D86843
:1037300022681A60536001222275DC60FFF78EFF59
:1037400001462046BDE81040FCF7E4BD384A0020A1
:1037500038B5074C074908480123002523706560E8
:1037600000F024FC0223237085F3118838BD00BFCC
:10377000A04C0020F84B0008384A002008B572B66B
:10378000044B186500F0E2FA00F08AFB024B0322BA
:103790001A70FEE7384A0020A04C002000F02CB937
:1037A0008B60022308618B82084670478368A3F10F
:1037B000840243F8142C026943F8442C426943F80C
:1037C000402C094A43F8242CC26843F8182C0222E2
:1037D00003F80C2C002203F80B2C044A43F8102C9D
:1037E000A3F12000704700BF2D030008384A0020D5
:1037F00008B5FFF7DBFFBDE80840FFF75BBF00003F
:10380000024BDB6898610F20FFF756BF384A002053
:10381000302383F31188FFF7F3BF000008B501469A
:10382000302383F311880820FFF754FF002383F32C
:10383000118808BD064BDB6839B1426818605A60D0
:10384000136043600420FFF745BF4FF0FF3070471F
:10385000384A00200368984206D01A680260506017
:1038600099611846FFF726BF7047000010B503683E
:103870009C68A2420CD85C688A600B604C60216036
:10388000596099688A1A9A604FF0FF33836010BDBF
:103890001B68121BECE700000A2938BF0A2170B52B
:1038A00004460D460A26601900F07AFB00F066FB1C
:1038B000041BA54203D8751C2E460446F3E70A2EC6
:1038C00004D9BDE87040012000F0B0BB70BD00001D
:1038D000F8B5144B0D46D96103F1100141600A2A75
:1038E0001969826038BF0A22016048601861A8180F
:1038F000144600F047FB0A2700F040FB431BA3429D
:10390000064606D37C1C281900F04AFB274635469C
:10391000F2E70A2F04D9BDE8F840012000F086BB89
:10392000F8BD00BF384A0020F8B506460D4600F045
:1039300025FB0F4A134653F8107F9F4206D12A46B3
:1039400001463046BDE8F840FFF7C2BFD169BB6809
:10395000441A2C1928BF2C46A34202D92946FFF746
:103960009BFF224631460348BDE8F840FFF77EBF83
:10397000384A0020484A002010B4C0E9032300233D
:103980005DF8044B4361FFF7CFBF000010B5194C41
:10399000236998420DD0D0E90032816813605A60E3
:1039A0009A680A449A60002303604FF0FF33A361D2
:1039B00010BD2346026843F8102F536000220260B6
:1039C00022699A4203D1BDE8104000F0E3BA93683F
:1039D00081680B44936000F0D1FA2269E169926832
:1039E000441AA242E4D91144BDE81040091AFFF775
:1039F00053BF00BF384A00202DE9F047DFF8BC80F4
:103A000008F110072C4ED8F8105000F0B7FAD8F88B
:103A10001C40AA68031B9A423ED81444D5E90032E0
:103A20004FF00009C8F81C4013605A60C5F80090B8
:103A3000D8F81030B34201D100F0ACFA89F3118804
:103A4000D5E9033128469847302383F311886B6901
:103A5000002BD8D000F092FA6A69A0EB04094A451D
:103A600082460DD2022000F0E1FA0022D8F8103090
:103A7000B34208D151462846BDE8F047FFF728BFBA
:103A8000121A2244F2E712EB090938BF4A462946C6
:103A90003846FFF7EBFEB5E7D8F81030B34208D050
:103AA0001444211AC8F81C00A960BDE8F047FFF7CC
:103AB000F3BEBDE8F08700BF484A0020384A002026
:103AC00038B500F05BFA054AD2E90845031B18191E
:103AD00045F10001C2E9080138BD00BF384A0020A5
:103AE00000207047FEE70000704700004FF0FF30F5
:103AF00070470000BFF34F8F024AD368DB03FCD44A
:103B0000704700BF003C024008B5094B1B7873B9F1
:103B1000FFF7F0FF074B1A69002ABFBF064A5A6039
:103B200002F188325A601A6822F480621A6008BD75
:103B3000A84C0020003C02402301674508B50B4B10
:103B40001B7893B9FFF7D6FF094B1A6942F0004280
:103B50001A611A6842F480521A601A6822F480527C
:103B60001A601A6842F480621A6008BDA84C0020EE
:103B7000003C02400728F0B516D80C4C0C492378BD
:103B80007BB90C4D0E4608234FF0006255F8047BBC
:103B900046F8042B013B13F0FF033A44F6D101230E
:103BA000237051F82000F0BD0020FCE7CC4C002031
:103BB000AC4C0020044C0008014B53F82000704727
:103BC000044C000808207047072810B5044601D9A6
:103BD000002010BDFFF7CEFF064B53F824301844E9
:103BE000C21A0BB90120F4E712680132F0D1043B8C
:103BF000F6E700BF044C0008072810B5044621D89A
:103C0000FFF778FFFFF780FF0F4AF323D360C3006D
:103C1000DBB243F4007343F002031361136943F40E
:103C200080331361FFF766FFFFF7A4FF074B53F8DC
:103C3000241000F031F9FFF781FF2046BDE8104065
:103C4000FFF7C2BF002010BD003C0240044C00083A
:103C5000F8B512F00103144642D185182E4A954258
:103C600057D82E4B1B6813F0010352D02C4DFFF791
:103C70004BFFF323EB60FFF73DFF40F20127032CDE
:103C800015D824F001046618254C401A40F201179B
:103C9000B142236900EB010524D123F00103236124
:103CA000FFF74CFF0120F8BD043C0430E7E7830731
:103CB000E7D12B6923F440732B612B693B432B61C4
:103CC00051F8046B0660BFF34F8FFFF713FF0368D3
:103CD0009E42E9D02B6923F001032B61FFF72EFFF1
:103CE0000020E0E723F44073236123693B43236111
:103CF0000B882B80BFF34F8FFFF7FCFE2D8831F828
:103D0000023BADB2AB42C3D0236923F00103236170
:103D1000E4E71846C7E700BF000008080038024083
:103D2000003C0240084908B50B7828B11BB9FFF7E1
:103D3000EBFE01230B7008BD002BFCD0BDE8084052
:103D40000870FFF7FBBE00BFA84C002001490248E5
:103D500000F0A4B800FF030000010020084611464F
:103D600000F0A4BE084600F0B7BE000038B5EFF37F
:103D700011859DB9EFF30584C4F30804302334B1F1
:103D800083F31188FFF79CFE85F3118838BD83F318
:103D90001188FFF795FE84F3118838BDBDE83840DF
:103DA000FFF78EBE38B5FFF7E1FF114C114AC0088E
:103DB00040EA4170A0FB025EC908A0FB040C1CEBAA
:103DC000050CA1FB04404FF000035B41A1FB021274
:103DD0001CEB040C43EB000011EB0E0142F100025E
:103DE000411842F10000090941EA007038BD00BFE6
:103DF000CFF753E3A59BC42010B50244064BD2B2C3
:103E0000904200D110BD441C00B253F8200041F88C
:103E1000040BE0B2F4E700BF502800400F4B30B570
:103E20001C6F240407D41C6F44F400741C671C6FBF
:103E300044F400441C670A4C236843F480732360F5
:103E40000244084BD2B2904200D130BD441C00B2B3
:103E500051F8045B43F82050E0B2F4E70038024028
:103E6000007000405028004007B5012201A9002041
:103E7000FFF7C2FF019803B05DF804FB13B50446D9
:103E8000FFF7F2FFA04205D0012201A90020019412
:103E9000FFF7C4FF02B010BD70470000704700007C
:103EA00070470000074B45F255521A6003225A60D2
:103EB00040F2FF729A604CF6CC421A60024B01222B
:103EC0001A70704700300040D44C0020034B1B7820
:103ED0001BB1034B4AF6AA221A607047D44C00204B
:103EE00000300040034B1A681AB9034AD2F874280C
:103EF0001A607047D04C002000300240024B4FF057
:103F00008072C3F8742870470030024008B5FFF78C
:103F1000E9FF024B1868C0F3407008BDD04C002088
:103F200008B5FFF7DFFF024B1868C0F3007008BD4B
:103F3000D04C002070470000FEE700000A4B0B4801
:103F40000B4A90420BD30B4BDA1C121AC11E22F003
:103F500003028B4238BF00220021FDF7BDB853F8A1
:103F6000041B40F8041BECE7B84D00083052002059
:103F7000305200203052002000F0CAB84FF0804389
:103F8000586A70474FF08043002258631A6102223A
:103F9000DA6070474FF080430022DA60704700001B
:103FA0004FF0804358637047FEE7000070B51B4B2D
:103FB00001630025044686B0586085620E46FFF70F
:103FC000DBFA04F11003C4E904334FF0FF33C4E912
:103FD0000635C4E90044A560E562FFF7CFFF2B4634
:103FE0000246C4E9082304F134010D4A2565802303
:103FF0002046FFF7D5FB0123E0600A4A03750092D3
:1040000072680192B268CDE90223074B6846CDE998
:104010000435FFF7EDFB06B070BD00BFA04C0020DB
:10402000244C0008294C0008A93F0008024AD36A22
:104030001843D062704700BF384A00204B68436085
:104040008B688360CB68C3600B6943614B69036213
:104050008B6943620B6803607047000008B5234B0F
:1040600023481A6942F0FF021A611A6922F0FF021E
:104070001A611A691A6B42F0FF021A631A6D42F054
:10408000FF021A651B4A1B6D1146FFF7D7FF02F1AD
:104090001C0100F58060FFF7D1FF02F1380100F547
:1040A0008060FFF7CBFF02F1540100F58060FFF75D
:1040B000C5FF02F1700100F58060FFF7BFFF02F15C
:1040C0008C0100F58060FFF7B9FF02F1A80100F54F
:1040D0008060FFF7B3FF02F1C40100F58060FFF7D5
:1040E000ADFFBDE8084000F08DB800BF00380240C9
:1040F00000000240304C000808B500F027FAFFF736
:1041000027FBBDE80840FFF7EDBE00007047000048
:104110000F4B1A6C42F001021A641A6E42F001024F
:104120001A660C4A1B6E936843F0010393604FF0CC
:10413000804331229A624FF0FF32DA6200229A61A4
:104140005A63DA605A6001225A611A60704700BFF0
:1041500000380240002004E04FF0804208B51169A9
:10416000D3680B40D9B2C9439B07116107D53023EF
:1041700083F31188FFF712FB002383F3118808BD36
:104180001E4B1A6962F0FF021A611A69D2B21A61F3
:104190004FF0FF301A695A69586100215A69596114
:1041A0005A691A6A62F080521A621A6A02F08052E0
:1041B0001A621A6A5A6A58625A6A59625A6A1A6CB8
:1041C00042F080521A641A6E42F080521A661A6ED9
:1041D0000B4A106840F480701060186F00F4407053
:1041E000B0F5007F1EBF4FF4803018671967536821
:1041F00023F40073536000F07DB900BF0038024023
:10420000007000403B4B3C4A1A643C4A4FF440412A
:1042100011601A6842F001021A601A689007FCD512
:104220009A6822F003029A60324B9A6812F00C02EC
:10423000FBD1196801F0F90119609A601A6842F41B
:1042400080321A601A689103FCD55A6F42F001025D
:104250005A67284B5A6F9207FCD5294A5A601A6848
:1042600042F080721A60254A53685804FCD5214BED
:104270001A689101FCD5234AC3F884201A6842F0D9
:1042800080621A601A681201FCD51F4A9A600322E4
:10429000C3F88C204FF00062C3F894201B4B1A68BF
:1042A0001B4B9A421B4B21D11B4A11681B4A91425E
:1042B0001CD140F203121A60164A136803F00F0370
:1042C000032BFAD10B4B9A6842F002029A609A686B
:1042D00002F00C02082AFAD15A6C42F480425A6465
:1042E0005A6E42F480425A665B6E704740F2037227
:1042F000E1E700BF003802400004001000700040F9
:10430000081940021030002400948838002004E08E
:1043100011640020003C024000ED00E041C20F416A
:10432000074A08B5536903F00103536123B1054AF5
:1043300013680BB150689847BDE80840FFF740B9D3
:10434000003C0140D84C0020074A08B5536903F0EF
:104350000203536123B1054A93680BB1D0689847B3
:10436000BDE80840FFF72CB9003C0140D84C0020C4
:10437000074A08B5536903F00403536123B1054AA2
:1043800013690BB150699847BDE80840FFF718B9A9
:10439000003C0140D84C0020074A08B5536903F09F
:1043A0000803536123B1054A93690BB1D06998475B
:1043B000BDE80840FFF704B9003C0140D84C00209C
:1043C000074A08B5536903F01003536123B1054A46
:1043D000136A0BB1506A9847BDE80840FFF7F0B880
:1043E000003C0140D84C0020164B10B55C6904F429
:1043F00078725A61A30604D5134A936A0BB1D06A46
:104400009847600604D5104A136B0BB1506B984760
:10441000210604D50C4A936B0BB1D06B9847E2058B
:1044200004D5094A136C0BB1506C9847A30504D509
:10443000054A936C0BB1D06C9847BDE81040FFF76C
:10444000BFB800BF003C0140D84C0020194B10B54C
:104450005C6904F47C425A61620504D5164A136D06
:104460000BB1506D9847230504D5134A936D0BB1DA
:10447000D06D9847E00404D50F4A136E0BB1506E0F
:104480009847A10404D50C4A936E0BB1D06E98479F
:10449000620404D5084A136F0BB1506F9847230488
:1044A00004D5054A936F0BB1D06F9847BDE8104013
:1044B000FFF786B8003C0140D84C002008B50348FF
:1044C00000F010F9BDE80840FFF77AB8584D002019
:1044D00008B5034800F006F9BDE80840FFF770B8DA
:1044E000C44F002008B5FFF737FEBDE80840FFF7CE
:1044F00067B80000062108B50846FFF78BF80621CB
:104500000720FFF787F806210820FFF783F8062128
:104510000920FFF77FF806210A20FFF77BF8062124
:104520001720FFF777F806212820FFF773F80721F7
:104530001C20FFF76FF80C212520FFF76BF8BDE872
:1045400008400C212620FFF765B8000008B5FFF7EA
:1045500017FE00F07BF800F03DF8FFF7D7FDBDE84F
:104560000840FFF709BD000002684368114301607D
:1045700003B1184770470000143000F0DFB90000A5
:104580004FF0FF33143000F0D9B90000383000F09C
:1045900055BA00004FF0FF33383000F04FBA00003A
:1045A000143000F0A5B900004FF0FF31143000F0D6
:1045B0009FB90000383000F0FFB900004FF0FF3223
:1045C000383000F0F9B90000012914BF6FF0130072
:1045D0000020704700F060B837B515460E4A0260FB
:1045E00000224260C0E902220122044602740B4606
:1045F000009000F15C014FF48072143000F04EF92D
:1046000000942B464FF4807204F5AE7104F138002B
:1046100000F0C6F903B030BD104D000838B5C369CD
:1046200004460D461BB904210844FFF79DFF2946A7
:1046300004F1140000F040F9002806DA201D4FF4C0
:104640000061BDE83840FFF78FBF38BD0023054A41
:1046500019460133102BC2E9001102F10802F8D10A
:10466000704700BFD84C00200268436811430160C6
:1046700003B1184770470000024AD36843F0C003F3
:10468000D360704700100140024AD36843F0C00372
:10469000D36070470044004010B50A4C0A4A2046D7
:1046A0000021FFF799FF094B094AC4E99723094CF8
:1046B000094A00212046FFF78FFF0849084BC4E94B
:1046C000971310BD584D00207946000880F0FA027B
:1046D00000100140C44F00208946000800440040FB
:1046E00040787D012DE9F041D0F85C62F7683368CD
:1046F000DA0504469DB20DD5302383F311884FF4BB
:1047000080610430FFF7B0FF6FF4807333600023E3
:1047100083F31188302383F3118804F1040815F022
:104720002F033AD183F31188380615D5290613D5FE
:10473000302383F3118804F1380000F065F9002874
:104740004EDA0821201DFFF78FFF4FF67F733B40A5
:10475000F360002383F311887A0616D56B0614D50F
:10476000302383F31188D4E913239A420AD1236CAE
:1047700043B127F040073F041021201D3F0CFFF7F5
:1047800073FFF760002383F31188D4F86822D3689D
:1047900043B3BDE8F041106918472B0714D015F05A
:1047A000080F0CBF00214FF48071E80748BF41F0AB
:1047B0002001AA0748BF41F040016B0748BF41F004
:1047C00080014046FFF750FFAD06736805D594F8A9
:1047D000641220461940FFF721FF3568ADB29EE70D
:1047E0007060B6E7BDE8F081F8B5154682680669E5
:1047F000AA420B46816938BF8568761AB5420446DD
:104800000BD218462A46FCF755FCA3692B44A3613A
:10481000A3685B1BA3602846F8BD0CD91846324636
:10482000FCF748FCAF1BE1683A463044FCF742FC19
:10483000E3683B44EBE718462A46FCF73BFCE36899
:10484000E5E7000083689342F7B51546044638BF94
:104850008568D0E90460361AB5420BD22A46FCF7C7
:1048600029FC63692B446361A36828465B1BA36032
:1048700003B0F0BD0DD932460191FCF71BFC019944
:10488000E068AF1B3A463144FCF714FCE3683B4454
:10489000E9E72A46FCF70EFCE368E4E710B50A44B2
:1048A0000024C361029B8460C0E90000C0E90511D7
:1048B000C1600261036210BD08B5D0E905329342C0
:1048C00001D1826882B98268013282605A1C4261D9
:1048D0001970D0E904329A4224BFC36843610021B1
:1048E000FEF7B8FF002008BD4FF0FF30FBE70000E7
:1048F00070B5302304460E4683F31188A568A5B130
:10490000A368A269013BA360531CA36115782269C7
:10491000934224BFE368A361E3690BB12046984743
:10492000002383F31188284607E031462046FEF72E
:1049300081FF0028E2DA85F3118870BD2DE9F74F79
:1049400004460E4617469846D0F81C904FF0300AA1
:104950008AF311884FF0000B154665B12A4631469F
:104960002046FFF741FF034660B941462046FEF767
:1049700061FF0028F1D0002383F31188781B03B076
:10498000BDE8F08FB9F1000F03D001902046C84771
:10499000019B8BF31188ED1A1E448AF31188DCE722
:1049A000C0E90511C160C3611144009B8260C0E988
:1049B0000000016103627047F8B504460D461646D3
:1049C000302383F31188A768A7B1A368013BA360D4
:1049D00063695A1C62611D70D4E904329A4224BF93
:1049E000E3686361E3690BB120469847002080F3D8
:1049F000118807E031462046FEF71CFF0028E2DA66
:104A000087F31188F8BD0000D0E905239A4210B55C
:104A100001D182687AB98268013282605A1C82614F
:104A20001C7803699A4224BFC36883610021FEF7A2
:104A300011FF204610BD4FF0FF30FBE72DE9F74F87
:104A400004460E4617469846D0F81C904FF0300AA0
:104A50008AF311884FF0000B154665B12A4631469E
:104A60002046FFF7EFFE034660B941462046FEF7B9
:104A7000E1FE0028F1D0002383F31188781B03B0F6
:104A8000BDE8F08FB9F1000F03D001902046C84770
:104A9000019B8BF31188ED1A1E448AF31188DCE721
:104AA0000B460146184600F009B80000024B0A46C2
:104AB00001461868FFF752B91C23002010B5054CB9
:104AC00013462CB10A4601460220AFF3008010BD08
:104AD0002046FCE700000000024B01461868FFF783
:104AE00041B900BF1C23002010B501390244904297
:104AF00001D1002005E0037811F8014FA34201D055
:104B0000181B10BD0130F2E72DE9F041A3B1C91A1D
:104B100017780144044603F1FF3C8C42204601D93A
:104B2000002009E00578BD4204F10104F5D10CEB49
:104B30000405D618A54201D1BDE8F08115F8018D14
:104B400016F801EDF045F5D0E7E70000034611F84F
:104B5000012B03F8012B002AF9D170476F72672EE1
:104B60006172647570696C6F742E435541565F476E
:104B70005053000040A2E4F1646891060041A3E5AF
:104B8000F2656992070000004261642043414E498A
:104B90006661636520696E6465782E0080000000A0
:104BA0000080000000008000000000000000000005
:104BB000BD190008012200085D210008FD19000848
:104BC000091A0008151C0008CD190008DD19000895
:104BD000D1190008D9190008D5190008311B00089F
:104BE000E119000825250008D5240008F11900085E
:104BF000051B000863300000F44B0008904A0020B9
:104C0000A04C0020004000000040000000400000D8
:104C1000004000000000010000000200000002004F
:104C2000000002006D61696E0069646C650000003F
:104C3000A001102800000000AAAAAAAA500110246E
:104C4000FFFF0000007700000000000000A40A0140
:104C500000000000AAA6AAAA80500000DFEF000012
:104C60000000007788000000000000000000000045
:104C7000AAAAAAAA00000000FFFF0000000000008E
:104C8000000000000000000000000000AAAAAAAA7C
:104C900000000000FFFF0000000000000000000016
:104CA0000000000000000000AAAAAAAA000000005C
:104CB000FFFF0000000000000000000000000000F6
:104CC00000000000AAAAAAAA00000000FFFF00003E
:104CD00000000000000000000000000000000000D4
:104CE000AAAAAAAA00000000FFFF0000000000001E
:104CF0000000000000000000000000000A000000AA
:104D000000000000030000000000000000000000A0
:104D1000000000009545000881450008BD450008D9
:104D2000A9450008B5450008A14500088D450008C3
:104D300079450008C9450008E903000000000000AB
:104D4000000007000000000040420F00FE2A0100A2
:104D5000D20400002023002000000000000000001A
:104D60000000000000000000000000000000000043
:104D70000000000000000000000000000000000033
:104D80000000000000000000000000000000000023
:104D90000000000000000000000000000000000013
:104DA0000000000000000000000000000000000003
:104DB0000000000000000000FFFFFFFFFFFFFFFFFB
:104DC000FFFFFFFFFFFFFFFFFFFFFFFFFFFFFFFFF3
:104DD000FFFFFFFFFFFFFFFFFFFFFFFFFFFFFFFFE3
:104DE000FFFFFFFFFFFFFFFFFFFFFFFFFFFFFFFFD3
:104DF000FFFFFFFFFFFFFFFFFFFFFFFFFFFFFFFFC3
:020000040801F1
:10000000000700208D120108B11102080D1102082D
:10001000791102080D110208451102088F1201081A
:100020008F1201088F1201088F12010865CE020895
:100030008F1201088F1201088F1201088F12010818
:100040008F1201088F1201088F1201088F12010808
:100050008F1201088F120108CD080308F508030864
:100060001D090308450903086D090308E5D30208C3
:100070000DD4020839D4020865D4020891D40208CC
:10008000B9D40208E5D402088F12010869050208F4
:1000900095050208A50502088F12010895090308B5
:1000A0008F1201088F1201088F1201088F120108A8
:1000B000910A0308A50A03088F1201088F1201088C
:1000C0008F1201088F1201088F1201088F12010888
:1000D0008F120108690A03087D0A03088F120108BC
:1000E000F90903088F1201088F1201088F12010805
:1000F0008F1201088F1201088F12010811D5020812
:100100008F1201088F120108B90A03088F12010823
:100110008F1201088F1201088F1201088F12010837
:100120003DD5020865D5020891D50208BDD5020863
:10013000E9D502088F1201088F1201088F120108F9
:100140008F1201088F1201088F1201088F12010807
:1001500011D602083DD6020869D602088F1201089E
:1001600071DA020819DC02088F1201088F120108E7
:100170008F1201088F1201088F1201088F120108D7
:100180008F1201088F1201088F1201088F120108C7
:100190008F1201088F1201088F1201088F120108B7
:1001A0008F1201088F1201088F1201088F120108A7
:1001B0008F1201088F1201088F1201088F12010897
:1001C0008F1201088F1201088F1201088F12010887
:1001D0008F1201088F1201088F1201088F12010877
:1001E000B519010801830108B1E60108DD0A02081A
:1001F0007D1302083D6902082987020881900208E0
:10020000F5B5020845BB020895BC020800000000D5
:1002100040A2E4F164689106B21573FB0CF18A37D1
:10022000F8E6020003BEC5930000E903FFFFFFFFED
:10023000FFFFFFFF81F0004102E000BF83F00043B9
:1002400030B54FEA41044FEA430594EA050F08BF71
:1002500090EA020F1FBF54EA000C55EA020C7FEA35
:10026000645C7FEA655C00F0E2804FEA5454D4EBB2
:100270005555B8BF6D420CDD2C4480EA020281EA7C
:10028000030382EA000083EA010180EA020281EAB4
:100290000303362D88BF30BD11F0004F4FEA013106
:1002A0004FF4801C4CEA113102D0404261EB410115
:1002B00013F0004F4FEA03334CEA133302D052429B
:1002C00063EB430394EA050F00F0A780A4F1010457
:1002D000D5F1200E0DDB02FA0EFC22FA05F2801891
:1002E00041F1000103FA0EF2801843FA05F3594177
:1002F0000EE0A5F120050EF1200E012A03FA0EFCF6
:1003000028BF4CF0020C43FA05F3C01851EBE3711F
:1003100001F0004507D54FF0000EDCF1000C7EEB3C
:1003200000006EEB0101B1F5801F1BD3B1F5001F7A
:100330000CD349085FEA30004FEA3C0C04F1010499
:100340004FEA445212F5800F80F09A80BCF1004FC2
:1003500008BF5FEA500C50F1000041EB045141EA44
:10036000050130BD5FEA4C0C404141EB0101013C0D
:1003700028BFB1F5801FE9D291F0000F04BF0146FC
:100380000020B1FA81F308BF2033A3F10B03B3F1CE
:1003900020020CDA0C3208DD02F1140CC2F10C025E
:1003A00001FA0CF021FA02F10CE002F11402D8BFBC
:1003B000C2F1200C01FA02F120FA0CFCDCBF41EA88
:1003C0000C019040E41AA2BF01EB0451294330BD57
:1003D0006FEA04041F3C1CDA0C340EDC04F1140434
:1003E000C4F1200220FA04F001FA02F340EA03000B
:1003F00021FA04F345EA030130BDC4F10C04C4F151
:10040000200220FA02F001FA04F340EA0300294630
:1004100030BD21FA04F0294630BD94F0000F83F47A
:10042000801306BF81F480110134013D4EE77FEA5D
:10043000645C18BF7FEA655C29D094EA050F08BFA9
:1004400090EA020F05D054EA000C04BF194610468A
:1004500030BD91EA030F1EBF0021002030BD5FEACE
:10046000545C05D14000494128BF41F0004130BDF6
:1004700014F580043CBF01F5801130BD01F000454A
:1004800045F0FE4141F470014FF0000030BD7FEABD
:10049000645C1ABF194610467FEA655C1CBF0B46B8
:1004A000024650EA013406BF52EA033591EA030FCF
:1004B00041F4002130BD00BF90F0000F04BF0021C7
:1004C000704730B54FF4806404F132044FF00005FA
:1004D0004FF0000150E700BF90F0000F04BF002173
:1004E000704730B54FF4806404F1320410F00045D9
:1004F00048BF40424FF000013EE700BF42004FEAD4
:10050000E2014FEA31014FEA02701FBF12F07F4350
:1005100093F07F4F81F06051704732F07F4208BF07
:10052000704793F07F4F04BF41F40021704730B50E
:100530004FF4607401F0004521F000411CE700BF5A
:1005400050EA010208BF704730B54FF000050AE0DD
:1005500050EA010208BF704730B511F0004502D5DE
:10056000404261EB41014FF4806404F132045FEAE0
:10057000915C3FF4D8AE4FF003025FEADC0C18BF89
:1005800003325FEADC0C18BF033202EBDC02C2F17B
:10059000200300FA03FC20FA02F001FA03FE40EA0D
:1005A0000E0021FA02F11444BDE600BF70B54FF011
:1005B000FF0C4CF4E06C1CEA11541DBF1CEA1355EF
:1005C00094EA0C0F95EA0C0F00F0DEF82C4481EA57
:1005D000030621EA4C5123EA4C5350EA013518BF77
:1005E00052EA033541F4801143F4801338D0A0FB64
:1005F00002CE4FF00005E1FB02E506F00042E0FB11
:1006000003E54FF00006E1FB03569CF0000F18BF16
:100610004EF0010EA4F1FF04B6F5007F64F54074BE
:1006200004D25FEA4E0E6D4146EB060642EAC62151
:1006300041EA55514FEAC52040EA5E504FEACE2EBE
:10064000B4F1FD0C88BFBCF5E06F1ED8BEF1004FC1
:1006500008BF5FEA500E50F1000041EB045170BD3D
:1006600006F0004646EA010140EA020081EA030181
:10067000B4EB5C04C2BFD4EB0C0541EA045170BD7D
:1006800041F480114FF0000E013C00F3AB8014F1F7
:10069000360FDEBF002001F0004170BDC4F1000440
:1006A000203C35DA0C341BDC04F11404C4F12005C1
:1006B00000FA05F320FA04F001FA05F240EA02001C
:1006C00001F0004221F0004110EBD37021FA04F652
:1006D00042EB06015EEA430E08BF20EAD37070BD0C
:1006E000C4F10C04C4F1200500FA04F320FA05F06B
:1006F00001FA04F240EA020001F0004110EBD3706D
:1007000041F100015EEA430E08BF20EAD37070BDDC
:10071000C4F1200500FA05F24EEA020E20FA04F3B5
:1007200001FA05F243EA020321FA04F001F0004164
:1007300021FA04F220EA020000EBD3705EEA430ED5
:1007400008BF20EAD37070BD94F0000F0FD101F004
:100750000046400041EB010111F4801F08BF013C3D
:10076000F7D041EA060195F0000F18BF704703F07B
:100770000046520043EB030313F4801F08BF013D02
:10078000F7D043EA0603704794EA0C0F0CEA1355BE
:1007900018BF95EA0C0F0CD050EA410618BF52EA78
:1007A0004306D1D181EA030101F000414FF000007E
:1007B00070BD50EA410606BF1046194652EA43068C
:1007C00019D094EA0C0F02D150EA013613D195EA00
:1007D0000C0F05D152EA03361CBF104619460AD148
:1007E00081EA030101F0004141F0FE4141F4700152
:1007F0004FF0000070BD41F0FE4141F4780170BD42
:1008000070B54FF0FF0C4CF4E06C1CEA11541DBFA6
:100810001CEA135594EA0C0F95EA0C0F00F0A7F8A8
:10082000A4EB050481EA030E52EA03354FEA0131D5
:1008300000F088804FEA03334FF0805545EA1313E8
:1008400043EA12634FEA022245EA111545EA1065B0
:100850004FEA00260EF000419D4208BF964244F147
:10086000FD0404F5407402D25B084FEA3202B61A66
:1008700065EB03055B084FEA32024FF480104FF43A
:10088000002CB6EB020E75EB030E22BFB61A7546AE
:1008900040EA0C005B084FEA3202B6EB020E75EB41
:1008A000030E22BFB61A754640EA5C005B084FEAA9
:1008B0003202B6EB020E75EB030E22BFB61A754676
:1008C00040EA9C005B084FEA3202B6EB020E75EB81
:1008D000030E22BFB61A754640EADC0055EA060E42
:1008E00018D04FEA051545EA16754FEA06164FEA85
:1008F000C30343EA52734FEAC2025FEA1C1CC0D131
:1009000011F4801F0BD141EA00014FF000004FF0BD
:10091000004CB6E711F4801F04BF01430020B4F17E
:10092000FD0C88BFBCF5E06F3FF6AFAEB5EB030C36
:1009300004BFB6EB020C5FEA500C50F1000041EB33
:10094000045170BD0EF0004E4EEA113114EB5C0400
:10095000C2BFD4EB0C0541EA045170BD41F48011D3
:100960004FF0000E013C90E645EA060E8DE60CEADB
:10097000135594EA0C0F08BF95EA0C0F3FF43BAFF8
:1009800094EA0C0F0AD150EA01347FF434AF95EAAF
:100990000C0F7FF425AF104619462CE795EA0C0F93
:1009A00006D152EA03353FF4FDAE1046194622E760
:1009B00050EA410618BF52EA43067FF4C5AE50EA3A
:1009C00041047FF40DAF52EA43057FF4EBAE12E72A
:1009D0004FF0FF3C06E000BF4FF0010C02E000BF0B
:1009E0004FF0010C4DF804CD4FEA410C7FEA6C5CEE
:1009F0004FEA430C18BF7FEA6C5C1BD001B050EA91
:100A0000410C0CBF52EA430C91EA030F02BF90EA7B
:100A1000020F0020704710F1000F91EA030F58BF3A
:100A2000994208BF90422CBFD8176FEAE37040F09C
:100A3000010070474FEA410C7FEA6C5C02D150EA3A
:100A4000013C07D14FEA430C7FEA6C5CD6D152EAF5
:100A5000033CD3D05DF8040B704700BF84461046BA
:100A600062468C461946634600E000BF01B5FFF7B9
:100A7000B7FF002848BF10F1000F01BD4DF808ED89
:100A8000FFF7F4FF0CBF012000205DF808FB00BF5A
:100A90004DF808EDFFF7EAFF34BF012000205DF8B4
:100AA00008FB00BF4DF808EDFFF7E0FF94BF012001
:100AB00000205DF808FB00BF4DF808EDFFF7CEFF02
:100AC00094BF012000205DF808FB00BF4DF808ED41
:100AD000FFF7C4FF34BF012000205DF808FB00BF12
:100AE0004FEA410C7FEA6C5C02D150EA013C0AD12A
:100AF0004FEA430C7FEA6C5C02D152EA033C02D11C
:100B00004FF0000070474FF0010070474FEA41027C
:100B100012F5001215D211D56FF47873B3EB62524F
:100B200012D94FEAC12343F0004343EA505311F076
:100B3000004F23FA02F018BF404270474FF0000008
:100B4000704750EA013005D111F0004008BF6FF046
:100B5000004070474FF00000704700BF4A0011D2BC
:100B600012F5001211D20DD56FF47873B3EB625207
:100B70000ED44FEAC12343F0004343EA505323FA13
:100B800002F070474FF00000704750EA013002D188
:100B90004FF0FF3070474FF0000070474FEA4102BE
:100BA000B2F1E04324BFB3F5001CDCF1FE5C0DD9CB
:100BB00001F0004C4FEAC0024CEA5070B2F1004F15
:100BC00040EB830008BF20F00100704711F0804F18
:100BD00021D113F13872BCBF01F00040704741F4DD
:100BE00080114FEA5252C2F11802C2F1200C10FAE1
:100BF0000CF320FA02F018BF40F001004FEAC123C5
:100C00004FEAD32303FA0CFC40EA0C0023FA02F368
:100C10004FEA4303CCE77FEA625307D150EA01333E
:100C20001EBF4FF0FE4040F44000704701F000400E
:100C300040F0FE4040F40000704700BF80F00040EC
:100C400002E000BF81F0004142001FBF5FEA4103A4
:100C500092EA030F7FEA226C7FEA236C6AD04FEAA4
:100C60001262D2EB1363C1BFD218414048404140E9
:100C7000B8BF5B42192B88BF704710F0004F40F49B
:100C8000000020F07F4018BF404211F0004F41F4B7
:100C9000000121F07F4118BF494292EA030F3FD083
:100CA000A2F1010241FA03FC10EB0C00C3F1200396
:100CB00001FA03F100F0004302D5494260EB400025
:100CC000B0F5000F13D3B0F1807F06D340084FEA90
:100CD000310102F10102FE2A51D2B1F1004F40EB85
:100CE000C25008BF20F0010040EA030070474900ED
:100CF00040EB0000013A28BFB0F5000FEDD2B0FA8A
:100D000080FCACF1080CB2EB0C0200FA0CF0AABFAC
:100D100000EBC25052421843BCBFD040184370474A
:100D200092F0000F81F4000106BF80F40000013250
:100D3000013BB5E74FEA41037FEA226C18BF7FEA27
:100D4000236C21D092EA030F04D092F0000F08BF69
:100D50000846704790EA010F1CBF0020704712F050
:100D60007F4F04D1400028BF40F00040704712F18F
:100D700000723CBF00F50000704700F0004343F0F4
:100D8000FE4040F4000070477FEA226216BF08462A
:100D90007FEA23630146420206BF5FEA412390EAED
:100DA000010F40F4800070474FF0000304E000BFE3
:100DB00010F0004348BF40425FEA000C08BF704794
:100DC00043F0964301464FF000001CE050EA010258
:100DD00008BF70474FF000030AE000BF50EA01026D
:100DE00008BF704711F0004302D5404261EB41015A
:100DF0005FEA010C02BF84460146002043F0B6437F
:100E000008BFA3F18053A3F50003BCFA8CF2083AA3
:100E1000A3EBC25310DB01FA02FC634400FA02FCAC
:100E2000C2F12002BCF1004F20FA02F243EB0200B3
:100E300008BF20F00100704702F1200201FA02FC15
:100E4000C2F1200250EA4C0021FA02F243EB020008
:100E500008BF20EADC7070477BB972B90029BEBFB9
:100E600000204FF0004106E008BF00281CBF6FF0D3
:100E700000414FF0FF3000F007BAADF1080C6DE90A
:100E800004CE002909DB002B1ADB00F095F8DDF811
:100E900004E0DDE9022304B07047404261EB410108
:100EA000002B1BDB00F088F8DDF804E0DDE902230D
:100EB00004B0404261EB4101524263EB430370478F
:100EC000524263EB430300F077F8DDF804E0DDE91C
:100ED000022304B0404261EB41017047524263EB90
:100EE000430300F069F8DDF804E0DDE9022304B013
:100EF000524263EB4303704753B94AB9002908BF14
:100F000000281CBF4FF0FF314FF0FF3000F0BCB99C
:100F1000ADF1080C6DE904CE00F04EF8DDF804E008
:100F2000DDE9022304B07047430803F05533C01ACB
:100F3000830803F0333300F03330184400EB101013
:100F400000F00F3000EB002000EB0040000E704777
:100F500007EE900AF5EEC07AF1EE10FA01D400F037
:100F60000BB8F1EE677A08B517EE900A00F004F8B6
:100F7000404261EB410108BDD0B5FFF7BFFA0C4B11
:100F8000002206460F46FFF711FBFFF7E7FD044678
:100F9000FFF792FA074B0022FFF708FB02460B46C9
:100FA00030463946FFF74AF9FFF7D8FD2146D0BD54
:100FB0000000F03D0000F0412DE9F047089D044697
:100FC0008E46002B4DD18A42944669D9B2FA82F2FC
:100FD00052B101FA02F3C2F1200120FA01F10CFA38
:100FE00002FC41EA030E94404FEA1C48210CBEFB70
:100FF000F8F61FFA8CF708FB16E341EA034306FBF9
:1010000007F199420AD91CEB030306F1FF3080F087
:101010001F81994240F21C81023E63445B1AA4B2D4
:10102000B3FBF8F008FB103344EA034400FB07F776
:10103000A7420AD91CEB040400F1FF3380F00A81B7
:10104000A74240F207816444023840EA0640E41BAC
:1010500000261DB1D4400023C5E900433146BDE858
:10106000F0878B4209D9002D00F0EF800026C5E9FA
:10107000000130463146BDE8F087B3FA83F6002E12
:101080004AD18B4202D3824200F2F980841A61EB8A
:10109000030301209E46002DE0D0C5E9004EDDE7A8
:1010A00002B9FFDEB2FA82F2002A40F09280A1EB90
:1010B0000C014FEA1C471FFA8CFE0126200CB1FBE5
:1010C000F7F307FB131140EA01410EFB03F08842DE
:1010D00008D91CEB010103F1FF3802D2884200F26B
:1010E000CB804346091AA4B2B1FBF7F007FB1011FD
:1010F00044EA01440EFB00FEA64508D91CEB04049B
:1011000000F1FF3102D2A64500F2BB800846A4EBF5
:101110000E0440EA03409CE7C6F12007B34022FAE0
:1011200007FC4CEA030C20FA07F401FA06F31C430F
:10113000F9404FEA1C4900FA06F3B1FBF9F8200C1C
:101140001FFA8CFE09FB181140EA014108FB0EF062
:10115000884202FA06F20BD91CEB010108F1FF3AB2
:1011600080F08880884240F28580A8F102086144BE
:10117000091AA4B2B1FBF9F009FB101144EA0141CC
:1011800000FB0EFE8E4508D91CEB010100F1FF3477
:101190006CD28E456AD90238614440EA0840A0FB0F
:1011A0000294A1EB0E01A142C846A64656D353D0E5
:1011B0005DB1B3EB080261EB0E0101FA07F722FA09
:1011C00006F3F1401F43C5E9007100263146BDE832
:1011D000F087C2F12003D8400CFA02FC21FA03F395
:1011E000914001434FEA1C471FFA8CFEB3FBF7F016
:1011F00007FB10360B0C43EA064300FB0EF69E423B
:1012000004FA02F408D91CEB030300F1FF382FD2D3
:101210009E422DD9023863449B1B89B2B3FBF7F67B
:1012200007FB163341EA034106FB0EF38B4208D954
:101230001CEB010106F1FF3816D28B4214D9023E95
:101240006144C91A46EA004638E72E46284605E7B3
:101250000646E3E61846F8E64B45A9D2B9EB020884
:1012600064EB0C0E0138A3E74646EAE7204694E714
:101270004046D1E7D0467BE7023B614432E7304647
:1012800009E76444023842E7704700BF02E000F01B
:1012900000F8FEE772B6374880F30888364880F3D6
:1012A000098836483649086040F20000CCF2000058
:1012B0004EF63471CEF200010860BFF34F8FBFF3DA
:1012C0006F8F40F20000C0F2F0004EF68851CEF26F
:1012D00000010860BFF34F8FBFF36F8F4FF0000026
:1012E000E1EE100A4EF63C71CEF2000108600620D5
:1012F00080F31488BFF36F8F1FF082F81FF07AF924
:101300004FF055301F491B4A91423CBF41F8040B36
:10131000FAE71D49184A91423CBF41F8040BFAE72D
:101320001A491B4A1B4B9A423EBF51F8040B42F824
:10133000040BF8E700201849184A91423CBF41F8D5
:10134000040BFAE71FF060F81FF0A2F9144C154DDA
:10135000AC4203DA54F8041B8847F9E700F01AFBA3
:10136000114C124DAC4203DA54F8041B8847F9E7DC
:101370001FF048B8000700200023002000000108EB
:1013800008ED00E00001002000070020F8E303085A
:1013900000230020002600200026002020930020AB
:1013A000E00101080C0201080C0201080C0201080E
:1013B0002DE9F04F2DED108AC1F80CD0C3689D4681
:1013C000BDEC108ABDE8F08F002383F31188284616
:1013D000A04700201EF046FAFEE71EF0E5F800DF09
:1013E000FEE7000010F8012B11F8013B012A28BF8D
:1013F0009A42F7D0D01A7047034613F8012B002AFF
:10140000FBD1181A0138704701F0FF01102A2BDBBD
:1014100010F0070F08D010F8013B013A8B422DD095
:1014200010F0070F42B3F6D1F0B441EA012141EACE
:10143000014122F007047FF000070023F0E8025684
:10144000083C85EA010586EA010685FA47F5A3FA14
:1014500087F586FA47F6A5FA87F68EB9EED1F0BC85
:1014600001F0FF0102F0070232B110F8013B013A2E
:1014700083EA010313B1F8D10020704701387047A7
:10148000002D06BF35460338073815F0010F07D188
:10149000013015F4807F02BF013015F4C03F0130E8
:1014A000F0BC0138704700BF38B500220023044665
:1014B0000D46FFF7EDFA28B920462946BDE8384029
:1014C00000F00AB8204605F1004100F005F840425E
:1014D00061EB410138BD00BFD0B50C4B0022064680
:1014E0000F46FFF763F8FFF739FB0446FEF7E4FF0A
:1014F000074B0022FFF75AF802460B4630463946A2
:10150000FEF79CFEFFF72AFB2146D0BD0000F03D10
:101510000000F0417047000070B504461C300BF02D
:10152000C3F804F1400007F083F804F5C0700BF035
:1015300001FB04F522700CF037F9154B15491960C1
:1015400004F56A70002314269DB206FB05120133D0
:10155000127C002AF8D1104B1D80104B1A6812B172
:101560000F480FF029FE186004F58053012104F59F
:101570009D50C3F8B82383F8B6131C300FF05CF805
:10158000084B1A680AB10848EBE71C60204670BD9A
:10159000C83A0020686D0308C63A0020883A002047
:1015A000546C0308042600206F6C0308F0B5354D19
:1015B00085B004461EF0DAFE1EF0ECFE28682023FB
:1015C0001A46006C4FF4614103F004FC28684FF4A4
:1015D000807380224FF4E131C06C03F0FBFB2046A6
:1015E00000F00CFA04F11C071EF0D4FE204601F0B6
:1015F00047FB38460BF066F91EF0CCFE0EF052F9B0
:101600002B68D86A03685B68984710B11E480FF0D2
:1016100089F804F1400601230DF10F0130468DF8E1
:101620000F3006F0C9FE94F940306BB194F90C10FC
:10163000002909DB38464FF461330522C9B20BF0AB
:10164000FDF9304607F066F804F5C0700BF0A8FB12
:1016500004F522700CF08EFA2B68586A03681B6838
:1016600098472B68586A002103680091D3F8BC4062
:1016700008220923A0470FF0CBFD044B186005B0EA
:10168000F0BD00BF30260020906C0308002600202B
:101690000148FFF78BBF00BF38260020F0B52DEDC5
:1016A000028B444D2C788BB0002C7FD10FF0B0FD15
:1016B000414B1B6840F2DC51C31A8B4202461AD9D7
:1016C00001232B703D4D2B68586A0368CDE9004417
:1016D0004FF0FF32D3F8C06021462346B0472B6855
:1016E000586A0368D3F8C43000210BB0BDEC028BFC
:1016F000BDE8F0401847324E3368C31A1D2B55D948
:10170000304B04AD03F11807186859682C4603C420
:101710000833BB422546F7D132602B4D274E9FED53
:101720002B8A00243368586A2B780168234403F01D
:1017300007030AAA03EB4303134413F8182C07EE1C
:10174000902AF8EEE77A13F8162C67EE887AFCEE0A
:10175000E77ACDED027A07EE902AF8EEE77A67EEA7
:10176000887AFCEEE77ACDED037A9DF80C200192A1
:1017700013F8173C07EE903AF8EEE77A62B267EE9C
:10178000887A0134FCEEE77ACDED037A9DF80C30CF
:101790000093D1F8C0709DF808300021B847082C9C
:1017A000C0D12B7801332B70336899E70BB0BDECB7
:1017B000028BF0BD082600200026002030260020E5
:1017C0000C260020206C0308102600209A99993ED0
:1017D0002DE9F341144C154EDFF86080144F20467C
:1017E0001EF02CFD134A0146121B134801F0F0FABB
:1017F0001DF0FEFD0446A4B1206AE1690191B042EA
:1018000014BF251AA8EB06051EF018FD0199024623
:101810002B46384601F0DCFA20461DF0F9FD04465F
:10182000E9E702B0BDE8F0810001002000070020D8
:10183000BA6C030800070020B06C030800230020E6
:1018400010B50F4C05F0E8FB2368986A0368052281
:10185000DB69002198472368986A036864211B6943
:1018600098472368986A036828215B68984723682B
:10187000986A0368BDE810401B690021184700BF43
:101880003026002073B505460FF0C2FC324A1368BB
:10189000C31AB3F57A7F044613D9304B10601B7816
:1018A00023B92F4A536983F4805353612D4B1B682E
:1018B000586A002103680091D3F8BC60082209230C
:1018C000B0470CF017FB284A136841F28831E31A3D
:1018D0008B4206D9016821B114600289234801F0C6
:1018E00077FA6B7BDA070AD5214A136841F288310F
:1018F000E31A8B4203D928461460FFF769FF6B7B1C
:101900009B070DD41B4A1368E31A132B21D82846D2
:1019100001F0E2FA284602B0BDE87040FFF7BEBE13
:101920000FF076FC43F698239842EBD91248FFF764
:1019300087FF12481EF02EFCBFF34F8F1049114B4A
:10194000CA6802F4E0621343CB60BFF34F8F00BF5D
:10195000FDE71460DBE700BF142600200023002011
:1019600000040240302600201C260020CC6C030816
:10197000182600202026002038260020010007B06D
:1019800000ED00E00400FA050148FFF77BBF00BF4F
:101990003826002038B5054B1C6823680A461D68A8
:1019A000034B01462046A847002038BD30260020C2
:1019B0002426002010B50A4C2046FFF7ADFD094A49
:1019C000094920461FF0C8F80FF080F8074B084A75
:1019D0001860BDE810400749074803F015B900BF7B
:1019E0003826002034690020151501083026002013
:1019F00089190108911601082426002013B5044610
:101A000006F0D4FA05F00AF8204606F04FFA18B1AD
:101A1000B4F90030022B0BD006F072FD04F0D0FCBC
:101A200002230DF106012046ADF8063006F014FD44
:101A300002230DF106012046ADF8063006F002FD46
:101A400002B0BDE8104006F06FB9000070B52DED92
:101A5000028B324B93F90A308CB00446002B51D0E4
:101A600000F5227007900BF00FFF94F89912D4F84C
:101A7000BC23242505FB0143D3F8A4329A4241D06C
:101A80000798C4F8BC330BF0E5FF00283AD094F86F
:101A9000993205FB034308A9D3F8AC220A9200252A
:101AA00001220AA893EDAC8A0B9502F003F808AB6B
:101AB00080B20293182640F20443CDE90036039029
:101AC00012A3D3E900230495204600F0EFFADFEDDE
:101AD000147A0B9578EE277A012208A90AA8CDED91
:101AE0000A7A02F003F808AB80B2CDE9016340F254
:101AF000054303900093049506A3D3E900232046F1
:101B000000F0D4FA0CB0BDEC028B70BD9AC8BD12C7
:101B100034C4C7CD7162D977642A2749382600209A
:101B20003393884330B52DED028B83B06946104660
:101B300002F0D6F9002840D1224B1C68224B1A78BB
:101B400052B9606A01251D7003681B689847E06AF6
:101B5000036829469B6B98470FF05AFB9FED1B8A41
:101B6000DDED017A1A4B9FED1B0A186067EE887A4B
:101B7000194BDFED1A0AFCEEE77A2320C3ED007A59
:101B8000174B93F9083007EE103AB8EEC77AB7EE64
:101B9000001A27EE000A04F04DF8DDED017AE06A44
:101BA00067EE887A0368FCEEE77AF0EE400ADB6BBA
:101BB0009DED000A17EE901A984703B0BDEC028B1A
:101BC00030BD00BF30260020183A002000007A44C3
:101BD000143A00200AD7233C103A002000000000ED
:101BE0003826002010B50C4C2368A3B10FF010FB71
:101BF0002368C01A094B1B6898420CD9084BDFEDCB
:101C0000090A1B68D86A03680021DB6BB0EE600A22
:101C100098470023236010BD143A0020103A00209A
:101C20003026002000000000BFF34F8F0549064B0F
:101C3000CA6802F4E0621343CB60BFF34F8F00BF6A
:101C4000FDE700BF00ED00E00400FA0513B5102227
:101C5000002104468DF8072020F084FF054B1B6807
:101C6000D86A03680DF107021B6B2146984702B042
:101C700010BD00BF30260020F0B58BB017460446DB
:101C80000E460FF0C5FA054604F012F803464FF46D
:101C9000C87005F5167504F58054B3FBF0F202FB2D
:101CA000103315FA83F3C4F8B033FD7E35B91F48FD
:101CB0000EF038FD84F8B4530BB0F0BD384605A9DA
:101CC00002F018FB07460028F6D101A8FFF7BEFF77
:101CD0009DF8165001A92A460DF1170020F0E8FEE4
:101CE00028B113480EF01EFD84F8B473E4E70F2DFD
:101CF0000CD8D4F8B03384F8B453A3F51673C4F8F1
:101D0000B03329460B480EF00DFDD5E79DF81410B1
:101D10000029D1D030461AF095FB9DF8142094F894
:101D2000B61305480EF0FEFCC6E700BF946E03082C
:101D3000BF6E0308E06E0308026F030807B5104684
:101D400001A901F0A1FD18B9034B9DF804201A70F8
:101D500003B05DF804FB00BF283A002007B5104629
:101D600001A902F075F958B9074B9DF804101B68DA
:101D7000D86AA1F1FF02036851421B68514198479C
:101D800003B05DF804FB00BF3026002037B50B48D8
:101D90000468606A0568CDE900230B46D5F8C05099
:101DA0004FF0FF320021A847606A0368D3F8C430BF
:101DB000002103B0BDE83040184700BF30260020A6
:101DC0002DE9F0412DED028B96B0804601A9104619
:101DD00002F0E6F800285BD1DFED308A07469DF877
:101DE0000420FBB29A4253D916AA02EB830313F8DC
:101DF000524C13F8515C13F8506C98F90930E40018
:101E0000AD00F600642BE4B205F0F805F6B237D069
:101E1000002B35DB07EE903AF8EEE77AFF2227EE4B
:101E2000A88A07EE904AF8EEE77A002167EE887AF2
:101E3000FDEEE77A17EE903A18B203F031FF07EEA5
:101E4000905AF8EEE77AFF2267EE887A0021FDEEDD
:101E5000E77AC4B217EE903A18B203F021FF07EE0A
:101E6000906AF8EEE77AC5B267EE887AFF22FDEE57
:101E7000E77A002117EE903A18B203F011FFC6B2CC
:101E800033462A4621464046FFF780FF0137A6E742
:101E900016B0BDEC028BBDE8F08100BF0AD7233C31
:101EA00008B5154B1B7833B1FF2B144B22D14FF4DF
:101EB00000329A611DE00FF0ABF9114A1368C31AA2
:101EC000642B16D90F4910600B78013303F00F0211
:101ED0004FF4AA43D34013F0010F4FEA43030A70B3
:101EE00003F002030CBF4FF4003200221343034AF5
:101EF000936108BD0222DCE7283A0020000402407A
:101F0000643A0020613A002038B5084615461C4660
:101F10001AF0A0FA60B99DF81030022B07D1012CFD
:101F200005D12FA3D3E90023C5E90023012038BD43
:101F300040F226439C424AD011D80B2C0BD864B1F6
:101F4000601E0A2809D8DFE800F0260808082E08D5
:101F5000080808363200282C21D00020E7E740F29C
:101F60004C439C422FD00AD8B4F5876F27D040F25B
:101F700039439C42F1D11CA3D3E90023D4E740F6B6
:101F8000B9339C4227D044F620639C42E5D118A384
:101F9000D3E90023C8E718A3D3E90023C4E718A3B3
:101FA000D3E90023C0E718A3D3E90023BCE718A3B3
:101FB000D3E90023B8E718A3D3E90023B4E718A3B3
:101FC000D3E90023B0E718A3D3E90023ACE718A3B3
:101FD000D3E90023A8E718A3D3E90023A4E700BFAF
:101FE000401DA12026812A0BC41EDD8B3CD9312047
:101FF000A1A6A1951A7065E99E6AC421818A46EE60
:1020000026417272DF25D7B7F017304A39059E5640
:10201000D5A4D139F922B6A7CDD269EBC51A133BA5
:10202000525DB1C2FEA99EBE03806A5575F300875A
:10203000011517CB0E03561FE9A2A272EAE738B1C9
:1020400013B59DF81040CDE9003413460A46014609
:10205000806AFFF759FF02B010BD000070B500F5AF
:1020600080560D46D6F8AC437CB90C2101201DF0FA
:102070008BFFC6F8AC0308B9002070BD0560846012
:102080000430FAE72646A46824B12368AB42F9D1AC
:10209000201DF2E70C2101201DF076FFB060002822
:1020A000EAD00560B3689C60B068E9E72DE9F041CB
:1020B00090B000F59D51BDF85870044616461C318D
:1020C00040F2434201A8984602F0DCFD012F0ED1F8
:1020D00046EA07412046FFF7C1FF054670B90024D4
:1020E00001A802F0F1FD204610B0BDE8F08104F532
:1020F00077701AF0AFF90028EAD1F0E73822002112
:1021000002A820F02FFD02238DF808309DF85C30E6
:102110008DF82030189B0993BDF86430ADF8283055
:10212000CDE90468ADF8187007950FF073F80D4B02
:10213000C01841F10001CDE90C0104F5777002A946
:102140001AF08AF9084B0028D5BF9A881A6801321C
:102150001218D4BF9A801A600028D4BF002401242A
:10216000BEE700BF40420F002C3A002030B589B0D6
:1021700004460FF04DF81B4A126903461007C2F3DC
:10218000C00103D4184B197009B030BD174802685C
:102190009A1A632AF8D9144903600A78FF2A1CBFE7
:1021A00001320A7007AD0B788DF8193001222946EB
:1021B00006A88DF8182001F053FB0023049380B289
:1021C00044F621631822CDE90250CDE900322046C1
:1021D00002A3D3E90023FFF769FFD5E76E46A7FB0B
:1021E0006EA44506000402406C3A0020683A0020C4
:1021F00030B58FB014460D4638220021684620F0D5
:10220000B1FCDDE91223CDE90223BDF85030ADF871
:10221000103004F119030593A37E8DF81830159B37
:102220000793BDF85830ADF820300EF0F3FF0D4B9A
:10223000C31841F100016A46CDE90A312846E17E22
:102240001AF04EF9084B0028D5BF9A881A68013257
:102250001218D4BF9A801A600028D4BF0020012031
:102260000FB030BD40420F002C3A0020F0B591B0C5
:1022700004460E46104608A9154602F003F9B0BB05
:102280009DF82030012B16D106F03AF904F098F8A9
:1022900005F04AFD05F08AFE184904F1400005F0FA
:1022A000B9FD174904F5C07005F0B4FD154904F5F2
:1022B000227005F0AFFD1022002106AF0CA820F01F
:1022C00051FC012239460CA88DF8382002F0FEF8A6
:1022D0000A23029307A3D3E9002380B2CDE9037058
:1022E000CDE9002331462A462046FFF781FF11B091
:1022F000F0BD00BFCDD269EBC51A133B547503087E
:1023000084800308788203082DE9F041ADF5487D0B
:1023100066AC05460E46174600214FF4C4722046AF
:1023200020F020FC0EF074FF2F4B4FF47A72B0FBBC
:10233000F2F0186093E8070084E8070002F00AFB57
:10234000037C237402F006FB437C63740323A374B1
:10235000264B5A6962610DF5DD709A68DB68A261EF
:10236000E361FFF773FC4EF603132A692384204BC5
:10237000002A18681F4B29DDCDE900320DF2CB2170
:102380001D4BC06A502202F0F9FD50210DF2CB2006
:1023900021F0D4F80DF11C0884F8320141460122E5
:1023A000204601F06FFE012302930DA3D3E9002321
:1023B00080B2CDE90380CDE9002331463A46284674
:1023C000FFF716FF0DF5487DBDE8F0810093502220
:1023D0000A4BC06A0DF2CB2102F0D0FDD5E700BF59
:1023E0009E6AC421818A46EE1C3A00201002010830
:1023F00030260020276F0308206F03081A7C03088B
:102400002DE9F0411546ADF5866D06460F461DF0E7
:10241000C1FF08A9284602F06FF80446002840F0E2
:102420009F8001464FF4D072A4A820F09BFB9DF83A
:10243000B880B8F1100F7ED808F1FF330F2B2BD8DE
:1024400042460DF1B9010DF2D13020F041FB424678
:1024500051490DF1B90021F049F80246B0B94F4891
:102460000DF11F0104F0C8FC0446002C63D09DF858
:10247000B83073B39DF828305BB39DF81F20013A44
:10248000032A6DD8DFE802F01C2E384122460DF1F8
:102490001F010DF2D130E5E7BDF82000479447AAAF
:1024A0000DF11F0105F02EF80446002843D001234A
:1024B00000930DF2D132112347A904F0D9FBD4E7E0
:1024C000012B4DD10C9B8DF81C3147A9204605F0FE
:1024D000A5FF9DF81F30013B032B41D8DFE803F037
:1024E0001C444A4F012B3BD10C9BADF81C3147A932
:1024F000204605F0CBFFECE7012B31D10C9B479335
:1025000047A9204605F0ECFFE3E7022B28D10CA9F0
:10251000204605F03DFFDCE701238DF8903294F969
:102520000030DA17CDE9A6325C210DF2D13021F06E
:1025300005F88DF8D00347AC01222146A4A802F08B
:1025400003F90B23029312A3D3E9002380B2CDE950
:102550000340CDE9002339462A463046FFF748FEBE
:102560000DF5866DBDE8F08101238DF89032B4F948
:102570000030D6E701238DF890322368D1E702239B
:102580008DF890322368A693CEE700BFAFF30080AA
:10259000D5A4D139F922B6A7406F0308496F0308C3
:1025A0002DE9F04FDFF8D8A08BB0804608F5777999
:1025B000484619F0D1FF0546002858D00024007E77
:1025C0000694CDE90744ADF8244002F0E1FA2A7EF2
:1025D0008DF8240005F1100107A820F079FA2B6886
:1025E00043F0004306930EF015FE224B0390C218F1
:1025F000DAF804000E4641F1000308F5805760B395
:102600000168009409690D4606A9A847A04224DC88
:10261000DAF8040003689B6A9847D0E90A23CDE9F9
:1026200004230EF0F7FDDDE90423801A61EB0301BA
:10263000114B834274EB01030FD397F8B533072B8B
:1026400012D90E4A87F8B5439388013393804846E0
:10265000039A334619F08EFF09E0484619F080FFCF
:10266000002387F8B533A1E7013387F8B5330BB002
:10267000BDE8F08F40420F007F841E002C3A0020FE
:102680004C3A00202DE9F0414FF00053DFF8E08094
:102690001B684345FCB005460C46164604D031483D
:1026A000DC22002120F05EFA4FF0005749A9C7F85C
:1026B0000080304601F06AFE002849D19DF824319F
:1026C0003B750BB9F37E3B759DF8252126480DF52A
:1026D000937120F0FDF9204619F0BCFE4FF0005335
:1026E00007AF58758122002128A820F03BFA39460F
:1026F000012228A801F090FE2823029317A3D3E912
:10270000002380B2CDE90370CDE900232146324693
:102710002846FFF76DFD154F3326013E16F0FF06E4
:10272000284608D0FFF73CFF3B68986A0368012100
:102730005B689847F1E7FFF783F8204619F08AFEB7
:1027400040F0304040F400201DF024FDFFF76CFA0B
:102750007CB0BDE8F08100BFAFF30080264172720B
:10276000DF25D7B704000020160000203026002007
:102770009AAD44C5F0B5044689B008460E461546E4
:1027800019F068FE68B92B7E022B21D1EB8A012B50
:102790001ED12A463146204609B0BDE8F040FFF779
:1027A0006BBAEB8A40F22642934200F0888011D83F
:1027B0000B2B0BD863B1013B0A2B09D8DFE803F0E0
:1027C0002E0808083E08080808675F00282B2DD04F
:1027D00009B0F0BD40F24C42934268D00ED8B3F538
:1027E000876F5CD040F239429342F1D12A4631469C
:1027F000204609B0BDE8F040FFF7E2BA40F6B93232
:10280000934264D044F620629342E1D12A46314695
:10281000204609B0BDE8F040FFF790BA2A4631469D
:10282000204609B0BDE8F040FFF76EBD2A463146AC
:10283000204609B0BDE8F040FFF724BF07AF2B48A2
:102840000DF070FF0122394606A88DF8182001F01E
:10285000F3FC0523029323A3D3E9002380B2CDE93F
:102860000023CDE903702A4631462046FFF7C0FC1D
:102870000EF0CEFC04F58054C4F8B803A8E72A464D
:102880003146204609B0BDE8F040FFF7B9BD2A4601
:102890003146204609B0BDE8F040FFF7E7BC2A46C4
:1028A0003146204609B0BDE8F040FFF73BB92A4663
:1028B0003146204609B0BDE8F040FFF74FBA2A463E
:1028C0003146204609B0BDE8F04000F019BC2A4668
:1028D0003146204609B0BDE8F04000F03BBE00BFE5
:1028E000AFF30080F017304A39059E56546F030845
:1028F0000A460146806AFFF73DBF000049421B4B74
:10290000112912D8DFE801F00911110D111111116F
:1029100011111519151D2125292D9A6801329A606A
:1029200070479A8901329A817047DA890132DA81D7
:1029300070475A8B01325A8370471A8B01321A83BF
:1029400070471A8A01321A8270475A8A01325A82B3
:1029500070479A8B01329A8370479A8A01329A8221
:102960007047DA8A0132DA82704700BF2C3A0020C1
:102970002DE9F04F374E97B00023CDE90B330A9382
:10298000ADF8343073680446002B5FD0324D012718
:102990004FF0000A4FF0000B70688DF814704FF084
:1029A00000088DF815800368CDE900AB0DF1150224
:1029B000D3F8089005A94346C8479DF81430002B6A
:1029C00044D0414620220EA820F0CCF8706803685D
:1029D00006AAD3F814800AA90DF11603C0470028EF
:1029E00034DD9DF8340002F0EFF80BA902468DF8B3
:1029F000500012A820F06CF804F577780A9B0E932B
:102A00000EA9DDE9062340461AF004F810F10D0F77
:102A1000014603D02046FFF771FFBDE70E9819F07D
:102A2000E9FF03900E9819F0DFFF039BCDE9000743
:102A300008AA41462046FFF767FA18B12B8A0133EE
:102A40002B82A9E76B8B01336B83A5E717B0BDE839
:102A5000F08F00BF4C3A00202C3A002007B500F55B
:102A60007771684619F068FFBDF804006423584385
:102A7000BDF80030B0FBF3F080B203B05DF804FBAA
:102A8000F0B597B004460EF0C3FB4FF47A73B0FB79
:102A9000F3F0434B434D1B682860D86A03685B6DB5
:102AA00098474FF6FF73984228BF184628810EA911
:102AB0000122284601F098FB0EAB80B20293182247
:102AC00040F255130025CDE9003203902EA3D3E93F
:102AD000002304952046FFF7E9FA637B59074ED59A
:102AE00001220EA93048314F00F03EFF0EAB80B2FC
:102AF00002931F264FF4AB73CDE90036039024A355
:102B0000D3E9002304952046FFF7D0FA78680368DC
:102B10009B6A9847002832D03A788DF838200268AE
:102B20000F924268ADF840208268ADF84220C2683A
:102B3000ADF844200269ADF846204269ADF848205E
:102B400082691392C269ADF85020026AADF8522032
:102B500007AF436AADF85430012239460EA800F0A1
:102B6000ADFE40F2571380B2CDE902700093049598
:102B700009A3D3E9002301962046FFF797FA17B07F
:102B8000F0BD00BFAFF30080F1C6A7C1D068080F49
:102B9000D1F886A9B8E33A76753CA33CAE0C08CED2
:102BA000302600201C3A00202C3A00204C3A00200D
:102BB000F0B506468DB000F5777019F04BFC2E4D40
:102BC00020B100232B7001200DB0F0BD0EF020FBD2
:102BD0002B7804463BB13046FFF740FF0121024607
:102BE00026480DF09FFD03F063F84FF4C87306F517
:102BF0008057B0FBF3F202FB130304F5167010FAD2
:102C000083F000238DF8183097F8B433C7F8B00379
:102C100023B901228DF8182087F8B63308A8FFF7EA
:102C200015F897F8B413C1F11004E4B2062C28BFCC
:102C3000062408AB224619440DF119001FF048FF85
:102C4000013406AB0025029318220123E4B2CDE93A
:102C50000032049506A3D3E9002303943046FFF71E
:102C600025FA87F8B4532846AEE700BFAFF30080DB
:102C7000401DA12026812A0B00230020646F030839
:102C800070B5244D244E4FF4807386B0AB8004465B
:102C90000EF0BEFA4FF47A73B0FBF3F0286062884E
:102CA000B4F902307F2A98BF33700DF11701002369
:102CB00004F10B008DF8173005F0B0FB41F238102D
:102CC00001F04CFE054608B10DF0A6F8134B1D604F
:102CD000134B00225D601A702DB12B6861685B6830
:102CE0000122284698470F4B009304F5777004F2B1
:102CF0000C410D4B01944FF47A62039019F076FB6E
:102D00003178039821B106B0BDE8704019F09ABB44
:102D100006B070BD1C3A00206D3A0020543A0020E5
:102D20004C3A002041200108F128010830B506285E
:102D3000134698BF1D4AC7B098BF155C07930C4651
:102D40004FF07C024FF0000127A888BF00251FF03C
:102D500009FF079B22465A210DF1BE000DF098FC99
:102D60005A2828BF5A2008AC8DF8BD002146012200
:102D700027A88DF89C5001F069FA0023049380B2D3
:102D800043F6FF731822CDE90240CDE9003208482E
:102D900004A3D3E90023FFF789F947B030BD00BF92
:102DA000AFF30080759D040C8EA454D620700308E8
:102DB000382600200EB403B503AA52F8041B019272
:102DC000FFF7B4FF02B05DF804EB03B070470000FA
:102DD0000FB407B504AA072052F8041B0192FFF7AD
:102DE000A5FF03B05DF804EB04B0704737B50446A7
:102DF00000F5777019F0BEFB2046FFF72FFE46283E
:102E000002D92B480DF08EFC2046FFF739FE94F9CD
:102E10000B50002D38D0002304F10B00EDB201A9B6
:102E20008DF8043005F0FAFA2A2D224C0AD1224DF1
:102E30002846FFF7CDFF2368986A036864215B6822
:102E40009847F5E72B2D04D11C48FFF7C1FF1C4B19
:102E500098474FF4FA6101A801F0FAFE2468A06ACD
:102E600003684FF47A715B689847E06A03689B6A6D
:102E7000984718B1012816D0124800E01248FFF711
:102E8000A7FF01A801F0F0FE104B00225A710EF0CE
:102E9000BFF947F23053984207D90D4803B0BDE857
:102EA00030401DF077B90B48E9E703B030BD00BFF3
:102EB0009C6F030830260020BA6F0308CB6F03080D
:102EC00038ED00E006700308DB6F03081C3A0020B1
:102ED000263A09B0F06F03082DE9F34104460EF0DD
:102EE00097F944490B68C31A322B05461BD9424B4C
:102EF0001B78C3B1414802780123934023F4AA43CD
:102F000023F055031B041B0C002B0EBF01260026CB
:102F10004FF4805343EA06730132394E02F01F0228
:102F2000B36102700D6004F580560EF071F9D6F8A9
:102F3000B033984202D92046FFF73AFE314A13686F
:102F4000EB1AB3F57A7F07D315600EF063F90246EA
:102F50000B462046FFF74AFF204600F063F8204664
:102F600000F0E2F8204600F09FFB2046FEF76EFDE1
:102F70002046FEF737FE2046FEF792FF2046FFF779
:102F8000F5F80EF03FF904F59D55DFF87C80074613
:102F90001C350EF037F9C01BB0F57A7F17D2D8F880
:102FA0000030986A03684FF480619B68984740F24C
:102FB000D772294601A801F065FE2046FFF7F0FA16
:102FC0002046FFF7D5FC01A801F07EFEE1E7D6F828
:102FD000B83363B10EF01CF9D6F8B833C01AB0F5A7
:102FE0007A7F04D92046FEF72BFCFEF71DFE02B0C7
:102FF000BDE8F0815C3A002000230020603A002008
:1030000000040240583A00203026002010B590F805
:103010000511044609F0C6FD6423C0B203FB004459
:10302000A06E10BD70B52DED048B90F985319EB06A
:103030000446002B58D090F88332002B54D00EF069
:10304000E7F8D4F8AC33C01A27284DD904F5C07579
:10305000284609F0CFFD2846D4F8AC63FFF7D6FF29
:10306000864241D094F88512284609F0BDFD00281B
:103070003AD02846FFF7CAFF94F88512C4F8AC038B
:10308000284609F08FFD6423C0B203FB00409FED8A
:103090001B0A00F5EE7002F03BFE0AAD282200216B
:1030A00014A8B0EE409AF0EE608AB0EE418A1FF0AC
:1030B00059FD0122294611A88DED119ACDED128AF4
:1030C0008DED138A00F0ACFC002380B2182204932B
:1030D00040F2E933CDE90250CDE90032204605A3A4
:1030E000D3E90023FEF7E2FF1EB0BDEC048B70BDF8
:1030F000AFF30080F2C20B46A9D4A7E26F12833A65
:1031000010B5A2B001A90446104600F0A3FE014686
:1031100038B99DF805300DF1060204F1400005F0C4
:103120005BFF22B010BD00002DE9F04390F9403064
:10313000ADF52D7D0446002B00F0EF8100F1400538
:10314000284605F067FE94F85061D4F8B02304EBEC
:103150000613D3F88C309A4200F0DF81C4F8B03304
:103160004FF4D072002144A81FF0FCFC94F8783191
:1031700033B9B02303FB064393F89930012B0CD8E5
:1031800094F8C0734FB90EF045F800220023CDE942
:103190004401CDE94623002313E0012384F8C03322
:1031A0003146284605F016FBCDE9440194F850114C
:1031B000284605F06BFB50EA0103CDE94601EAD051
:1031C0000223B02202FB06428DF82031D2F8B01063
:1031D0000A2381FB0310CDE94A10D2F8AC10D2F8D3
:1031E000A82081FB0310CDE94C10534394F85011F3
:1031F00008AA2846CDE94E3305F0B8FE78B14E9BBB
:10320000DDED086A9FED4F7A079307EE903AF8EEEE
:10321000E77AE6EEC77AFDEEE77ACDED4E7AB02397
:1032200003FB065203FB06468C32D6F8CC105091B5
:103230005168519194F850119268529203FB0143E6
:1032400093F8CA208DF84C2193F8992094F878319E
:103250003BB9062A0AD8DFE802F004045D6163691D
:103260006E0000238DF84D31ADF84E31062309AACA
:1032700028468DF8503105F099FA38B1DDED097A1C
:1032800067EEA77ACDED567ACDED557A94F85011C8
:103290000AAA284605F094FA28B1DDED0A7A67EE0D
:1032A000A77ACDED577A0BAF94F850113A462846DD
:1032B00005F072FA48B1D7ED007A67EEA77ACDED46
:1032C0005A7ACDED597ACDED587A9DF850119FED8F
:1032D0001E7A1E48DFED1E6A9FED1E6A55AB002266
:1032E000D6B2B14238D9D3ED007AF0EEE75AF4EE17
:1032F000475AF1EE10FA09DCF4EEE67AF1EE10FA34
:1033000004D9F4EEC67AF1EE10FA00DB186001324F
:103310000433E5E702228DF84D21A5E70322FAE701
:1033200003238DF84D3140F201139DE703238DF8FF
:103330004D31022398E703238DF84D314FF481730B
:1033400092E700BF00007A44FFFF7F7F0000C07F4C
:1033500000EF7FC700EF7F470CAE3146012244A843
:1033600000F05CFC4FF0000880B240F227434FF0C1
:103370001809CDE90260CDE90039CDF8108073A3BA
:10338000D3E900232046FEF791FE2022414644A8BF
:103390001FF0E8FB94F85031DFED696AB02202FBC0
:1033A00003433146B3F8C620B3F8C83007EE102AFD
:1033B00007EE903AB8EEC77AF8EEE77A27EE267A6B
:1033C00067EEA67A012244A88DED467ACDED477AC4
:1033D00000F0AEFB40F2254380B2CDE902600093DD
:1033E000CDF8108050A3D3E90023CDF804902046F7
:1033F000FEF75CFE94F85011CDF818812846CDE90F
:10340000448805F089FD94F962308DF814013BB1D0
:10341000284605F091FD18B9469B43F001034693F9
:103420009DF8143143B10AA9284605F01BFD18B9CF
:10343000469B43F00203469394F850113A462846BF
:1034400005F08AFD08B13B6844930122314644A847
:1034500000F0EAF90023049380B244F623634FF0AE
:103460001809CDE90260CDE90039204630A3D3E93F
:103470000023FEF71BFE94F87931002B4DD194F810
:103480005011B02303FB014393F8EC30002B44D0E0
:10349000D4F8B883B8F1000F3FD100970AAB09AA5E
:1034A000284605F02FFEC0B33B68D4F8B4239A42F7
:1034B00033D0DDED0A7A9FED237ADFED236AC4F87D
:1034C000B433F4EEC77A9DED097AADF8128101228A
:1034D000F1EE10FA27EE267A67EEA67AACBF134615
:1034E0000023314644A88DF810218DF811318DED5F
:1034F000457ACDED467A00F069F944F6226380B250
:10350000CDE902600093CDF810800BA3D3E900232E
:10351000CDF804902046FEF7C9FD0DF52D7DBDE8E0
:10352000F08300BFAFF30080D2BFDBC3C4BDE89B14
:10353000697F00BBABB43CBA1234EDEC39AE5C3100
:103540000AD7233C0000003435FA8E3C5F43370F26
:1035500000E741CAF0B5A5B004460E46104603A9DF
:10356000154601F091F9002840F0908030469DF812
:103570000D7018F06FFF874240F08880D4F8C43394
:10358000002B75D09DF90E305A1C01D194F90C30E6
:10359000002B7BDB424A092B106877DC03F1100219
:1035A00050F82260002E71D094F9D01399420BD0BC
:1035B000D4F8CC2342B1C9B209294FF000026DD82A
:1035C000103150F821100A6184F8D033D4F8CC338C
:1035D000B34208D0D4F8C40301F09EFD0023C4F820
:1035E000CC63C4F8D433D4F8CC0300284ED09DF873
:1035F0000F3094F8D86303F0010284F8D82302B1A5
:10360000284A114601F0F4FBEB7E84F8D1339DF893
:103610000C30049984F8D233D4F8D433994200D1D1
:103620007EB994F8D8334BB141B11E4B00934FF49F
:103630000063D4F8CC031A4601F0EAFB049BC4F8FB
:10364000D433D4F8CC33D4F8C4231A610DF0E0FDA0
:103650009DF81420C4F8C803C2B194F8D833D4F844
:10366000CC03ABB10F4B0DF1150101F0DFFB0DE009
:10367000142001F073F9064618B14FF4806101F08F
:10368000FBFCC4F8C463002E7FF47CAF25B0F0BD12
:1036900003680DF11501DB689847F7E71261FFDE5B
:1036A00030260020E460E4F22DE9F043D0F8CC337A
:1036B000C9B00446D3B190F8D133BBB1D0F8C4330C
:1036C000A3B1D0F8C8530DF0A3FD40F6B733401BAB
:1036D000984294F8D8330CD92BB10022D4F8CC03FB
:1036E000114601F085FB0023C4F8CC3349B0BDE896
:1036F000F08373B1344E0825D4F8CC0333467822D6
:1037000027A901F0A3FB002803DD013D15F0FF050B
:10371000F2D12BA7D7E900674FF00908D4F8C4030A
:1037200001F00CFD0028E1D008F1FF3818F0FF0887
:10373000DCD0D4F8C40306A901F0B0FD069D814693
:10374000002DD3D08422002127A81FF00BFA94F873
:10375000D1338DF89D3094F8D2338DF89C30782D8C
:10376000D4F8D43328932A4694F8D0338DF89E3079
:1037700028BF7822494607AD0DF1A50006928DF8C5
:10378000A4201FF0A5F90122294627A801F030F84E
:10379000002380B21022049340F6B933CDE9003201
:1037A000CDE9025032463B462046FEF77FFC00281A
:1037B0009CD00699D4F8C40301F0F4FCAEE700BF36
:1037C000E9A2A272EAE738B1E460E4F237B50C4648
:1037D000002105462160217103460122204619F08F
:1037E00063F801226B1C1146204619F05DF895ED37
:1037F000010A19F0A9F80DF10603ADF80600102230
:103800000221204619F050F895ED020A19F09CF8B3
:103810000DF10603ADF8060010222046122119F022
:1038200043F8052003B030BD13B504460846002117
:1038300001602346C0F803102022019019F034F8EB
:103840000198231D0122202119F02EF8019804F17E
:1038500008031722212119F027F8072002B010BD14
:1038600013B5044608460021018023460822019032
:1038700019F01AF808220198631C114619F014F87F
:10388000022002B010BD000013B50446007F10B145
:10389000A38A012B0CD80023009108221946204648
:1038A00018F0C4FE237FA08A23B9B0FA80F0400943
:1038B00002B010BD013818BF0120F9E770B50C4601
:1038C000192605463246002120461FF04BF92B46AB
:1038D00020460822002118F0E7FF2B1D2046202259
:1038E000082118F0E1FF05F10803204610222821E5
:1038F00018F0DAFF05F10A0320461022382118F0EB
:10390000D3FF05F10C0320461022482118F0CCFF0C
:1039100005F10E0320461022582118F0C5FF05F1CD
:10392000100320461022682118F0BEFF05F1140391
:1039300020462022782118F0B7FF05F11803204611
:103940001022982118F0B0FF05F11A03204610222A
:10395000A82118F0A9FF204605F11C031022B82168
:1039600018F0A2FF304670BD70B50C461C26054607
:103970003246002120461FF0F5F82B462046202233
:10398000002118F091FF2B1D20461022202118F055
:103990008BFF05F1080320462022302118F084FF18
:1039A00005F10C0320461022502118F07DFF05F18F
:1039B0000E0320461022602118F076FF05F1100357
:1039C00020461022702118F06FFF05F112032046E7
:1039D0001022802118F068FF05F114032046102200
:1039E000902118F061FF05F1160320461022A02156
:1039F00018F05AFF05F1180320461022B02118F0E4
:103A000053FF05F11A0320461022C02118F04CFF85
:103A10002046AB191022D02118F046FF304670BD69
:103A20002DE9F3410E46044617460021192230467F
:103A30001FF098F8A0460025B8EC010A18F084FFA2
:103A40002946ADF806000DF1060310223046103568
:103A500018F02AFF302DEFD1237B092B28BF092333
:103A60008DF805303FB929460DF105030422304693
:103A700018F01AFF342510344FF000089DF8053077
:103A8000984505EB081704D3F81DC00802B0BDE83F
:103A9000F081B4EC010A18F057FF0DF10603ADF800
:103AA000060010223946304618F0FEFE08F10108E3
:103AB000E4E7000037B50C4600212160A1800346F1
:103AC00005462022204618F0EFFE95ED010A18F079
:103AD0003BFF0DF10603ADF8060010222046202121
:103AE00018F0E2FE062003B030BD000073B50026DA
:103AF0000E6090ED000A0C46054618F025FF0DF10A
:103B000006033146ADF806001022204618F0CCFE20
:103B100095ED010A18F018FF1022ADF806000DF11E
:103B200006032046114618F0BFFE042002B070BD07
:103B300073B50C46102605463246002120461FF07C
:103B400011F895ED000A18F0FFFE0DF1060332465C
:103B5000ADF806000021204618F0A6FE95ED010AFA
:103B600018F0F2FE0DF1060332463146ADF80600BC
:103B7000204618F099FE95ED020A18F0E5FE0DF1C9
:103B800006033246ADF806002021204618F08CFED0
:103B900095ED030A18F0D8FE0DF106033246ADF894
:103BA00006003021204618F07FFE95ED040A18F03B
:103BB000CBFE0DF106033246ADF80600402120464B
:103BC00018F072FE95ED050A18F0BEFE0DF1060321
:103BD0003246ADF806005021204618F065FE95EDFE
:103BE000060A18F0B1FE0DF10603ADF806003246E4
:103BF0002046602118F058FE05F11C0320460722DC
:103C0000702118F051FE204605F11D030622772190
:103C100018F04AFE304602B070BD00002DE9F347AF
:103C20000D460446002190462846DE221EF09AFFEB
:103C3000234638220021284618F036FE3822114645
:103C400004F10803284618F02FFE04F110030322A4
:103C50007021284618F028FE04F111030822802163
:103C6000284618F021FE04F1180325228821284651
:103C700018F01AFE04F120032522AD21284618F081
:103C800013FE04F128031B22D221284618F00CFE53
:103C900004F12C031B22ED21284618F005FE04F147
:103CA000300320224FF48471284618F0FDFD04F102
:103CB000340320224FF49471284618F0F5FD04F1E6
:103CC000380320224FF4A471284618F0EDFD04F1CA
:103CD0003C0306224FF4B471284618F0E5FD04F1C8
:103CE0003D0302224FF4B771284618F0DDFD04F1C0
:103CF0003E0304224FF4B871284618F0D5FD04F1B4
:103D00003F0306224FF4BA71284618F0CDFD94F80F
:103D10004030242B28BF24238DF8033006220DF1D8
:103D200003034FF4BD71284618F0BEFD04F1440AA8
:103D30004FF4C0774FF000099DF80330994507F123
:103D400010062BD394ED350A18F0FEFD0DF1060395
:103D5000ADF8060010223946284618F0A5FD94F863
:103D6000D830012B28BF01238DF80430B8F1000FA3
:103D700007D1314601AB0122284618F095FD07F125
:103D8000110604F586744FF000099DF8043099453A
:103D900015D3F01DC00802B0BDE8F087BAEC010AE7
:103DA00018F0D2FD3946ADF806000DF106031022D9
:103DB000284618F079FD09F101093746BCE7A4F15E
:103DC0002C0A06F16007B046534641462022284699
:103DD00008F1200818F068FD47450AF1040AF3D1FC
:103DE000A4F11C0806F1CC0A434639462422284691
:103DF000243718F059FDBA4508F10808F4D114F831
:103E0000043C242B28BF24238DF8053006F1D20171
:103E10000DF105030622284618F046FDD836A046C7
:103E200000279DF805309F4203D309F10109C034F2
:103E3000ABE7B8EC010A18F087FD3146ADF8060093
:103E40000DF106031022284618F02EFD103601371A
:103E5000E7E70000F7B5047F05460E462CB1838ADC
:103E6000822B02D9012003B0F0BD00230096082266
:103E70001946284618F0DAFBDCB9731C08220093B7
:103E800011462346284618F0D1FB10247378802B66
:103E9000E8D8012372785F1C013B934210D32B7F3B
:103EA000A88A0734E408B3B9844294BF00200120F3
:103EB000D9E7AB8ADB00083BDB0873700824E5E731
:103EC000F3190093214600230822284618F0AEFB80
:103ED00008343B46DEE7201A18BF0120C3E7000084
:103EE0007FB50446007F0D4610B1A38A042B22D86B
:103EF0000DF10E060123102200210096204618F035
:103F000095FBBDF80E0018F04DFD1022012385ED44
:103F1000000A11460096204618F088FBBDF80E00F6
:103F200018F040FD85ED010A237FA08A2BB90328F4
:103F30008CBF0020012004B070BD043818BF0120E0
:103F4000F9E70000F7B50C46009215460968002312
:103F50000822064618F06AFB21686F1C08312160B0
:103F6000009700230522304618F060FB2168AF1C43
:103F700005312160009700230622304618F056FBD9
:103F80002168033506312160009500230522304663
:103F900018F04CFB236800200533236003B0F0BD0C
:103FA0002DE9F043067F85B005460C4636B1838A7D
:103FB0003D2B03D9012005B0BDE8F0830023039316
:103FC000002E3BD13346009405223146284618F096
:103FD0002DFB039B053303932378142BEAD8671C2E
:103FE00023789E421BD23A4603A92846FFF7AAFF30
:103FF00004370028DED10136F2E7013FDAD022781B
:1040000019FB0282224403A92846FFF79BFF0028E0
:10401000D0D1237801332370039B9E42EDD8039BBC
:104020002A7FA88A0733DB0822B9834294BF002085
:104030000120C0E7181A18BF0120BCE72370AE8A20
:10404000F600073E15274FF004094FF00108E3E79B
:1040500013B50446007F10B1A38A012B0CD80023AE
:10406000009108221946204618F0E0FA237FA08A22
:1040700023B9B0FA80F0400902B010BD013818BF72
:104080000120F9E72DE9F3470D460446002190464B
:10409000284640F279121EF065FD234620220021B9
:1040A000284618F001FC231D02222021284618F082
:1040B000FBFB631D03222221284618F0F5FBA31DFC
:1040C00003222521284618F0EFFB04F108031022F3
:1040D0002821284618F0E8FB04F1100308223821B3
:1040E000284618F0E1FB04F111030822402128467C
:1040F00018F0DAFB04F1120308224821284618F0D0
:10410000D3FB04F1140320225021284618F0CCFBE5
:1041100004F1180340227021284618F0C5FB04F171
:1041200020030822B021284618F0BEFB04F1210329
:104130000822B821284618F0B7FB04F12207C02650
:104140003B46314608222846083618F0ADFBB6F546
:10415000A07F07F10107F3D194F832308DF80730D2
:1041600031460DF107030822284618F09DFB002672
:1041700004F1330A9DF807304FEAC6099E4209F55B
:10418000A47720D394F83231502B28BF50238DF8D8
:104190000730B8F1000F08D139460DF107030722A7
:1041A000284618F081FB09F24F17002604F2331459
:1041B0009DF807309E4207EBC6010DD30731C808B2
:1041C00002B0BDE8F0870AEB06030822394628460C
:1041D00018F06AFB0136CDE7A3190822284618F02B
:1041E00063FB0136E4E7000013B5044608460021EE
:1041F00001602346C0F803102022019018F054FB00
:104200000198231D0222202118F04EFB0198631D06
:104210000322222118F048FB0198A31D0322252127
:1042200018F042FB019804F108031022282118F02D
:104230003BFB072002B010BD08B50346084600212D
:104240000170012218F030FB012008BD2DE9F34177
:104250000D4604460021164628467B221EF082FCAD
:10426000234603220021284618F01EFB63781F2BEB
:1042700028BF1F238DF8063005220DF10603032108
:10428000284618F011FB01239DF80620DF0003F1FA
:104290000108013B9A421CD894F821305A2B28BFC0
:1042A0005A238DF807303EB939460DF1070307222E
:1042B000284618F0F9FA0737002622349DF807300F
:1042C0009E4207EBC6010DD30731C80802B0BDE816
:1042D000F08104EB080308223946284618F0E4FA76
:1042E0004346D1E7A3190822284618F0DDFA013623
:1042F000E4E70000F7B5047F05460E462CB1838A3B
:10430000122B02D9012003B0F0BD00231946072269
:104310000096284618F08AF9731C009301220023A6
:104320000721284618F082F9D4B9B31C009305225E
:1043300023460821284618F079F90D24B378102B6C
:10434000E0D83746B278BB1B934210D32B7FA88AA4
:104350000734E408B3B9844294BF00200120D2E7B7
:10436000AB8ADB00083BDB08B3700824E6E7FB1CE4
:104370000093214600230822284618F057F90834F4
:104380000137DFE7201A18BF0120BCE7F7B5047F2B
:1043900005460E462CB1838ACA2B02D9012003B0F0
:1043A000F0BD0023194600960822284618F03EF971
:1043B000731CD4B90822009311462346284618F0EE
:1043C00035F910247378C82BE8D8012372785F1C64
:1043D000013B934210D32B7FA88A0734E408B3B97A
:1043E000844294BF00200120D9E7AB8ADB00083B60
:1043F000DB0873700824E5E7F319009321460023D6
:104400000822284618F012F908343B46DEE7201A45
:1044100018BF0120C3E70000F7B50D460446002190
:104420001646284681221EF09DFB234608220021C5
:10443000284618F039FA94F901206378002AB8BFA9
:104440007F238DF807309EB90DF10703072208215D
:10445000284618F029FA0F27002602349DF8073065
:104460009E4207EBC60105D30731C80803B0F0BD73
:104470000827F1E7A3190822284618F015FA013693
:10448000ECE7000037B50446007F0D4610B1A38A63
:10449000072B15D800231946009508222046083519
:1044A00018F0C4F80123009530220821204618F0A6
:1044B000BDF8237FA08A2BB906288CBF00200120DD
:1044C00003B030BD073818BF0120F9E738B50C46F6
:1044D000002121600546C4F803100346302220461F
:1044E00018F0E2F9204605F108030122302118F006
:1044F000DBF9072038BD00002DE9F04390F81C805F
:1045000085B006460D46B8F1000F06D0838AE02B31
:1045100003D9012005B0BDE8F083002319460D2220
:104520000095304618F082F80DF10F030093032236
:1045300000230D21304618F079F89DF80F30042B38
:10454000E7D82B72013B032B03D8DFE803F02530BB
:104550003B461024B8F1000F5FD105F1980300939A
:10456000214643460722304618F060F8073495F894
:1045700098305C2BCDD82F4695F898207B1B934222
:1045800052D3337FB08A0734E408002B58D18442D9
:1045900094BF00200120BDE705F1100300934022E5
:1045A00001231021304618F041F85024D2E705F1DC
:1045B00010030093202201231021304618F036F812
:1045C0003024C7E705F110030093082200231021CF
:1045D000304618F02BF81824BCE705F110030093BF
:1045E000082200231021304618F020F82B7C802B65
:1045F0008FD8002705F111092B7CFC009F4204F1A4
:104600001804A7D209EB07030093082200232146D0
:10461000304618F00BF80137EEE7B38AC4EBC3035A
:10462000DB0885F89830A2E707F19903009321464B
:1046300000230822304617F0F9FF083401379BE7C2
:10464000201A18BF012065E7F7B50C4613780968F2
:104650008DF8063015460DF106030322064618F0C4
:1046600023F92168033121602B78013B032B0CD8FF
:10467000DFE803F0020D161F05F108034022304663
:1046800018F012F923684033236003B0F0BD05F140
:1046900008032022304618F007F923682033F3E797
:1046A00005F108030822304618F0FEF823680833A5
:1046B000EAE72B7A802B28BF80238DF80730082269
:1046C0000DF10703304618F0EFF823680833236034
:1046D000002709359DF807309F42D6D2EB19216893
:1046E0000822304618F0E0F82368083323600137C9
:1046F000F0E7000073B50C46137809688DF80730B1
:1047000015460DF107030222064618F0CDF8216880
:10471000023121602B78012B03D0022B0BD002B089
:1047200070BD05F108034022304618F0BDF823683B
:1047300040332360F3E705F108032022304618F0E8
:10474000B3F823682033F4E773B50D46044600211F
:104750001646284640F273121EF004FA052322463C
:1047600001A928460193FFF76FFF019B04F1900216
:10477000053301A928460193FFF766FF019B04F565
:104780009072063301A928460193FFF7B3FF019BFE
:1047900004F59872063301A928460193FFF7AAFF92
:1047A00094F840315C2B28BF5C238DF803304EB960
:1047B0000DF1030301990722284618F075F8019BB3
:1047C00007330193002604F241149DF80330019948
:1047D0009E4203D30731C80802B070BDA319082256
:1047E000284618F061F8019B083301930136ECE785
:1047F000F7B50D4604460021164628467F221EF0D6
:10480000B1F9234608220021284618F04DF8631C10
:1048100007220821284618F047F8A31C05220F217B
:10482000284618F041F8E31C04221421284618F009
:104830003BF81822231D1146284618F035F8237A34
:10484000782B28BF78238DF807309EB90DF1070328
:1048500007223021284618F027F837270026093488
:104860009DF807309E4207EBC60105D30731C80803
:1048700003B0F0BD3027F1E7A3190822284618F04D
:1048800013F80136ECE70000F7B5047F05460E4645
:104890002CB1838A7F2B02D9012003B0F0BD002305
:1048A000194608220096284617F0C0FE731C009394
:1048B000072200230821284617F0B8FEB31C0093F6
:1048C000052201230F21284617F0B0FEF31C0093A8
:1048D000042200231421284617F0A8FE331D1822B5
:1048E000009311460023284617F0A0FEDCB906F11C
:1048F00008030093072223463021284617F096FE2E
:104900003724337A782BC7D83746327ABB1B934289
:1049100010D32B7FA88A0734E408BBB9844294BF24
:1049200000200120B9E7AB8ADB00303BDB083372A3
:104930003024E6E707F1090300932146002308220B
:10494000284617F073FE08340137DEE7201A18BF37
:104950000120A2E7004870477070030801218842D7
:1049600038BF08461BF010BBFFF7F8BF08B11BF0BB
:104970000FBB7047FFF7FABF10B4026854681A46BD
:1049800023465DF8044B184700207047012070470C
:1049900000207047002070470020704770470000DB
:1049A00000207047002070477047000070470000EB
:1049B00037B505460C468322011D01A800F062F9B7
:1049C000611EC9B202299EBF05EBC1010023C1E9E6
:1049D000073301A800F078F903B030BD2DE9F743A3
:1049E0001E461B885B070546884620D4011D4222CF
:1049F00001A800F047F92C4605F118094C4513D0E1
:104A0000E3696BB12B6828465B6C98473388276A4B
:104A1000C1B243F00403E0694246B8470834EDE709
:104A2000236A002BEED1F9E701A800F04DF901202F
:104A300003B0BDE8F08300007FB56D4685E8060051
:104A40000446011D712203A81E4600F01BF92146F1
:104A50000022C869D3B288B9086A78B995E803001A
:104A600004EBC2021C32013382E8030001243370DC
:104A700003A800F029F9204604B070BD0132032AD2
:104A800001F10801E5D10024F2E700002DE9F04F23
:104A90002DED028B8BB004468B465322011D01A8DD
:104AA000BDF858809FED258B00F0ECF8254604F109
:104AB0001809002708F0040AA94536D0EB690BB99C
:104AC0002B6A63B1BAF1000F0BD1236820465B6CEF
:104AD00098474346C1B25A46D5E90706B04708355C
:104AE000EAE7002FFBD18DED028BADF810705B462D
:104AF00005AA0BF1080C18685968174603C7083354
:104B000063453A46F7D1186838609B88BB800CF043
:104B100081FB0423ADF810302368CDE902019B6CC2
:104B200002A9204698470127D9E701A800F0CCF850
:104B300001200BB0BDEC028BBDE8F08F000000003F
:104B40000000000030B503680968DD0FB5EBD17FC8
:104B500023F0604421F060424FEAD1700BD0002B6B
:104B6000B8BFA40C0029B8BF920C944202D034BF45
:104B70000120002030BD944205D1C1F38070C3F301
:104B800080738342F6D194422CBF00200120F1E7CC
:104B9000082817D90C280CD910280CD914280CD99E
:104BA00018280CD920280CD930288CBF0F200E20B3
:104BB0007047092070470A2070470B2070470C206F
:104BC00070470D2070470000082817D909280CD01D
:104BD0000A280CD00B280CD00C280CD00D280CD097
:104BE0000E2814BF4020302070470C207047102042
:104BF000704714207047182070472020704700002D
:104C0000436818478368184710B5024C8260C0E9B2
:104C1000004110BD08710308007B00F001007047DF
:104C2000704700008160828070470000826838B55C
:104C300004465AB1037B13F0010507D143F0010389
:104C400003739047237B65F30003237338BD000093
:104C500010B5044B1B680446986A03681B699847A3
:104C6000204610BD3026002010B5054B1B680446B9
:104C7000986A036800211B699847204610BD00BF51
:104C800030260020F8B50C4B01601E680446B06A5F
:104C900003681B6C17469847054610B1F36AA3F8E2
:104CA0004270206803689B6898471DB1F36A002230
:104CB000A3F842202046F8BD3026002010B5044657
:104CC000FFF7E0FF204610BD10B5044600680368FA
:104CD000DB689847204610BDC181B1FA81F04009D8
:104CE00070470000C089704770470000002070477F
:104CF0007047000070470000002070470020704798
:104D0000704700004FF4B450704700000020704717
:104D10000020704700207047002070470020704737
:104D2000007B70477047000007B503688DF80710D7
:104D3000DB6801220DF10701984703B05DF804FB21
:104D400008B5036801225B6A98470028D4BF002099
:104D5000012008BD07B503680DF10701DB6998471D
:104D600020B19DF8070003B05DF804FB4FF0FF3061
:104D7000F9E7000013B5044608460191FCF73CFB37
:104D800023680199DB680246204602B0BDE8104066
:104D9000184700000CF03EBA10B444682CB9036800
:104DA0005DF8044BD3F88030184700205DF8044BC1
:104DB0007047000082681AB90368D3F8903018472A
:104DC0000020704782681AB90368D3F894301847F6
:104DD0000020704730B4456825B90468E46FA446E4
:104DE00030BC604730BC704700231A46FFF7F2BF63
:104DF000436813B18B4200D041B9836813B1934229
:104E000000D01AB9C0E90112012070470020704794
:104E100030B44468029D0CB1AC4204D10468E46F24
:104E2000A44630BC604730BC7047000010B44468F2
:104E30000CB19C4205D103685DF8044BD3F8803077
:104E4000184700205DF8044B7047000037B5054651
:104E5000806808B1984212D12B680191D3F8843050
:104E600092B2284698470446286928B1002C03DDF1
:104E70000199224600F0F2F9204603B030BD00242B
:104E8000FAE700000023FFF7E1BF00000139012924
:104E90008CBF002001207047002070470020704721
:104EA000002070477047000000230B70704700001F
:104EB00070470000704700000020704700207047D6
:104EC000002070474368C26893423CBF8268D15457
:104ED000436801334360012070470000F8B5054680
:104EE0000C468F180026BC4207D02B6814F8011B13
:104EF0009B68284698470644F5E73046F8BD000011
:104F00000020704700207047002070470020704745
:104F100038B590F89C308B4204460D460CD080F892
:104F20009C100CF075F92368C4F8A0005B6820465B
:104F3000984708B984F84D5038BD00007FB50D463C
:104F40001446194600267AB1531E0B4A6846CDE92D
:104F50000026089ACDE9025300F00EFA0198844227
:104F600004D92E5404B070BD1346EEE7002CF9D0DE
:104F70002C4404F8016CF5E72C71030808B410B553
:104F800085B007AC54F8043B00940394FFF7D6FFB8
:104F900005B0BDE8104001B07047000070B5044690
:104FA00008F0A8FF5E224FF4000108F08FFF0D4EBD
:104FB0000D4B1D6833783BB9E86A0422214648301E
:104FC0000CF02AF901233370EB6A2A2283F8462079
:104FD000EB6A93F89C301BB9044821460CF0ECF8BE
:104FE00070BD00BF6E3A002030260020107103080B
:104FF00007B503680DF10701DB69984720B19DF8FB
:10500000070003B05DF804FB4FF0FF30F9E7000044
:10501000F8B506460F4614460025AC420AD0336860
:1050200030469B699847431C01D12846F8BD785506
:105030000135F2E72046F9E70EB403B503AA036889
:1050400052F8041B5B680192984702B05DF804EBCC
:1050500003B0704700F090B913B5044608460191BB
:10506000FCF7CAF923680199DB680246204602B0C2
:10507000BDE810401847000070B500260446C0E99E
:10508000026601200D461AF07FFFB04208BF354688
:10509000206065602674204670BD000010B5037C5A
:1050A000044613B900681AF073FF204610BD0000D3
:1050B00070B5057C04460E46DDB9BFF35B8FC56055
:1050C000BFF35B8FBFF35B8F8560BFF35B8F43687C
:1050D0008B420CD000681AF05BFF314601201AF0B9
:1050E00053FF206010B96560284670BD66600125D9
:1050F000FAE70025F8E7000038B505460C4644B14C
:1051000021462846FFF7D4FF20B904EB4404A40845
:10511000F5E7204638BD00000023BFF35B8FC36076
:10512000BFF35B8FBFF35B8F8360BFF35B8F704711
:10513000BFF35B8F0068BFF35B8F704770B50546A8
:105140000C30FFF7F5FF05F1080604463046FFF77F
:10515000EFFFA04206D930466D68FFF7E9FF25440E
:10516000281A70BD3046FFF7E3FF201AF9E7000068
:1051700070B50546406898B105F10800FFF7D8FF03
:1051800005F10C0604463046FFF7D2FF8442304654
:1051900094BF6D680025FFF7CBFF013C2C44201A1B
:1051A00070BD000038B50C460546FFF7C7FFA042AA
:1051B00010D305F10800FFF7BBFF04446868B4FB97
:1051C000F0F100FB1144BFF35B8F0120AC60BFF333
:1051D0005B8F38BD0020FCE72DE9F04114460746FF
:1051E0000D46FFF7C5FF844228BF0446D4B1B84638
:1051F00058F80C6B4046FFF79BFF30442860404650
:105200007E68FFF795FF331A9C4203D86C6001203B
:10521000BDE8F0816B60A41B3B68AB602044E86094
:105220000220F5E72046F3E738B50C460546FFF7C0
:105230009FFFA04210D305F10C00FFF779FF044453
:105240006868B4FBF0F100FB1144BFF35B8F0120F1
:10525000EC60BFF35B8F38BD0020FCE72DE9FF4118
:10526000884669460746FFF7B7FF6C4606B204EB6F
:10527000C6060025B44209D06268206808EB050123
:105280001DF026FC636808341D44F3E729463846C0
:10529000FFF7CAFF284604B0BDE8F081F8B505461F
:1052A0000C300F46FFF744FF05F108060446304670
:1052B000FFF73EFFA042304688BF6C68FFF738FF1B
:1052C000201A386020B130462C68FFF731FF2044A7
:1052D000F8BD000073B5144606460D46FFF72EFFD5
:1052E000844228BF04460190DCB101A93046FFF793
:1052F000D5FF019B33B93268C5E90233C5E9002403
:1053000001200CE09C4238BF01942860019868603D
:105310008442F5D93368AB60241AEC60022002B0F5
:1053200070BD2046FBE700002DE9FF410F466946AE
:10533000FFF7D0FF6C4600B204EBC0050026AC427C
:1053400009D0D4F8048054F8081BB81942461DF05F
:10535000BFFB4644F3E7304604B0BDE8F0810000EF
:1053600038B50546FFF7E0FF044601462846FFF73B
:1053700019FF204638BD00002DE9F04F2DED028BBE
:1053800006468DB0904691F80090B9F1000F00F0FC
:10539000DE82B9F1250F08D04B1C039333684946D0
:1053A0009B68304698470399EDE791F801908B1C74
:1053B000B9F1250F0393F1D00025AA462C461F2CE6
:1053C0003BD8B9F12B0F2DD01CD8B9F1200F2BD021
:1053D000B9F1230F2ED0A9F13003DBB2092B36D857
:1053E00060064BBF05EB85050AEB8A0A03EB450512
:1053F00003EB4A0A4EBF05F0FF050AF0FF0A44F02E
:10540000200407E0B9F12D0F11D0B9F1300FE2D12E
:1054100044F00104039B13F8019B0393B9F1000FBF
:10542000CDD126E044F0020444F00404F2E744F055
:105430000804EFE744F01004ECE77F2CCBD92306F7
:1054400017D5B9F16C0F14D144F48074E2E7B9F1C7
:105450002E0F05D1620600F17A8244F04004D9E7AC
:10546000B9F16C0F02D144F08004D3E7B9F1680FB1
:10547000D0D0A9F14503022B61D809F1200944F0ED
:1054800010045FFA89F908F1070828F00708F8E81E
:105490000201FBF783FB14F0400F08BF062524F040
:1054A000C004B9F1650F08EE100AA4B250D144F05F
:1054B000400427060DD59FED977AF0EEC87AF4EEFA
:1054C000C77AF1EE10FAC2BF4FF63F73234043F0A4
:1054D000400414F0800346D03B2DA94628BF4FF06E
:1054E0003B0909F101095FFA89F907271722002111
:1054F00006A802931DF036FB4A46394606A8B0EED0
:10550000480A0CF04FF89DF81830019303F0090297
:10551000012A029B83462FD0A0072FD414F0040F3A
:105520000CBF00222022019911F00C0758D0002A4C
:1055300040F0AB82BAF1030F50D8174637E0A9F11B
:105540006503022B00F25B8124F01004A4B29AE7F9
:10555000B9F1660F02D144F08004AAE7002DA8D06B
:10556000013DEDB2A5E70A2D83BF0A2599462F46D6
:105570002F4698BF9946B9E72D22D4E72B22D2E7D0
:105580000427AAEB07072107FFB20AD43368029267
:105590009B6820213046013F984717F0FF07029A89
:1055A000F4D122B1336811469B6830469847019B7D
:1055B000594D13F0080F594B08BF1D46013D04F02B
:1055C000100415F8011F002900F0B5800CB1203936
:1055D000C9B2336830469B689847F2E70327D0E7A3
:1055E000CDF808B0002B36D0019BD944DB065FFA1A
:1055F00089F907D59DF81930312B04BF09F1FF391E
:105600005FFA89F94FFA89F3002B44DDB9F1080FED
:1056100028BF4FF0080914F0800304931ABF2BEA47
:10562000EB730133052302B101330DB1691C0B4447
:105630009A45C4BFAAEB0303DFB214F0090F2FD1C0
:1056400077B3336805929B6820213046013F984725
:10565000FFB2059AF4E76006DDD45D4504DB1BF17B
:10566000040FA8BF44F080046B1C06A90B4435B19D
:1056700013F80119302902D1013DEDB2F7E72106F7
:10568000C9D505F101095D455FFA89F906DDA5EB8C
:105690000B05EDB2BFE74FF00109BCE70025BAE703
:1056A00022B1336811469B6830469847220708D4D8
:1056B0003FB1336830219B683046013F9847FFB2C5
:1056C000F6E7049B002B47D02BEAEB74ABEB040A04
:1056D00006AB9A44ABEB09096D42A34517DBA14524
:1056E00015DA9AF80110013CA54219DC002900F0F6
:1056F000D281336830469B689847631C04D1336875
:105700002E219B68304698470AF1010AE5E73021CF
:10571000E9E700BF7F96184B5C71030858710308D6
:10572000A34507D19DF81930352B0FD802D1019B25
:10573000DD060BD559B9002F3FF435AE3368202173
:105740009B683046013F9847FFB2F4E73121336848
:105750009B6830469847EEE79DF8191031291EBF27
:10576000019B03F0EF030193336830469B68984731
:10577000E5B9336814F0100F14BF452165219B680B
:1057800030469847BBF1000F29DACBF100030293B2
:105790002D21336830469B6898473021029B092BA6
:1057A00023DD01310A3BC9B20293F7E733682E21AA
:1057B0009B68304698470235EDB24FF002094B46E0
:1057C0000CAA1A44336812F8181C9B6809F10109E5
:1057D0005FFA89F930469847A945F0D1C9E702D167
:1057E000019BDC06D1D42B21D3E7336830469B687C
:1057F00098470299336830319B68C9B2A9E7B9F17B
:10580000630F37D0B9F1730F4FD0B9F1640F63D183
:1058100024F0900714F4807FBFB20DF118097BD0FB
:1058200008F1070222F007029046516858F8080B69
:10583000002904DA404261EB410147F080070A2366
:105840004A4600F07BF9A0EB0900C4B27B0640F1A8
:105850009F8027F00109AC421FFA89F980F0D280BD
:1058600007F01403102B03D127F011071FFA87F953
:10587000AB468FE058F8043B8DF8183001250DF148
:105880001809200701D4AA451CD84D445746A945FC
:105890003FF451AF336819F8011B9B6830469847B5
:1058A000002FF4D0013FFFB2F1E758F8049B14F049
:1058B000400F14BF29464FF0FF3148461DF03EFE11
:1058C0000546DEE7336820219B6830460AF1FF3A3F
:1058D00098475FFA8AFAD6E7B9F1690F98D0B9F11B
:1058E000750F27D124F01004A7B20A2317F4807F84
:1058F000DBB20DF1180944D008F1070828F00708B9
:10590000F8E802014A4600F019F9A0EB090027F077
:105910008007C4B2BFB299E758F8040B0028B8BF9B
:1059200040424FF00A024946B8BF47F0800700F0F6
:10593000B7F888E724F00607B9F1700FBFB214D0AA
:105940000AD8B9F1580F13D0B9F16F0F17D00DB0B5
:10595000BDEC028BBDE8F08FB9F1780FF7D1F906F5
:1059600001D547F004071023C0E747F01007F6E71A
:10597000E20601D547F006074FF40473B6E70823A3
:10598000B4E758F8040B1A46494600F089F8BCE71A
:10599000A346B94619F0100F41D00CAB234413F8BD
:1059A000193C302B30D129F016091FFA89F919F06A
:1059B000080744D119F0010F35D0DA4545D904EB79
:1059C0000A05A5EB0B05EDB2336819F0100F9B68C3
:1059D0003FD030213046984719F0040F08D0336883
:1059E00019F0020F9B6814BF582178213046984760
:1059F0003368AC429B6839D230213046013D98472C
:105A0000EDB2F5E7A346C5E719F0040F02D10BF19B
:105A1000010B01E00BF1020B5FFA8BFBC7E719F0FA
:105A2000860FC4D0F3E73368DA459B680FD920218D
:105A300030460BF1010B98475FFA8BFBF3E7DA4531
:105A400005D9AAEB0B07FFB2BEE72546BCE7002746
:105A5000BAE719F0860FCBD019F0020F14BF2B2133
:105A6000202119F0800F18BF2D21BFE7651E06AB5E
:105A700053FA85F5336815F801199B68013CE4B2C7
:105A800030469847002CF5D155E6BAF1040F3FF6A1
:105A900077AD002786E5A3457FF44DAE42E600BF13
:105AA000082A30B505D10346C008FCD130330B704D
:105AB0000DE0102A0DD100F00F0202F13003392B56
:105AC00088BF02F13703000901F8013BF3D1084612
:105AD00030BD03460022DCB223F00103023342F161
:105AE0000002580840EAC270C31842EB520218097B
:105AF00040EA0270C01842EB1212030A43EA026342
:105B0000181842EB1222030C43EA02431B1842EB23
:105B10001242D31842F100001B0943EA0073C3EBA1
:105B20004315C3EB85053034020904EB450453EA01
:105B3000101001F8014BCED1C9E70000082B30B599
:105B40000AD10346C00840EA4170C90850EA01047E
:105B5000F7D13033137013E0102B13D100F00F0482
:105B600004F13003392B4FEA101088BF04F13703DA
:105B700040EA0170090902F8013B50EA0103EDD146
:105B8000104630BD20F00104023441F100036108E9
:105B900041EAC3710C1943EB5303210941EA037134
:105BA0000C1943EB1313210A41EA03610C1943EB6F
:105BB0001323210C41EA0341091943EB13435918FC
:105BC00043F10003C5B2080940EA0370C0EB40147A
:105BD000C0EB84043035190905EB440550EA131372
:105BE00002F8015BCED1CBE770EE600ADFED057AFB
:105BF000F0EEE00AF4EEE70AF1EE10FA4CBF0120F5
:105C0000002070470000003408B52DED028B9FED99
:105C1000088AF0EE480A1BF00FF9B5EEC00AF1EE63
:105C200010FA48BF30EE080ABDEC028B08BD00BF79
:105C30000000B44310B5B4EE400AF1EE10FA2DEDB9
:105C4000028B0446B0EE608AF0EE418A0FD708F06E
:105C500051F9A2B24FF4806108F038F938EE288A81
:105C6000B6EE000A28EE000ABDEC028B10BDB4EEC1
:105C7000E00AF1EE10FA07D4B4EE410AF1EE10FAA0
:105C8000C8BFB0EE410AEFE7B0EE600AECE70000F3
:105C9000884203D39042014628BF11460846704708
:105CA000884203DB90420146A8BF11460846704770
:105CB000094A136849F2690099B21B0C00FB0133D1
:105CC0001360064B186844F2506182B2000C01FB6D
:105CD0000200186080B270470823002004230020CF
:105CE000036800EE103A7047024682B000685168BF
:105CF0006B4603C39DED000B02B0704701234A1EA3
:105D000003FA02F202421CBF8B40C01A7047000027
:105D1000D0ED010A90ED021AD0ED007A60EE200A73
:105D200020EE011A27EE800A88B008B0704700BF45
:105D300091ED005AD1ED015A91ED026AD0ED006A61
:105D400090ED017AD0ED027A76EE856A37EE257A0B
:105D500077EE867AC0ED006A80ED017AC0ED027AB6
:105D6000704700BFD0ED006A90ED017AD0ED027A65
:105D700066EE806A27EE007A27EE800AC0ED006AA0
:105D800080ED017A80ED020A704700BF90ED007A45
:105D9000D0ED017A90ED026AC7EE006A87EE807A54
:105DA000C6EE007AC0ED006A80ED017AC0ED027A9D
:105DB000704700BFD0ED007AF4EE677AF1EE10FA8A
:105DC00010D6D0ED017AF4EE677AF1EE10FA09D62A
:105DD000D0ED027AF4EE677AF1EE10FA6CBF012092
:105DE0000020704701207047D0ED007A9FED0F7AB8
:105DF000F0EEE77AF4EE477AF1EE10FA14DCD0ED2B
:105E0000017AF0EEE77AF4EE477AF1EE10FA0BDC65
:105E1000D0ED027AF0EEE77AF4EE477AF1EE10FA7E
:105E2000CCBF01200020704701207047FFFF7F7F1B
:105E300008B52B2900F28282DFE811F04400460207
:105E4000400233022A021B02680157014E016E0113
:105E500058003F01790184014500D4000401EF009E
:105E60003901290120010B0191010A02E501DF013D
:105E700045005800D101C401B901AA019F01C70022
:105E8000BE00B700AA009B00700061002C006D02EC
:105E900062025102D0ED016AD0ED007A9FEDDD6A19
:105EA00036EEA77A77EEE67AD0ED026A27EE067A2A
:105EB00067EE867AF1EE666AC0ED016A80ED027ADD
:105EC000C0ED007A08BD90ED007AD0ED016AD0ED0A
:105ED000027AF1EE666AB1EE477AF1EE677AC0EDCA
:105EE000006A80ED017AC0ED027A08BDD0ED027A39
:105EF000036842680260F1EE677A4360F3E7D0ED31
:105F0000007A90ED026ADFEDC36A37EE867A77EEAB
:105F1000C67A27EE267A67EEA67ACFE7D0ED017A29
:105F2000DFEDBD5ADFEDBD6A9FEDBD7A90ED006AF1
:105F3000DFEDBC4A9FEDBC5A67EEA66A27EE877A72
:105F400067EEA57ADFEDB95AE6EE246AA6EE057A89
:105F5000E6EE257ADFEDB64A90ED026A9FEDB55A7E
:105F6000DFEDB55AE6EE246AA6EE057AE6EE257A6E
:105F7000B5E790ED027AD0ED007A43688360B1EE28
:105F8000477AF1EE677A80ED007AC0ED017A08BDBC
:105F900090ED017AD0ED007A8368B1EE477AF1EEA8
:105FA000677A80ED027A0360EFE7816802684368F0
:105FB00041608260036008BDD0ED017A83680268A9
:105FC000F1EE677AC0ED017AF3E790ED027AD0ED59
:105FD000017A0368B1EE477AF1EE677A80ED017AD3
:105FE00083606DE7D0ED007A90ED017ADFED935A92
:105FF0009FED886A77EE876A77EEC77A90ED027A2E
:1060000066EEA56A67EE867AB1EE477AC0ED016A60
:10601000C0ED007A80ED027A08BD90ED026AD0ED05
:10602000007ADFED7C6A436837EE867A77EEC67ACF
:1060300067EEA67A27EE267A8360C0ED017A80EDBE
:10604000007A08BDD0ED027A43688360F1EE677A8A
:106050009BE7D0ED026AD0ED007A9FED6E6A37EED5
:10606000E67A77EEA67AD0ED016A67EE867AF1EEEF
:10607000666A27EE067AC0ED026ADEE7D0ED017AA5
:106080008368F1EE677AC0ED027A436008BDD0ED17
:10609000026AD0ED007A9FED5F6A436837EEE67AD8
:1060A00077EEA67ADFED656A67EE867AC2E78268E8
:1060B0004168036881600260E7E7D0ED017A90ED06
:1060C000007A9FED546A77EE876A77EEC77A90ED93
:1060D000027A66EE866A95E790ED017AD0ED027A53
:1060E000B1EE477AF1EE677AFBE6D0ED007A90EDFB
:1060F000016ADFED486A36EE677A77EE867A27EE38
:10610000267A67EEA67A80ED017AD9E6D0ED007A9C
:106110004368F1EE677A46E7D0ED007A90ED017AB8
:106120009FED3C6A77EEC76A77EE877ACFE790ED0E
:10613000007AD0ED027AB1EE477AF1EE677A80ED1F
:10614000007AD0E6D0ED007A90ED017ADFED315A99
:106150009FED3A6A77EE676A77EE877A4EE790EDC1
:10616000017AD0ED027A0368B1EE477AF1EE677AF0
:1061700080ED027AC0ED007A87E7D0ED007A4368BF
:1061800082684260F1EE677AC0ED007A836008BDF4
:10619000D0ED026AD0ED017A90ED007AF1EE666AF8
:1061A000B1EE477AF1EE677AC0ED016AC7E7D0ED4C
:1061B000017A90ED007A83684360F1EE677AB1EE80
:1061C000477A7BE6D0ED016AD0ED027A90ED007A55
:1061D000F1EE666AF1EE677AB1EE477A6CE690ED21
:1061E000027AD0ED007A4368B1EE477AF1EE677A31
:1061F00080ED017AC0ED027ADCE6D0ED027A036828
:10620000F1EE677AECE6D0ED007A8368F1EE677A1A
:10621000F0E700BFF304353FDB26B93E46D0BC3E75
:10622000C9355BBFCF78123E4F0DAABEC6AC6EBF5C
:106230004D1F6BBFF184CABEF63BCC23F30435BFC0
:10624000F304353F81177E3FA296F93DA296F9BD32
:10625000D0ED026AD0ED007A5FED075A1FED096AB2
:1062600037EEA67A77EEE67AD0ED016A67EEA57A88
:10627000FDE6D0ED006AD0ED017A1FED106A37EE31
:10628000A67A77EEE67A5FED126A27EE067A38E7AD
:1062900090ED007AD0ED017AB1EE477AF1EE677AAF
:1062A00071E6D0ED016AD0ED007A1FED1B6A37EE82
:1062B000E67A77EEA67A5FED1F6AE6E7D0ED017A1F
:1062C0000368F1EE677A55E7D0ED007A90ED016A48
:1062D0005FED256A37EE867A77EEC67A0FE7D0ED66
:1062E000017A90ED026A5FED2A6A36EE677A77EE00
:1062F000867A27EE267A67EEA67A80ED027A44E661
:10630000D0ED017A90ED026A5FED336A37EE867A5E
:1063100077EEC67AEDE7D0ED027A1FED366A1FED13
:10632000367AD0ED006A5FED375A27EE877A67EE4E
:10633000867AA6EE867AE6EEA57A00E707F0DAFD21
:10634000BDE8084040F211124FF4800107F0BEBDD5
:1063500090ED020A90ED017AD0ED007A20EE000A6D
:10636000A7EE070AA7EEA70AB1EEC00A704700BF62
:106370007047000038B5056804462DB12846FEF781
:106380008DFE2846FEF7F2FA204638BD1346024637
:10639000014802F015B900BFC23A002013B504222B
:1063A000054B0193044601460DEB0200FFF7EEFF9B
:1063B000024B1C8002B010BDFFFF3F00B43A00202A
:1063C00007B5502304228DF80430412300210DEB42
:1063D00002008DF8053006238DF806308DF8071081
:1063E000FFF7D4FF0420FFF7D9FF03B05DF804FBEB
:1063F00000EB0212907B20B91BB19289120758BFA3
:106400003F20984008447047430608D4000A08D04B
:10641000054B1B88184214BF012000207047002044
:1064200070470120704700BFB83A002010B50B4BF1
:106430001A880B4B01301B6880B2142404FB003314
:10644000824207D9DC898C4203F1140304D0013065
:1064500080B2F5E7002010BD0120FCE7C63A00201D
:10646000C83A002082898368D20648BF1B68184654
:106470007047000082898368D20648BF1B681846AF
:106480007047000007B5042300220DEB03010B4801
:10649000019202F05DF89DF80430502B07D19DF871
:1064A0000530412B03D19DF80630062B01D0FFF7B4
:1064B00087FF012003B05DF804FB00BFC23A002053
:1064C00082894368920705D51B68181E18BF0120F2
:1064D0000B6070470120FBE737B58B891446DA075C
:1064E0000D4605D523684A6813442360012012E055
:1064F0009B07FBD50A4B1B68142201A902FB003045
:10650000FFF7DEFF48B1019922686B680A44D3584F
:106510001BB15B1A236003B030BD0020FBE700BF56
:10652000C83A00202DE9F04F8BB01F469DF85480EB
:10653000069114235343059308F10603DBB2054685
:1065400016464FF0000B07935FFA8BFA07EB0A1918
:1065500099F80F40002C4CD0062C28D1B8F10B0F25
:1065600021D84846FFF77EFF0446C8B1169B099321
:1065700009AA49463046FFF7AFFF88B11499434650
:1065800052463846FFF734FF099B0293079B069952
:10659000CDE90003324623462846FFF7C3FF18B96A
:1065A0000BF1010BD0E700200BB0BDE8F08F149980
:1065B000434652463846FFF71BFFB0EB953FEFD1FD
:1065C000C5F30423A342EBD10B4C059B206809A91A
:1065D0001844FFF775FF0028E2D0D9F80430099A73
:1065E0001344169A1344069A13602068059B1844B6
:1065F000DAE72046D8E700BFC83A00202DE9F04F7F
:106600001F4B5FFA80F8B3F800A0C0F3403348EAAC
:1066100003281C4B1E680F4687B00546C0F3042BA9
:1066200000211FFA81F9CA4527D9F3894345344629
:1066300020D1337C062B0FD13046FFF71BFFC8B1AA
:106640000023CDE9013300934A46034639462846E4
:10665000FFF768FF044609E09B450BD105A93046CA
:10666000FFF72EFF0028F5D0059B3B60204607B0C2
:10667000BDE8F08F01311436D3E70024F6E700BF00
:10668000C63A0020C83A00202DE9F04F98468DB058
:10669000142353430693484B9DF85890DDF868B097
:1066A00004461868069B0E4618440AA91746FFF7C9
:1066B00007FF00287DD00023079309F10603DBB212
:1066C00009939DF81CA006EB0A15EB7B002B70D0FC
:1066D000062B3BD12846FFF7C5FE0890002831D095
:1066E000B9F10B0F65D8179B0B930BAA29463846B7
:1066F000FFF7F2FE30B39BF80030012B59D85A1C3B
:106700000BEB83038BF8002041465D6052464B46FD
:106710003046FFF76DFE1B9A0899CDE904B2199A2D
:106720000392189A02920B9A0192099A00920346D8
:106730003A462046FFF7A8FF00BB9BF80030013B1C
:106740008BF80030079B01330793BAE7179A686804
:1067500010440A9A1044A04213D14B465246414677
:106760003046FFF745FE189B1B9A1860199B1D6069
:1067700000231370104B1868069B18440DB0BDE839
:10678000F08F052BDED1031D9C4203D000F10803DE
:106790009C42D7D11B9B201A8008187052464B464A
:1067A00041463046FFF724FE189B1860199B1D6078
:1067B000E0E70020E2E700BFC83A00202DE9F04FF3
:1067C0008BB00025DFF8A4A0079306460F4690463D
:1067D0001560254B1B881FFA85FB5B4541D9DAF80C
:1067E0000000142303FB0B0409A9204694F8109021
:1067F000FFF766FE98B3B9F1060F17D12046FFF7F1
:1068000039FE014658B3149B0593079B0297CDE9C7
:1068100003830023CDE900335A463046FFF734FFA7
:106820000446E0B120460BB0BDE8F08F0998B042B5
:1068300004D1149A00233B601370F3E7B9F1050FFC
:106840000DD1031D9E4203D000F108039E4206D1E4
:10685000149B301A8008187000233B60E2E7013572
:10686000B7E70024DEE700BFC63A0020C83A0020A0
:106870002DE9F04798460D88234B0446C5F30809D7
:10688000186809EB890588B000EB850507A928463B
:10689000119E95F810A01746FFF712FE20B90025AB
:1068A000284608B0BDE8F0870021BAF1060FC8F805
:1068B000001013D12846FFF7DDFD0028EFD0109B14
:1068C0000091CDE90383CDE901170B4605960146FA
:1068D0004A462046FFF7D8FE0546E1E70798A04262
:1068E00002D139603170DBE7BAF1050FD7D1031D52
:1068F0009C4203D000F108039C42D0D1241AA40882
:10690000002334703B60CBE7C83A00200138C0B2A6
:1069100004289ABF014B185C00207047747203086A
:106920002DE9F04F2DED028B83B000240093931DD1
:10693000DBB208EE103A05460E461746A246A046C0
:106940004FF0010BE0B2010105EB001090F80F9041
:10695000B9F1000F5AD0837B3F2B02D92E480AF0A1
:106960002BFC17B1002B08BF3F23C3F1200EA3F16E
:10697000200C2AFA03F208FA0EFE28FA0CFC42EA6E
:106980000E0242EA0C0212F0010FC3F1200CA3F137
:106990002002E3D10BFA02F22BFA0CFC42EA0C02C1
:1069A0000BFA03F3B9F1060F43EA0A0A42EA0808B0
:1069B00013D10B2FD2D8FFF755FD814658B1685837
:1069C000FAF71AFD009B1844C3B218EE102A31469C
:1069D0004846FFF7A5FF0134B4E74846FFF796FFA6
:1069E00001900028BAD06858FAF706FD009B1844B9
:1069F000C0B2B9F1050F04BF0230C0B21028019B2C
:106A0000ACD83088043003443380E4E703B0BDECF5
:106A1000028BBDE8F08F00BF607103082DE9F04FD5
:106A200085B00423DFF89890ADF80E3000244FF0C5
:106A3000140A214B1B881FFA84F8434539D9D9F829
:106A400000300AFB08F15D182F7CB5F80EB0062F58
:106A500023D1B8F1000F02D118480AF0ADFB284647
:106A60000193FFF707FD0646A8B1019B5858FAF7B6
:106A7000C3FC0022C3B20DF10E013046FFF750FFF8
:106A800059464046FFF7D2FC0028E5D1062F02D038
:106A9000AB899B07E0D40134CBE73846FFF736FFDC
:106AA0000028D9D0BDF80E3004331844ADF80E00DC
:106AB000E6E705B0BDE8F08FC63A00206071030834
:106AC000C83A0020437803F01F021F2A0FD0027833
:106AD000C3F3401342EA032340F2FF12934206D06D
:106AE00000680138C31C94BF0020012070470120BA
:106AF000704700002DE9F341224FDFF890800646F1
:106B00000D4604247B88A34237D904230DEB0301EF
:106B10002246384601F01CFD9DF80510737881EA85
:106B20000302D20618D196F800C09DF80400C3F302
:106B30004013C1F340124CEA032340EA022293427D
:106B40000AD13268019B534013EA080F04D12C800C
:106B5000012002B0BDE8F08101A8FFF7B3FF20B12A
:106B6000094B2C801C800020F3E701F01F00FFF789
:106B7000CDFE031D1C44A4B2C4E74FF6FF732B8067
:106B8000F1E700BFC23A0020B43A002000C0FFFF86
:106B900070B50C462046114615461E461CF0CEFC2C
:106BA000831CAB420AD85F22225422180330A84229
:106BB00006F1580656709CBF0022E25470BD0000DA
:106BC0002DE9F74FDDE90D5407468A461646096858
:106BD0009DF830809B4622469DF83C300093284625
:106BE0001CF098FC4FF000099BF800105FFA89F246
:106BF0009142019212D9214628461CF09FFCC0B256
:106C00008442019A07D90BEB82025168221A096863
:106C100028441CF07FFC09F10109E5E7E6B12146B3
:106C200028461CF08BFCC3B29C4204D93168E21A9E
:106C3000E8181CF06FFC009B13B9B8F1000F13D0DB
:106C4000F37B052B10D1434622462946384603B034
:106C5000BDE8F04FFFF79CBF009B13B9B8F1000FE0
:106C600002D09AF81030ECE703B0BDE8F08F0000D6
:106C7000F0B58BB007AC1F460023C4E9013307937E
:106C80000DF11303CDE90043154606AB05AA0646F0
:106C9000FFF7EEFD014610B928700BB0F0BD9DF86E
:106CA0004030069A0195CDE902739DF813300093A8
:106CB00030462346FFF784FFEFE700002DE9F04F51
:106CC000984689B014234B43DFF828A10392044669
:106CD0000E4604934FF000095FFA89F52B0108EB8B
:106CE0000515059395F80FB0BBF1000F7FD0BBF1F0
:106CF000060F58F803702AD13846FAF77DFB39465B
:106D0000024620461CF0D0FB002869D12846FFF738
:106D1000A9FB0746002863D0039B079307AA2946CF
:106D20003046FFF7D9FB00285AD0059B58F80300DE
:106D3000FAF762FB129B0093079A3B4631462044C8
:106D4000FFF7BCFF00284BD009B0BDE8F08F3946F3
:106D500020461CF079FB88B9DAF80000049B07A9EB
:106D60001844FFF7ADFB00283AD0129B83F800B01F
:106D70006868079B1844039B1844E5E7BBF1050FBF
:106D80002ED1102138461CF0D9FB5FFA80FB5A4601
:106D9000394620461CF0AAFB10BB14F90B305F2BC0
:106DA0001ED10BF1010B14F80B30583B022B17D8F6
:106DB000DAF80000049B07A91844FFF781FB78B1BB
:106DC0006868079B129A1844039B184404231370A5
:106DD00014F90B30592B06D05A2B06D0582BB3D0B0
:106DE00009F1010978E70430AEE70830ACE758460E
:106DF000AAE700BFC83A00202DE9F04F8BB0DFF8BA
:106E0000C8B002910446174600252E4B1B881FFA76
:106E100085FA534552D9142253465343DBF80020D8
:106E200002EB0309D35899F81080B8F1060F33D15B
:106E30001021184603931CF081FB039B5FFA80F836
:106E40004246194620461CF051FB0646002833D125
:106E50004846FFF70FFB034670B3029A009204EB1B
:106E6000080032465146FFF729FF804620B37FB124
:106E70000DF11303009306AA07AB05A9CDE9076638
:106E800005960996FFF79AFC069B0BB19B893B8000
:106E900040460BB0BDE8F08F194620461CF0D4FAEE
:106EA00050B9029B07A983F800804846FFF708FB0A
:106EB00020B1DDF81C80EBE70135A6E74FF00008B4
:106EC000E6E700BFC63A0020C83A002030B50B4BB9
:106ED0001C880B4B1B68002295B2AC420CD91D7C60
:106EE000062D06D15D68854203D1DB890B80012028
:106EF00030BD01321433EFE70020F9E7C63A002035
:106F0000C83A002010B590B00023CDE908330693AD
:106F10000A930DF11703009306A908AB07AA0446CC
:106F2000FFF74CFC014668B111230122CDE9023282
:106F30000BAB01939DF817300093079A08AB2046DE
:106F4000FFF73EFE10B010BDF0B5304D87B040F2F7
:106F5000A51202908DF80C1006460C4601A8291DBA
:106F6000FDF790FE052204A92868FEF7DDF9074623
:106F700001A8FDF7A9FE052F06D1049BB34203D15A
:106F80009DF81430A3423ED0214E224F4FF4B072F0
:106F9000314601A8FDF776FE2868FEF7E9F80428D7
:106FA00021D92868052202A9FEF758F9431F5C423F
:106FB0005C4101A8FDF788FE2CBB3C68E36A93F8AE
:106FC0009C3093B9A06A036801211B699847A06AA5
:106FD00003684FF4FA719B689847A06A0368002120
:106FE0001B699847D2E70024E3E7A06A03681B6C9B
:106FF00098470028E6D006F07DFF40F2FA424FF4B1
:10700000801106F063FF07B0F0BD00BF8C3A00208E
:10701000903A0020302600202DE9F341154E164FFE
:10702000C92406F10408013CA4B2FCB140F24B12A1
:10703000414601A8FDF726FE3068FEF77FF80546B9
:1070400001A8FDF741FE042D10D93D68A86A036828
:107050000A211B699847A86A03680A215B68984758
:10706000A86A036800211B699847DCE702B0BDE805
:10707000F08100BF8C3A00203026002000B58BB094
:107080000023CDE90733049309930DF10D03009319
:1070900005AA07AB04A9FFF791FB10B3059B23B327
:1070A000DB7BC2898DF8182003F01F03C2F3002296
:1070B0001B0243EA4233049A43EA82339DF81820C4
:1070C0000DF10E01134306A80693FFF713FD40B11F
:1070D0009DF8193003F01F03052B03D09DF80D30E8
:1070E00003B100200BB05DF804FB037CD9E700007E
:1070F000F0B5144F3B8889B006460D46FBB10DF143
:107100000B030024009304AA05AB03A9CDE90544B1
:1071100003940794FFF752FB88B10B4B38881B6828
:10712000A2B290420BD91A46013411688E4203F183
:107130000C03F5D1137A2B70012009B0F0BD0020AB
:10714000FBE700BFBC3A0020B03A002013B50DF1B8
:1071500007010446FFF7CCFF10B92046FFF78EFF6A
:1071600002B010BD07B5074B1B884BB10DF10701ED
:10717000FFF7BEFF08B19DF8070003B05DF804FB00
:107180001846FAE7AC3A002010B50C46FFF7EAFFC4
:1071900040B9A30608D5054B1B6813B1186AC0F3A4
:1071A000800010BD0020FCE70120FAE748690020BC
:1071B0000138032816D8DFE800F002080E13FDEEB0
:1071C000C07A17EE903A0B707047BDEEC00A10EE11
:1071D000103A0B807047BDEEC00A81ED000A70477F
:1071E00081ED000A7047000037B5036803F00043E3
:1071F00003600A4B1B880C4613B9002003B030BD56
:10720000074D01A92868FFF75BF90028F5D014B1F4
:107210002B681B7C23700198F0E700BFC63A002062
:10722000C83A00202DE9F04F8FB09B469DF8703092
:107230000B93142343439DF860901A9D0A930746CD
:1072400088460892002307939DF81CA008EB0A16B5
:10725000F47B002C00F0BC80B089FFF7D5F8002843
:1072600000F0B380062C2FD13046FFF7FBF8044620
:10727000002800F0AA80199B0D930DAA31463846CC
:10728000FFF72AF9002800F0A0804B4652465946E5
:107290004046FFF7ADF81D9A05920B9A04921B9A8F
:1072A000CDE902520D9A019209F10602D2B20346CB
:1072B00000922146089A3846FFF7B4FF002800F0F4
:1072C00084800FB0BDE8F08F089B1B780993002BDA
:1072D0003CD02B8867F308032B8052464B46594617
:1072E0004046FFF785F83B4B03EA40302B6823F01C
:1072F000FF4323F4FF0323F4FC4318431B9B286044
:1073000003B11C70344B18680A9B0DA91844FFF791
:10731000D7F8002859D00D9A73681344199A981811
:107320000B9A002ACDD02D4A1278002AC9D0F27BC0
:10733000012AC6D1B2895207C3D5199A9B56002B90
:10734000BFD1EB7843F08003EB70BAE74B4652466F
:1073500059464046FFF74CF82B68C3F35133984227
:1073600033D1089A0123137095F90330002B06DA04
:10737000EB78099A62F3C713EB701046A1E7052C6E
:1073800023D16B78C3F34302022A1ED8013262F381
:1073900044036B701B9B13B11B9A042313700E4B99
:1073A00018680A9B0DA91844FFF78AF868B170683D
:1073B0000D9C95F801B0199B2044CBF3430B184466
:1073C0000BF1FF3B00EB8B007BE7079B01333AE7B8
:1073D000204676E700E0FF7FC83A00200C2300201B
:1073E0002DE9F04F8BB0DFF8EC9004880792002273
:1073F0008DF82720B9F800201F46C4F308039A42ED
:1074000005460E461C4662D9DFF8CC801BB2D8F880
:10741000001003EB83039A0001EB83031B7C052B15
:1074200018D14378C3F34301022915D8013161F320
:10743000440343700EB104233370D8F80010687809
:107440000A44C0F34300431E506800EB83000BB0B6
:10745000BDE8F08F062B04D001340123A4B28DF8CF
:1074600027304FF0140B4FF0000AB9F80030A34258
:107470002DD9D8F800200BFB04229089FEF7C4FF19
:10748000B8B1117C062917D11046FEF7F3FF01466B
:1074900078B1079B0597CDE90363CDE901A5CDF848
:1074A00000A000230DF127022046FFF7BBFE0028B5
:1074B000CDD10134A4B2D8E72B68C4F3080403F09B
:1074C000004323432B6006B131705068BFE70020B2
:1074D000BDE700BFC63A0020C83A002073B5054694
:1074E0000C461646334601220DF107012846FFF7E8
:1074F00077FF28B19DF80730042BF3D804B123702F
:1075000002B070BDF8B514460746002220460E466C
:10751000FFF76AFE002540B1BD4206D00022314689
:107520002046FFF7DBFF0135F5E7F8BD01390329F8
:107530000BD8DFE801F00204060800F07BBF00F082
:10754000B1BF00F0D7BF00F033BF9FED010A704715
:107550000000C07F37B5037A02888DF8042003F05D
:107560001F03C2F300221B0243EA4233426843EA8C
:1075700082339DF804200C4613430DF1020101A84B
:107580000193FFF7B7FA054670B19DF8050000F0CA
:107590001F00FFF7BBF9BDF802200432034692B288
:1075A0000348214600F0D4FF284603B030BD00BF99
:1075B000C23A00202DE9F0472DED028B82B004463F
:1075C00000AF007AFFF7A2F9C31D23F00703E946D5
:1075D000ADEB030D0E46804669462046F0EE408A2C
:1075E000EA46FFF7B7FF88B3E0680022F91DFFF70E
:1075F00003FC054640B9344BE2681B68334998697F
:1076000003681B68984721E0B2071BD5227AFB79F3
:107610009A4222D1F7EE000AB0EE680AFEF7E4FAC9
:10762000D8B1D6B94246514628461BF041FA68B156
:107630005146424628461BF04BFA31462846FFF792
:1076400083FC03E0FFF71AFD0028DFD00837CD46A2
:10765000BD46BDEC028BBDE8F087FB79042B07D952
:10766000194BE2681B681A49986903681B68C9E7E7
:10767000217A0429F4D85046FFF758FFF307B0EEFB
:10768000408A0BD5FFEE000AFEF7AEFA9FED110A15
:107690000028B7EE008A08BFB0EE408AF979284684
:1076A000FFF744FFF0EE400AB0EE480AFEF79CFAFE
:1076B00002460028CAD1294628EE280AF879FFF7A1
:1076C00077FD1146BAE700BF302600207471030829
:1076D0008D7103080000000070B515462DED028B7A
:1076E0000446B0EE408A00EB0116B44207D02046B3
:1076F0002946B0EE480AFFF75DFF1034F5E7BDEC10
:10770000028BBDE87040FFF787BC0000B7EE000AAF
:10771000FFF7E2BFB4EE400AF1EE10FA10B50446EE
:107720000CD69FED327AF0EEC07AF4EE477AF1EEA5
:1077300010FA03DC042902D180ED000A10BD0329F0
:1077400019D1B5EEC00A9FED2A7ADFED2A7A9FEDB6
:107750002A1ADFED2A0AF1EE10FA58BFF0EE477A46
:1077600030EE270A40F6C900FEF764FABDEEC00A03
:1077700084ED000AE2E702291AD1B5EEC00A9FEDB6
:107780001C7ADFED1C7A9FED1E1ADFED1E0AF1EE6A
:1077900010FA58BFF0EE477A30EE270A40F6CE00D6
:1077A000FEF748FABDEEC00A10EE103A2380C5E796
:1077B0000129C3D1B5EEC00A9FED0D7ADFED0D7A38
:1077C0009FED111ADFED110AF1EE10FA58BFF0EE3D
:1077D000477A30EE270A40F6D300FEF72BFAFDEE8B
:1077E000C07A17EE903A2370A8E700BFFFFF7F7FB3
:1077F0000AD7233C0AD723BC0000004F000000CF6B
:1078000000FEFF46000000C70000FE42000000C36B
:107810002DE9F3411D4690F90030232B0F46904689
:107820004FF000042CD01749019401AA1CF038FD38
:10783000064618B9002002B0BDE8F081F9F7DCFD7A
:107840001028F7D80F4901AA20461CF029FD00286E
:10785000F0D021461CF0A0FC0A4988ED000A01AADC
:107860003E6020461CF01CFD30B10749F9F7BAFD17
:1078700010B901202870DEE700232B700120DAE721
:107880002046D8E7A8710308AF71030830B5044655
:107890009DB00D4606F008FF01232146002206F0A8
:1078A00091FE431C044624D006F0FEFE23466322CC
:1078B00003A906F0BFFEA0B10DF1020302AA01A9BF
:1078C00003A8FFF7A5FF0028EED0019800220DF1D4
:1078D0000301FFF791FA0028E6D02B8801332B80B3
:1078E000E2E706F0E1FE214606F096FE01201DB01B
:1078F00030BD0020FBE700002DE9F0479EB01546A3
:10790000019006F0D1FE01230199002206F05AFEF3
:10791000431C064602D1334809F04EFCDFF8CCA0E8
:10792000DFF8CC80DFF8CC90012706F0BDFE3346AF
:10793000632205A906F07EFEF0B10DF10A0304AA48
:1079400003A905A8FFF764FF0028EED003980022E2
:107950000DF10B01FFF750FA044600283FD02A88AA
:10796000BAF80030934212D806F0C4FA40F64C122E
:107970004FF4801106F0AAFA06F096FE314606F0A2
:107980004BFE194B01201F701EB0BDE8F0870C2084
:10799000D8F8001042438C502A88D8F80030049957
:1079A00000FB0232516029889DF80A2000FB013358
:1079B0001A7222B1B9F800300133A9F800302B88CF
:1079C00001332B802046FFF759FB0028ADD19DF8ED
:1079D0000B109DED040A2046FFF79CFEA5E7074625
:1079E000A3E700BFBC710308C03A0020BE3A0020E4
:1079F000B03A0020AC3A00202DE9F7430D46064688
:107A000000286DD018F0ECFA074610B9354809F097
:107A1000D3FB00233449ADF8003001AA01931CF0D8
:107A20003FFCDFF8C48088B16946FFF72FFF0446AA
:107A300030B9384618F0ACFA204603B0BDE8F08300
:107A400001AA414600201CF02BFCECE7DFF8A890CF
:107A5000384618F09DFAD9F8000008B1FCF78AFF03
:107A6000224BDFF89880224F00241C80BDF80030A4
:107A7000A8F800400C2058433C80FCF775FFC9F87B
:107A8000000008B91B48C2E7BDF80030A8F8003074
:107A900023B33046019418F0A3FA06460028B5D067
:107AA0001149ADF8024001AA1CF0FAFBDFF838805A
:107AB00070B10DF102022946FFF71EFF044608B916
:107AC0003046B7E701AA414600201CF0E9FBEFE78A
:107AD000304618F05DFABDF800303B800124ABE77A
:107AE0000446A9E7E871030814720308AC3A0020C1
:107AF000BC3A002016720308B03A0020BE3A0020BB
:107B000010B50446FFF778FF28B921460248BDE8C2
:107B1000104008F007BE10BD407203082DE9F04385
:107B20004FF000089DB005460E461746A2F80080AB
:107B3000002E35DDB2B200239CB2A24203F101094E
:107B400002D9EB5C0A2B29D1632C28BF632422467F
:107B5000294603A81AF0BCFF1CAB1C44A6EB09067F
:107B600004F8648C9DF90C30232B4D44E0D0002B9D
:107B7000DED00DF1020302AA01A903A8FFF748FE17
:107B80000028D5D0019800220DF10301FFF734F948
:107B90000028CDD03B8801333B80C9E74B46CBE77B
:107BA00001201DB0BDE8F0832DE9F04FDFF82881FA
:107BB0000546D8F800009FB00E4608B1FCF7DAFE83
:107BC000434FDFF818A1DFF8189100240DF10A02E5
:107BD00031462846C8F800403C80AAF80040A9F881
:107BE0000040ADF80A40FFF799FF00286DD0BDF8BE
:107BF0000A300C205843FCF7B7FEC8F8000010B953
:107C0000344809F0D9FABDF80A303B80A346BDF8E4
:107C10000A30A34257D9002E55DDB1B2002297B2E7
:107C2000B94202F1010302D9AA5C0A2A49D1632FA1
:107C300028BF63273A46294605A801931AF048FF52
:107C40001EAB1F44019B07F864BCF61A1D449DF946
:107C50001430232BDBD0002BD9D002AB04AA03A90C
:107C600005A8FFF7D5FD0028D1D0039800220DF11B
:107C70000901FFF7C1F807460028C8D00C2303FB11
:107C800004F2D8F800309850D8F800301344049A21
:107C90005A609DF808201A7222B1B9F800300133F9
:107CA000A9F8003001343846A4B2FFF7E7F90028FC
:107CB000ADD19DF809109DED040A3846FFF72AFD65
:107CC000A5E71A46ABE7AAF800301FB0BDE8F08F71
:107CD000BE3A002016720308B03A0020BC3A0020D9
:107CE000AC3A002002460248418A1430FFF75CBFDC
:107CF0007C72030810B50A4B1B680446D86A0368F7
:107D00005B69984710B12146FFF7FAFE054B5B8A85
:107D100023B12046BDE81040FFF7E4BF10BD00BF0F
:107D2000302600207C72030830B5002085B0FFF7B4
:107D3000E1FF214B1A7872B901221A701F4B204AB9
:107D40001B680292986A1F4A0368039204AA12E908
:107D500006009B6A98471C4D04246B88A34229D9CE
:107D6000042322466946284600F0F2FB6846FEF7E7
:107D7000A9FE18B1154B1C8005B030BD009801A9B3
:107D8000FEF73CFC60B19DF8010000F01F00FEF71B
:107D9000BDFD221D0346019992B2284600F0D8FB92
:107DA0009DF8010000F01F00FEF7B0FD0430044410
:107DB000A4B2D2E70020DFE7C13A0020302600203D
:107DC0006F3A0020F1820108C23A0020B43A002044
:107DD00070B50E4B1E880E4B1B68002294B2A64253
:107DE00009D91C4601322568854203F10C03F5D1FF
:107DF00094ED010A70BD8B891B0649BF8B6891ED1C
:107E0000020AC01A90ED000AF4E700BFBC3A002055
:107E1000B03A00202DE9F04105460F464FF000082A
:107E20005FFA88F307EB0311CC7BDCB1042C0BD891
:107E30004E682E443046FFF7CBFF31462046FFF711
:107E4000B7F908F10108EBE7052CFAD14C682C448E
:107E50002046FFF7BDFF84ED000A84ED010A84EDA2
:107E6000020AEEE7BDE8F08170B50E4B1E880E4B9E
:107E70001B68002294B2A64209D91C46013225682B
:107E8000854203F10C03F5D194ED010A70BD8B8995
:107E90001B0649BF8B6891ED020AC01A90ED000ADB
:107EA000F4E700BFBC3A0020B03A00202DE9F041D1
:107EB0008AB00023CDE90733039309930DF1090339
:107EC000009304AA07AB03A90446FEF777FC054616
:107ED00020B9002630460AB0BDE8F081049B002B93
:107EE0003AD0DB7BEA898DF8142003F01F03C2F33C
:107EF00000221B0243EA4233039A43EA82339DF88D
:107F000014200DF10A01134305A80593FEF7F2FDB5
:107F1000064658BB06A92846FEF7D2FA0028D9D053
:107F20009DF815700499DDF8188007F01F07B9B1A6
:107F30009DF81C3093B1089A012B556802D0099B1B
:107F40005B681D442046FFF743FF496841442944CC
:107F50003846FFF72DF9BDE7037CC3E73546F1E767
:107F600029462046FFF780FF4146F1E79DF81500BE
:107F70009DF8093000F01F02052A0FD0002BA8D170
:107F800000F01F00FEF7C2FCBDF80A2004320346D1
:107F900092B22146044800F0DBFA9BE7002BEFD0B9
:107FA000A4EB8304ECE700BFC23A00202DE9F043C4
:107FB00085B0FEF767FA134E134F00254FF01408F3
:107FC0003288ABB29A4219D91C463B6808FB04348C
:107FD00094F81090B9F1040F0ED803A92046FEF7CB
:107FE0006FFA48B1039801902146FFF73DFF0198D1
:107FF00001464846FFF7DCF80135E1E705B0BDE88A
:10800000F08300BFC63A0020C83A00202DE9F347AC
:10801000DFF88C901F4940F678226846FCF732FE64
:10802000B9F800702FB11C4B1A881C4B1B889A4260
:1080300028D0194E194D05244FF00008B9F80070EA
:108040001FB132882B889A421CD0013C14F0FF04E7
:1080500018D00022114601A83788CDF80480FFF718
:10806000C3F84FF0000A1FFA8AF30AF1010A28B197
:108070000022114601A8FFF731FAF4E7A9F8003011
:108080002F80DBE76846FCF71FFE384602B0BDE8EC
:10809000F08700BF703A0020AA3A0020BA3A0020C8
:1080A000B63A0020024A138801331380704700BF9C
:1080B000AA3A00202DE9F0412DED028B90B000236B
:1080C000CDE9083305930A930DF1110300930E4691
:1080D00008AB06AA05A90446FEF770FB0546D8B111
:1080E0000699F1B1CA7BEB898DF81C3002F01F02B2
:1080F000C3F300201302059A9DF8117043EA403340
:1081000043EA82339DF81C201A43C3F30423052B52
:10811000079200F0868037B110B0BDEC028BBDE84D
:10812000F081027CDFE7012B05D121B18B895B0750
:1081300001D5FFF7B7FF274677E0BDF812204FF6CD
:10814000FF739A420AD14C4B83F800804B4B4C4949
:108150001B68986903681B689847DDE79DF81D1048
:1081600001F01F01042925D99DF81D00BDF812203A
:10817000444900F01F00FEF7C9FB49881318083373
:108180008B424AD20432104480B2FEF707F99DF8C0
:108190001D0000F01F00FEF7B9FBBDF812100431FE
:1081A000024689B23846FEF7F1F8BDF812100422F3
:1081B00007A85EE02046FFF7B9F90699F0EE408A7D
:1081C00071B12046FFF704FEB0EE408AF0EE400A9F
:1081D000B0EE680AFDF708FD38B1002EC4D19BE768
:1081E00029462046FFF740FEEEE7002EBCD19DF861
:1081F0001D3003F01F03032BB6D09FED230A38EE8A
:10820000C88AF0EEE88A68EE808AB0EEC88AB4EEDA
:10821000E88AF1EE10FAA7D57EE7174B01221A7013
:1082200094E7002F87D0A4EB870711234FF00108B4
:10823000CDE902380BAB01939DF81130009329462C
:108240002046069A08ABFEF7BBFC0DF1120107A809
:10825000FEF750FC00283FF470AF9DF81D0000F0C1
:108260001F00FEF753FBBDF812100431024689B21D
:108270003846FEF78BF84FE7A83A0020302600205A
:1082800064720308C23A002017B7D1387FB5164D83
:108290002E1D40F27F12314601A8FCF7F3FC28683E
:1082A000FCF74CFF042812D92868052202A9FDF723
:1082B00057F8431F5C425C4101A8FCF705FD44B13F
:1082C0009DF80C1002980122FFF7F4FEE1E700246C
:1082D000F2E7064B1B68986A03685B6B984708B126
:1082E000FFF794FE04B070BD8C3A002030260020C9
:1082F000FFF7CCBF10B50446FCF738FB204610BD95
:1083000038B51148114D08F097F9114A11490E4836
:1083100018F022FC2846002340F8043B08F08CF9B2
:108320001420FCF71BFB044610B19B21FCF7A4FEB4
:108330000949074A05482C6018F00EFCBDE8384092
:108340000648002100F0EEB8703A00208C3A002078
:10835000346900207163010875630108C23A002086
:1083600091ED007AD0ED007ADFED086A80ED007AB9
:1083700077EEC77AF0EEE77AF4EEE67AF1EE10FAED
:108380004CBF01210021FEF7DFBD00BF000000341B
:10839000D1ED007A90ED007AF4EE477AF1EE10FA22
:1083A00004D0C0ED007A0121FEF7CEBD7047000079
:1083B00090ED000A7047000038B504460D46FEF700
:1083C000C5FE10B995F90030237038BD91F9003021
:1083D0000370704791F9002090F90010914202D08B
:1083E0000270FEF78FBD704791F9001090F90030D0
:1083F0009FED097A01705B1A07EE903AF8EEE77A82
:10840000F0EEE77AF4EEC77AF1EE10FA4CBF0121F4
:108410000021FEF799BD00BF0000003491F9002053
:1084200090F90010914203D002700121FEF78CBD3B
:108430007047000090F9003000EE103AB8EEC00A24
:108440007047000038B504460D46FEF77FFE10B9B0
:10845000B5F90030238038BDB1F90010B0F9003013
:108460009FED097A01805B1A07EE903AF8EEE77A01
:10847000F0EEE77AF4EEC77AF1EE10FA4CBF012184
:108480000021FEF761BD00BF00000034B1F90020FB
:10849000B0F90010914203D002800121FEF754BDD3
:1084A00070470000B0F9003000EE103AB8EEC00A94
:1084B0007047000038B504460D46FEF747FE08B980
:1084C0002B68236038BD00000B6803607047000014
:1084D0000A6801688A4202D00260FEF713BD704745
:1084E0000A6801688A4203D002600121FEF72CBDB0
:1084F0007047000090ED000AB8EEC00A7047000017
:1085000008B5064B1B68586903685B68984720B933
:10851000BDE80840024808F005B908BD3026002033
:108520009073030830B50023084A01704380147823
:108530008C4204BF4488958803F1030304BF641987
:1085400044801E2B02F10602F1D130BDB073030846
:108550002DE9F84F184EDFF8649007468A461D460D
:1085600006F13C0831783B78994204D1B4889442B2
:1085700009D8121B92B20636B045F3D1B5FA85F090
:108580004009BDE8F88F12FA85F3A342D9F800300C
:1085900058697388C8BFA41A1A440368D4BFACB220
:1085A000A4B2D3F808B092B223465146D8472D1B47
:1085B000E4D0A2440022DEE7B07303083026002096
:1085C0002DE9F84F184EDFF86490074692461D4695
:1085D00006F13C0832783B789A4204D1B4888C4248
:1085E00009D8091B89B20636B045F3D1B5FA85F032
:1085F0004009BDE8F88F11FA85F3A342D9F800309D
:1086000058697388C8BF641A19440368D4BFACB2F0
:10861000A4B2D3F80CB05246234689B2D8472D1BDA
:10862000E4D0A2440021DEE7B07303083026002026
:1086300010B5044601F032FA4FF0FF33E36204F163
:10864000300007F0F9FF04F1640008F093FE002306
:10865000C4F88C30C4F89030C4F8943006492046F1
:10866000FFF7D8FB054B1A6812B1054808F0A4FDC6
:108670001C60204610BD00BF54750308D03A00208E
:10868000EC730308084699B1C81FC3B2102B0ED86B
:1086900010280CD8DFE800F0090B090B0B0B0B09B5
:1086A0000B0B0B0B090B0909090000207047012077
:1086B0007047000007B50DF10601FEF707FC08B38F
:1086C00012490B68DB0718D4114BBDF806201A803D
:1086D0001A821A841A86A3F84020A3F85020A3F81F
:1086E0006020A3F87020A3F88020A3F89020A3F8BE
:1086F000A020A3F8B02001230B60054800220C2124
:10870000FFF704F803B05DF804FB00BFCC3A00208B
:1087100010230020F7B504460DF1070101278DF85D
:108720000770FFF749FE2046FFF7C4FF94F91530A4
:10873000032B15D104F128063046FEF707FD054648
:1087400070B90DF1070130468DF80770FFF74CFE48
:108750000DF1070104F115008DF80750FFF744FEF5
:1087600004F080F9217805462046FFF78BFF30B1F1
:1087700000220521284604F06BF8C4F80C01002300
:10878000E36184F858306388013B9BB2C72B84BFF8
:10879000C823638003B0F0BDB02303FB010191F84F
:1087A000A90010B1D1F8983013607047B02303FBD3
:1087B000010191F8AA0010B1D1F89C301360704704
:1087C000B02303FB010191F8AB0010B1D1F8A03048
:1087D000136070472DE9F843B02303FB010384467F
:1087E000D3F8B8200F4622B9D3E9300150EA01038B
:1087F0002CD0B02606FB07C6B6F8600000283FD094
:10880000D6E930231F4DDFF880901343A0FB0545C8
:108810001ED042375CF8270003F0B4FC074608F08E
:10882000F9FC14EB090245F14904D3194FF47A75A8
:1088300044F10004A3FB053205FB0422D6E93045D0
:10884000001B61EB0501181842EB0101BDE8F8833C
:10885000F06D492310EB090043F10003071945EBC4
:10886000030408F0D5FCD6F8B810401AC0194FF42C
:108870007A7344F10004A0FB030103FB0411E5E754
:108880000146E3E700840C24B0F5F79010B5B0235F
:1088900003FB0103B3F86040ACB1423150F8210052
:1088A00003F070FC094BA4FB0313094C091943F1B5
:1088B00049034FF47A72081843F10003A0FB020148
:1088C00002FB031110BD20462146FBE700840C2467
:1088D000B0F5F79000EBC101C1F82821A1F82C31C7
:1088E0007047000001EB810310F92330022B0BD1FC
:1088F000C38C5B0718D500EBC1000D4BC0F82831C5
:108900002E23A0F82C317047DBB21A2B0CD8012291
:1089100002FA03F3074A1A4032B100231A4600EB69
:10892000C100C0F82821ECE7034A2E23F7E700BF77
:10893000F4750308008C00042475030838B5044658
:10894000F9B9D0F80C01E0B1B4F82C31CBB103681F
:108950009B6A9847D4F80C31B4F82C2119688242EC
:10896000CD68D4F8281128BF02461846A847D4F885
:1089700028310344C4F82831B4F82C31181AA4F86B
:108980002C0138BD2DE9FF4701EB8103044610F9A6
:1089900023500F4600EB8308002940F00481A5F125
:1089A0000903D0F80C610E2B10D8DFE813F010008B
:1089B0000F0000010F000F0010000F000F000F004C
:1089C0000F000F000F000F00100010000EB900255F
:1089D00002E1012380F8203108F01AFCD4F81431A8
:1089E000C31AB3F5966F074625D9D4F81C31002B6E
:1089F0003FD1336830461B6E9847C4F81C01122DD6
:108A000048D0112D4FF0000348D14FF40062D4F844
:108A10001C113046FCF7DEF933680021DB6B304671
:108A2000984794F92430C4F81471002B0BDD002111
:108A30002046FFF757FF94F92430002B03DD002177
:108A40002046FFF77BFF0F2D2AD025F010030A2BBD
:108A500036D14FF4D070FBF781FF0546002800F0B7
:108A6000BB80009604F158034246214601F0A0F86D
:108A7000B2E094F818310133DBB2082B08BF0023B1
:108A800084F8183194F81821554B53F82230C4F863
:108A90001C31B4E74FF400630022B8E71A46B6E78A
:108AA0004FF4CC70FBF75AFF0546002800F0948085
:108AB000009604F158034246214600F0D5FD8BE0B4
:108AC000B4F82C31002B82D1336830465B6998476B
:108AD0005FFA85FAB0F5005F28BF4FF400500AF145
:108AE000FF3987B25FFA89F9002F3FF470AF33681E
:108AF00030469B699847B9F1010FC1B20AD894F882
:108B00001821374B53F8223094F9242052BBB3F587
:108B1000164F30D2E38CAAF1110213F0010F14BFEB
:108B20004FF461334FF4E123012A18D894F8180167
:108B30002B4A52F820209A4211D104F2211001F060
:108B4000D9FF60B1112D4FF4BF600CBF0127022780
:108B5000FBF704FF054600283ED001971BE0781E76
:108B600087B2C1E7B3F5E13FD4D3E28C520702D418
:108B7000B3F5613FCED104F22110039101F0BAFFA9
:108B800003990028C6D04FF4BF60FBF7E7FE054607
:108B900010B300230193009604F158034246214686
:108BA00002F038FB18E00B2D7FF411AF00261423E0
:108BB00003FB0743002283F820214FF4FC70FBF7EE
:108BC000CDFE054640B1B02303FB07430096583362
:108BD0004246214600F03AFB284604B0BDE8F08743
:108BE00004750308F8B504460D46B02608F010FBDE
:108BF00006FB0546002386F859304FF6FF730746FB
:108C0000A6F88630A6F8883029462046FFF7BAFE37
:108C100090B1012286F8592004EB051305F14202B8
:108C2000194644F82200DF644FF47A63A1F850300B
:108C3000BDE8F84003F036BBF8BD00002DE9F74F62
:108C400001EB8103044610F923A0BAF1070F0D468A
:108C50000FB24FEA81090DD0BAF1000F0DD1B0214A
:108C600001FB05044FF6FF7384F859A0A4F8863081
:108C7000A4F8883003B0BDE8F08F90F81231CB40F3
:108C8000DA07F7D48144D9F8083123B903B0BDE835
:108C9000F04FFFF7A7BF90F92430002B01DDFFF75D
:108CA0004DFED9F8080103689B689847019008F0C9
:108CB000AFFA019906464FEA0518002962D1A0448F
:108CC000D8F84C30C31AB3F57A6FD3D94FF0B00B44
:108CD0000BFB05405A46583019F044FF0BFB054288
:108CE0004FF6FF73A2F88630A2F888305FFA8AF355
:108CF0004FF47A61172B82F85850C8F84C60A8F8E6
:108D0000501004D83F4921FA03F3DB070BD4D9F8FC
:108D1000080198BBB02101FB05450023C9F80831C3
:108D200085F8593002E0012382F8593004EB07142A
:108D3000B4F85030F52B61D994F85220B3F5FA6F9E
:108D400002F1010284F8522094D294ED157A07EED4
:108D5000903AB5EEC07AF1EE10FA81BFF8EEE77AFC
:108D6000DFED296A67EEA67ADFED286A8CBFE7EEB1
:108D7000267AF8EE677AC4ED157A7BE703685B68BC
:108D80009847C7E74FF0B00A0AFB054A9AF8C8307F
:108D900053B10023DAE930014FF47A72F8F7ACF8F6
:108DA000002306468AF8C830B02303FB054393F836
:108DB000BC206AB9012283F8BC20D9F808010368F5
:108DC0009B6A9847124903466A1C0620F9F7F2FF8E
:108DD00004EB080304EB0511DA6CB21AA1F8502079
:108DE000B02101FB0545DE6495F85920012A9DD983
:108DF00094F83821002A99D19E6497E7002284F8DC
:108E00005220A2E70042C0000AD7A33C48E17A3FC3
:108E10000874030813B540F21E42044600F1300105
:108E200001A8FBF72FFF00212046FFF707FFD4F82A
:108E3000083113B1012384F8113101A8FBF744FF75
:108E400002B010BD10B40C4611461A463CB9D0F819
:108E5000080120B103685DF8044B5B6918475DF8B1
:108E6000044B704710B590F900300C460BB9002048
:108E700010BDD0F8080118B9002323700120F7E7CE
:108E800003681B6998470028F1D1F5E7174B136079
:108E900010B449BBB0F91030002B0DDD07EE903A4D
:108EA0009FED137AF8EEE77A67EE877AC2ED007AE3
:108EB00001205DF8044B7047D0F8083113B190F8E9
:108EC000591049B990F9000010B900231360EFE779
:108ED000431E58425841ECE71968CC6918461146C0
:108EE00023465DF8044B18470020E2E7CDCCCC3D8B
:108EF0006F12833A90F811318B420BD9142303FB84
:108F00000100B0F90200002804DDC828A8BFC8206D
:108F100080B27047C820704759B990F9283043B9DA
:108F200090F900302BB1D0F8080110B103681B6A2A
:108F3000184700207047000008B5034690F922004A
:108F400040B1D3F8080128B103685B6A984780F004
:108F50000100C0B208BD000031B9D0F8080118B155
:108F6000036811469B6B184700207047B02301FB34
:108F7000030191F8B40010B1D1F8B030136070471C
:108F800041B990F90000122806D0A0F11703584209
:108F900058417047002070470120704770B50D465A
:108FA00090F918107F29044613460ED02A46C9B2FC
:108FB000BDE87040FFF746BFD4F8080150B1036820
:108FC00029465B69BDE8704018470021FFF7D8FFCC
:108FD0000028F1D070BD000011F0010F2DE9F84F0D
:108FE0000446884691461E4605D11A464946BDE8C4
:108FF000F84FFFF7D3BFD0F83031002B4BD0D4F867
:1090000030A1C8F34105B4279AF8003007FB05A743
:109010004FEAD8080637002B48D1D4F8303183F80E
:109020000180D4F83011012303FA05F20B781343C1
:109030000B7032464946384619F04AFDB32ED4F833
:10904000303153D86A1C9A7005EB4505D4F830319D
:10905000C5EB051506EB85059D80D4F83051AA783F
:1090600012B3012328789340013B98421CD1F7F7B3
:109070005BFFB4F834311844A4F83401AA88A91D60
:109080002046FFF78BFFD4F8302100239370D4F8EB
:109090003021137008E040F2D621012016F074FF51
:1090A000C4F830010028AAD1BDE8F88F9AF8012051
:1090B000424509D1EB40DB07AFD532464946384639
:1090C00019F0F6FC0028EFD04FF0000B8AF802B040
:1090D000D4F830A19AF80000F7F726FFB4F836313B
:1090E0001844A4F836018AF800B096E71A780F2AD7
:1090F000B3D104229A70D4F830314FF434729A808C
:10910000ABE700002DE9F743984690F83931DDF8D8
:10911000289004460E4673BBB02505FB010595F863
:10912000AC7017B3EB6F1360D5F88030C9F800301E
:1091300001AAFFF7ABFE70B1DDED017A9FED0F7A6A
:10914000D9F8003067EE877AFCEEE77A17EE902ABE
:109150009B1AC9F80030B02101FB064494F8AD30E9
:109160003BB1D4F8A430C8F80030384603B0BDE8AD
:10917000F083034BF7E70027F7E700BF00007A44CE
:10918000000020410120704770470000014B0B6038
:1091900001207047CDCC4C3E012070470120704724
:1091A0000120704700207047704700000020704782
:1091B0007047000006207047004870472476030877
:1091C0007047000010B50446FBF7D0FB204610BDE9
:1091D00070B586B001AD04460E4612220021284625
:1091E00019F0C0FC0221032264238DF804108DF8CD
:1091F00006308DF80B200D238DF80F108DF81620FA
:10920000042194F8DC218DF807308DF8101001232B
:1092100007218DF81210D1188DF808208DF80D3027
:109220008DF8116084F8DC110022E95C01330A44F6
:10923000122BD2B2F9D160688DF815200368132281
:10924000DB682946984706B070BD0000F0B589B0CC
:1092500004460E9D009502F077FF314A2260626855
:109260000023C4F8D03004F5F475C4F8E831C4F82C
:10927000EC31C4F8F03142B9E3682A491A78032086
:10928000F9F798FD204609B0F0BD274E07933068E6
:10929000716802AA03C2CDE905333189118002A8A1
:1092A000012630F8022B462A0CD8510908AF07EBEB
:1092B000810102F01F0251F80C7C06FA02F23A43D7
:1092C00041F80C2C0133052BEBD105AB03CBC4F8D3
:1092D000E80118686960A8602069012305A91230B7
:1092E0008DF81430FFF768F8226992F91230927CF9
:1092F000012A0ED8A26892F92420002A03DD19461B
:109300002046FFF765FF07F083FF6E30C4F8E001E9
:10931000B8E7E268054912780320F9F74BFDB1E799
:10932000887603082C760308386C0308497603080E
:109330002DE9F04186B005460E46904600211422E4
:1093400068461F4619F00EFC02238DF80030642396
:109350008DF802300F2307228DF8033003238DF898
:1093600007308DF80B208DF81430062295F8DC318B
:109370008DF80C2001240A228DF80D201A1985F889
:10938000DC218DF804308DF809408DF80E808DF8C1
:109390000F708DF81160234600221DF80310013371
:1093A0000A44142BD2B2F8D168688DF813200368F0
:1093B0001522DB686946984706B0BDE8F0810000D9
:1093C00070B5044607F024FF0646D4F8E801F7F725
:1093D000ABFD0546D4F8EC01F7F7A6FD0544D4F83B
:1093E000F001F7F7A1FDADB294F8E4310544ADB258
:1093F000AB422EDA236993F912209B7C012B2DD8E6
:10940000D4F8E031B34224D2B4F8E6310125462B3A
:109410000CD8580904EB800003F01F01D0F8E801D4
:1094200005FA01F1014216D0A4F8E631012394F8BF
:10943000E6112046FFF77CFF94F8E431013384F80D
:10944000E431B4F8E6316E360133C4F8E061A4F8D3
:10945000E631012003E001339BB2D8E7002070BD64
:1094600038B5C368426E5A60C368B0F868201A8184
:10947000C368B0F86A2083F8322090F86C3013F09B
:10948000010F0446C36800F0978003225A7090F8D9
:109490006D30D8070CD5E36804225A7094F86D201B
:1094A000910705D55207E3684CBF062205225A7082
:1094B000D4F86F00D4F87310E56844A3D3E900230F
:1094C000F7F774F843A3D3E90023F7F76FF8F7F73A
:1094D0001DFB6861D4F87700D4F87B10E5683BA3E6
:1094E000D3E90023F7F762F83AA3D3E90023F7F7AB
:1094F0005DF8F7F70BFBA861314BD4F87F00D4F887
:109500008310E5680022F7F751F8F7F7FFFA2861B2
:10951000E56807F07DFE286694F88730DB071CD5E8
:10952000E368D4F88820DA61DFED267A94ED230A27
:10953000E56820EE270AFCF767FB204685ED080A60
:1095400002F034FED4ED247AE368F1EE677AC3EDDD
:109550000F7AE368012283F8502094ED277ADFED3B
:109560001A6AE36827EE267ABCEEC77A17EE102A4D
:10957000DA85D4ED287AE36867EEA67AFCEEE77A1E
:1095800017EE902A1A8694ED2C7AD4ED2B7AE368A4
:1095900077EE877AB6EE007A67EE877AC3ED117AB6
:1095A000E368D4F8B8209A64E268012382F8523064
:1095B000E26882F8533038BD012278E7AFF30080CB
:1095C00000005940E02E65420000C842F8C1631A0D
:1095D000DCA54C4000000000D0126341F0B5836868
:1095E00093F92430002B85B0054628DC002605F1D0
:1095F0006407686803685B69984720B36868036814
:109600009B69984701AAC1B23846CDE90166039625
:1096100002F0F8FF01280446EBD1019B03F006029B
:10962000062AE6D103F44072B2F5407FE1D1DB04B3
:10963000DFD52846FFF714FF204605B0F0BDFFF741
:10964000BFFE0028D2D10020F7E7000006207047B7
:1096500000487047C87603087047000010B50446FC
:10966000FBF784F9204610BD37B5069D00950446EA
:1096700002F06AFD114B23600023C4E91B3384F818
:10968000683084F87430AA2384F8793141F2442395
:10969000A4F87A31A36893F924305BB16068084973
:1096A00003680E22DB689847606806490368222237
:1096B000DB689847204603B030BD00BF64770308DD
:1096C000D0760308DF76030870B5B0F8812190F8F2
:1096D0007C31B0F87D51D0F889111A44044602F06B
:1096E000F1FD632D00F0BC80AE2D00F0E5802A2D49
:1096F00040F09F80E368B4F887211A81E368D4F8CA
:1097000089215A60E56807F083FD2866D4F87D005A
:10971000D4F88110E66879A3D3E90023F6F746FF71
:10972000F7F7F4F97061D4F88500D4F88910E66889
:1097300072A3D3E90023F6F739FFF7F7E7F9B06131
:10974000E368012683F85C60D4F89530E26807EEA0
:10975000903AF1EE677AC2ED167A654BD4F88D0037
:10976000D4F891100022F6F721FFF7F7CFF9E1685E
:109770000246204602F030FEE36894F8B62083F8F3
:109780003220D4F89D3007EE103AD4F8A13007EE1D
:10979000903A67EEA77AE368E7EE077AB1EEE77AE8
:1097A00083ED117AE368D4F8A5209A64E3689FED0D
:1097B000517A83F85260E36883F85360D4F8AD209F
:1097C000E36807EE902A67EE877AFCEEE77AC3ED4E
:1097D000207AE36894F8B62083F88420D4F87530B2
:1097E000E268DBBBD4F87930222B0FD81F2B33D89B
:1097F000102B16D00F2B07D9122B03D8102B03D008
:1098000004230FE0142BFBD001230BE0322B02D0FA
:1098100003D8302BF8D1062304E0443B012BEFD9C9
:10982000F2E70323537094F8623043F0010384F8A5
:10983000623094F8623013F001000CD09A07C3F341
:10984000400008D5E268616E526891424ED123F023
:10985000030384F8623070BD0523E3E75670E2E746
:10986000D4F88910D4F88500E668F7F797F9F06125
:10987000D4F89110D4F88D00E668F7F78FF93062CC
:10988000204602F093FCD4F89500D4F89910E668CD
:10989000F7F784F907EE900AF1EE677AC6ED0F7AD2
:1098A000E368012283F85020D4F88931636694F884
:1098B000623043F00203BAE7D4F87D20DFED0E6A90
:1098C000E36807EE102A27EE267ABCEEC77A17EE79
:1098D000102ADA85D4F88120E36807EE902A67EE33
:1098E000A67AFCEEE77A17EE902A1A860020B2E7F5
:1098F0000000594000007A440000C8420000000007
:10990000D012634110B590F87430013B0446082B27
:1099100006D8DFE803F010191D26374C50586000B8
:10992000AA2904BF012380F87430002380F8953100
:1099300084F8963104E0442904D1022384F8743079
:10994000002010BD0023F9E71229FBD10323F5E71E
:10995000042380F8743080F8953180F87C1100235E
:10996000E6E7B0F895311B2BECD8C218013382F82A
:1099700079119AB2A0F8953190F87C319342DFD8F2
:109980000523DBE7B0F89531FF2BDBD890F87C019D
:109990001A1A2244013382F875109AB2A4F895314C
:1099A000B4F8813103449A42CADB0623C6E7C0F803
:1099B00075110723C2E7D0F8753103EB0121C0F818
:1099C00075110823BAE7D0F8753103EB0141C0F8EF
:1099D00075110923B2E7D0F8753103EB0161C0F8C6
:1099E0007511002094F87C2184F8740004F2791138
:1099F00007F022FFB4F8812104F1750107F01CFF84
:109A0000D4F87531834204D12046BDE81040FFF7F9
:109A10005BBE236F0133236792E700007FB5836845
:109A200093F924300446F3B107F0F2FB94F8683060
:109A3000032B054617D8E26E824214D2164A666896
:109A400052F8231001910846F7F7D6FC33680199C4
:109A5000DB6802463046984794F86830C8350133D1
:109A6000E56684F868304FF40056002560680368A6
:109A70000DF10F01DB69984750B19DF80F1020469A
:109A8000FFF740FF013E2843B6B2C5B2002EEDD12C
:109A9000284604B070BD00BF4C77030810B5002302
:109AA000044643608360C3600249FEF7B3F9204671
:109AB00010BD00BFA4770308062070470048704718
:109AC00014780308014B0B60012070470AD7A33DAF
:109AD000D0F880300B60012070470000836893F954
:109AE000243023B1806E831F5842584170470120B3
:109AF00070470000D0F8803013F4746F0CBF012061
:109B00000020704710B50446C06E16F041FA20469A
:109B100010BD000010B50446FFF7F4FF2046FAF729
:109B200025FF204610BD00008268C36F92F92220F5
:109B3000022A03F4207304D0A3F52073584258413D
:109B40007047B3F5207F08D0064B1B68DB6A93F89B
:109B50009C3023B990F884007047012070470020A2
:109B6000704700BF302600201FB5836893F924306A
:109B70008BB1836E062B0ED0C26804214FF0030C0C
:109B80001278CDE9011C90F862100091013203496E
:109B90000620F9F70FF905B05DF804FB1878030803
:109BA000C3681B7813B98368187870470020704722
:109BB00037B5069D0095044602F0C6FA0F4B2360A8
:109BC0000F4B63670023A36784F8863007F020FB00
:109BD000E3682067012283F88520A368DB8C9B075C
:109BE00004D42046FFF7DCFF1A2803D1E3680122E2
:109BF00083F82C20204603B030BD00BF447B03080F
:109C00004C7803082DE9F341B0F88C3040F6BC7273
:109C1000C3F30C039342044600F0C8810FD840F60A
:109C2000A77293423BD040F6AE72934200F04B8154
:109C300040F6A172934200F0378100201FE141F20B
:109C40001472934200F0628141F233729342F4D174
:109C5000FFF7A6FF1A28F0D12046B4F88E20D4F8DA
:109C6000901002F02FFB94F89700E36810F08F003B
:109C700040F08181D4F898209FEDC67A07EE902AB3
:109C8000F4EE477AF1EE10FA00F07581B1EEE77A62
:109C9000012283ED137AE36883F85520EFE0B0F8F2
:109CA00094304FF6FF7299B2914205D0C268138189
:109CB000C368D0F890205A60B4F88E20D4F8901081
:109CC000204602F0FFFAE56807F0A2FA2866D4F809
:109CD000B430DFEDB17A07EE103AB4EEE77AF1EE88
:109CE00010FA3BDDE2685363E368D4F8B8209A6366
:109CF000D4F8BC30E26807EE903AF1EE677AC2ED34
:109D00000F7AE368012583F85050E168204602F09D
:109D100079FAB4F8D630E268DFEDA06A0A214B4345
:109D2000C2F88030B4F8E220E36807EE102AB8EEFB
:109D3000477A27EE267A83ED117AB4F8E420E368B7
:109D400007EE902AF8EE677A67EEA67AC3ED127AEC
:109D5000E36883F85250E36883F85350D4F898606E
:109D6000D4F89C7085A3D3E9002330463946F6F732
:109D7000ADFE00285FD083A3D3E9002330463946E7
:109D8000F6F714FC81A3D3E90023F6F70FFCF6F7EE
:109D9000BDFEE5686861D4F8A000D4F8A410E568B9
:109DA00078A3D3E90023F6F701FC78A3D3E90023D5
:109DB000F6F7FCFBF6F7AAFEA861D4F8B020DFEDB9
:109DC000757AE36807EE102AB4EE677AF1EE10FABE
:109DD0000CBF0122002283F85C20D4F80C80D4F858
:109DE000A86098F85C30D4F8AC7093B1D4F8B05057
:109DF0002846F6F783FB02460B4630463946F6F70F
:109E00001DFA07EE905AF1EE677A06460F46C8ED46
:109E1000167A39463046F6F7C1FEDFED617AE16821
:109E200007EE100A67EE277A2046FDEEE77A17EE76
:109E3000902A02F0D1FA94F8D230E268FF2B82F82F
:109E4000323002BFE368002283F8322094F8963063
:109E500003F00F03082B09D8DFE803F005141714EB
:109E60001A1D171A1D00E36801225A7094F89630E3
:109E700013F0400F4FF0010010D0E368587002B0AB
:109E8000BDE8F081E3680322EFE7E3680422ECE732
:109E9000E3680622E9E7E3680522E6E71A06EED55D
:109EA000E36802225A70EAE7B0F88E20D0F89010EA
:109EB00002F008FAE368B4F89C20DA85E368B4F8A5
:109EC0009E201A86B9E6B0F88E20D0F8901002F0E5
:109ED000F9F9D4F89C30D4F8A010E367D4F88030B6
:109EE00083EA010212F4746F0BD0E268127801F475
:109EF0007461009103F474632A4901320620F8F773
:109F000059FFD4F8A030C4F8803096E6B0F88E201F
:109F1000D0F8901002F0D6F9D4F8983007EE103A45
:109F2000D4F89C3006EE903AD4F8A03007EE903A80
:109F3000F4EE676AF1EE10FAC8BFF0EE667AB4EE9E
:109F4000677AF1EE10FAC8BFF0EE477A9FED167A05
:109F5000E368F4EEC77AF1EE10FA08DBB1EEE77AC7
:109F6000012283F85120E36883ED107A65E6002032
:109F700083F8510083E70022DA645EE60000000007
:109F8000006A08C1F8C1631ADCA54C40000000005B
:109F9000D0126341FFE65BAF005043C80AD7A33B32
:109FA0000000C8425C78030800000034B0F88E203E
:109FB000D0F8901002F086F994F89600E36870B932
:109FC00083F88400E368C3F88000E368C3F88C007A
:109FD000E368C3F88800E368C3F890004FE794F89B
:109FE000982083F88420B4F8C5304FF6FF7293426E
:109FF0001CBF0A225343E26808BF0023C2F8803026
:10A00000D4F89C60D4F8A07031A3D3E90023304683
:10A010003946F6F733FD002841D12DA3D3E90023BB
:10A02000D4F8A400D4F8A810F6F728FDB8BB28A3EC
:10A03000D3E90023D4F8AC00D4F8B010F6F71EFD35
:10A0400068BBB4F8C0204FF6FF739A4227D01F4B6D
:10A05000D4F80C80002230463946F6F7A7FAF6F716
:10A0600055FDC8F88C00D4F8A400D4F8A810174BFC
:10A07000E6680022F6F79AFAF6F748FDC6F8880077
:10A0800010A3D3E90023D4F8AC00D4F8B010E668EC
:10A09000F6F78CFAF6F73AFDC6F89000CDE5A3681E
:10A0A000DB8C9B077FF5C9ADE3680020C3F88C000B
:10A0B000E368C3F88800E368C3F89000E36883F8B6
:10A0C0005400DCE60000000000408FC000408F40DC
:10A0D000BBBDD7D9DF7CEBBD2DE9F84F90F88630BA
:10A0E000013B04460D46082B06D8DFE803F0404B41
:10A0F0004F575B63677FB400242908D1012380F8A0
:10A1000086300023A0F890310020BDE8F88F90F849
:10A110009731DFF800925E1CF6B203444FB2032E73
:10A1200080F89761B24683F892714FF00608A8BF95
:10A130004FF0030A00F5C97B59F8040B5246594603
:10A1400019F0D4F978B9042E06D1303F092FDBD9A4
:10A15000002384F89731D7E7D6D93E2DF8D10123D3
:10A1600084F89831F4E7B8F10108E5D1F0E7402927
:10A1700003D1022384F88630C6E7522940F09D803F
:10A180000923F7E7A0F88A100323F3E7B0F88A1051
:10A1900001EB0525A0F88A500423EBE7A0F88C100A
:10A1A0000523E7E7B0F88C1001EB0525A0F88C50EB
:10A1B0000623DFE7A0F88E100723DBE7B0F88E1048
:10A1C00001EB0525ADB2AB07A0F88E50A5F108054F
:10A1D0000CBF08230023F82D80F8863094D9002383
:10A1E00080F88630A36F0133A3678DE7B0F8903114
:10A1F000FF2B98BFC21803F1010398BF82F890109B
:10A20000B0F88E209BB2083A9342A0F89031FFF646
:10A210007BAFB3F5807F50D8002202218C3007F04D
:10A2200033FB0221024604F18E0007F02DFBB4F847
:10A230008E100246083904F1900007F025FB002338
:10A2400084F88630B4F88A308342CBD12046BDE80A
:10A25000F84FFFF7D7BCB0F89021FE2A2DD883180D
:10A26000013292B20A2983F89010A0F890217FF46D
:10A270004BAF8318002183F8901090F890303A2B60
:10A280001BD1C66ECEB100F19201053A304619F0ED
:10A290002DF9054688B9304615F07AFEA36EE566BD
:10A2A000062B07D8DFE803F0040B0F1D2B0D2D0044
:10A2B0000123A36606F0ACFF206700235AE70523BD
:10A2C000F7E70223F5E794F862300133DBB2032BA2
:10A2D00084F86230EED90323A366002384F8623049
:10A2E000E8E794F86230A2680133DBB284F86230A8
:10A2F00092F920200AB1022BDCD90423D9E70623E6
:10A30000D7E703F0F7FD4FF4CE724FF4801103F05E
:10A31000DDFDCFE7147B0308406802490368112282
:10A32000DB6818478878030838B5836893F92230CA
:10A33000054653B3C06F10F4007414D1EB68144990
:10A340001A7806200132F8F735FDEB6811491A78C2
:10A3500006200132F8F72EFD2846FFF7DDFF85F8CD
:10A360008440002038BDC30507D5EB680A491A7838
:10A3700001320620F8F71EFDF3E710F0800404D147
:10A38000EB6806491A780132F3E70120EAE700BFDB
:10A390009C780308BC780308DD780308F678030886
:10A3A00010B5044605490720F8F704FD6068044924
:10A3B0000368BDE81040DB68132218471C790308C6
:10A3C000307903082DE9F04304464068036887B0FC
:10A3D0005B699847002506462F46B5420BD060685A
:10A3E00003689B699847C1B22046FFF775FE074393
:10A3F000FFB20135F1E706F00BFFA36893F92420C3
:10A400000546E2B1A26E062A00F0FC80616E814230
:10A4100015D2216F01F5FA61814221D2606FF6F702
:10A42000EBFF0646606803689B6A9847B04206D314
:10A430006068616F03683246DB6898472567E268A9
:10A44000906A2D1AB5F5967F82BF002382F85430AA
:10A45000E268384688BF82F8553007B0BDE8F0831F
:10A4600094F898110029EAD0E16E09BB052A1FD89B
:10A47000DFE802F003349AA0B7452369606893F9D6
:10A480001220036805921B6C98477049704B059A1F
:10A49000012808BF0B4604F16C066E490093304654
:10A4A0004FF4613306F028F9013001D10023E3664F
:10A4B000E06E0028C3D0F6F79FFF06466068036889
:10A4C0009B6A9847B042BAD36068E16E036832462F
:10A4D000DB689847002384F89831B0E72046FFF7FF
:10A4E0005FFB5D4B5D4A5E491A2818BF1A46236917
:10A4F00004F16C0093F9123000920122D2E7236933
:10A50000597893F9016011F06F0FD1D0524B554A31
:10A5100016F0010F08BF1A4616F0020F04F16C0086
:10A5200006D0DFF870C1504B11F0010F08BF634631
:10A5300016F0040F2DD0DFF860E1DFF860C111F0F4
:10A54000030F08BFF44616F0080F25D0DFF850813E
:10A55000DFF850E111F0070F08BFC64616F0200FD4
:10A560001DD0DFF84491DFF8448111F00F0F18BFC0
:10A57000C846760616D53D4E11F02F0F3C4918BF40
:10A580003146CDE90281CDE900CE3A4906F0B4F872
:10A590008AE7DFF8C4C0D6E7DFF8BCE0DEE7DFF823
:10A5A000B880E6E72C49ECE794F86220324B53F888
:10A5B000222009E093F92030012B0BD0022B0DD083
:10A5C000002B7FF475AF2D4A2D4904F16C0006F085
:10A5D00093F869E794F862202A4BE8E70623A3661C
:10A5E00066E72046FFF7DCFA1949274A1A2818BF00
:10A5F0000A46264904F16C0006F07EF800287FF434
:10A6000055AF55E793F92230022B7FF418AF204B5A
:10A610001B68DB6A93F89C301BB1012384F88430FB
:10A620000DE794F88430002B3FF409AFE36F9B05EE
:10A630007FF505AF636E8342BFF401AF2046FFF79D
:10A64000AFFE05F57A736366F9E600BF4979030842
:10A65000447903089B790308AE7103085179030814
:10A66000BE7903083A6F0308557A03088579030811
:10A6700086790308197A03082C7B03082C7A0308CF
:10A680003C7A0308087B03088E790308377A0308AD
:10A6900030260020567A03086F7903086E79030884
:10A6A00078790308777903087F79030880790308AC
:10A6B00006207047836893F924302BB1D0F8BC058D
:10A6C000B0FA80F04009704701207047D0F8BC35DF
:10A6D0000B6001207047000000487047847B03082E
:10A6E00090F8C035822B08D81A0611D4033B012BF1
:10A6F0000ED9084B0B6001207047FF2BF9D1054B99
:10A700000B60836893F92400B0FA80F04009704729
:10A71000014BEFE7AE47613E8FC2F53D0020704729
:10A72000704700000120704710B5054B03600446D8
:10A73000D0F8F40508B1FAF719F9204610BD00BFAA
:10A740007C7E030810B50446FFF7EEFF2046FAF7BB
:10A750000DF9204610BD000013B5D0F8BC1500233C
:10A76000012202FA03F40C420CD0C2681278009164
:10A770000649013251F8233005490620F8F71AFB43
:10A7800002B010BD0133162BEBD1F9E7C47D0308ED
:10A790008C7B0308C1F302710139C9B204299ABF45
:10A7A000014B585C00207047BC7D030830B5D0F8E1
:10A7B000DC357BB190F8E0550020C2B2954209D952
:10A7C00053F830208A4200F1010401D140B230BD7B
:10A7D0002046F2E74FF0FF30F9E7000030B5039C68
:10A7E0000A44914209D011F8015B18782844C0B29C
:10A7F0001870257828442070F3E730BD2DE9F0412A
:10A80000044640681D46036886B09B6ABDF8306008
:10A8100088461746984706F1080398424FF0000013
:10A820003AD3B5238DF810308DF8137062230DF1F3
:10A830000F078DF80E008DF80F008DF811300422EF
:10A840000DF10E030DF11201204600978DF81280D4
:10A85000ADF81460FFF7C2FF324629462046009744
:10A86000FFF7BCFF606803680622DB6804A998470D
:10A87000606803683246DB68294698476068036869
:10A880000122DB680DF10E01984760680368012220
:10A89000DB6839469847012006B0BDE8F08100002A
:10A8A00013B50446406803689B6A9847072806D991
:10A8B000002300931A4606212046FFF79FFF02B0AF
:10A8C00010BD00001FB590F89734052B05D9FFF790
:10A8D000E7FF002005B05DF804FB02238DF80C10A3
:10A8E0008DF80D200093012203AB0621FFF786FFB0
:10A8F000F0E70000F0B5044640681D46036885B0E7
:10A900009B6A0F46164698470A280FD903230093DF
:10A91000012203AB062120468DF80C708DF80D60E6
:10A920008DF80E50FFF76AFF05B0F0BD0020FBE781
:10A9300090F8D2350133DBB280F8D2352BB990F8DC
:10A94000752490F87A14FFF7D5BF7047022938B5FF
:10A950000546184641D00A2939D001291ED1122AAC
:10A960001AD8012A1AD9931E102B17D8DFE803F042
:10A97000171D0916233F1616161616161616161646
:10A9800029000123202483423BD1D5F8BC3523EA9A
:10A990000403C5F8BC3501E0202A2CD038BD95F859
:10A9A000D64584F001030224EDE795F8D64584F0FE
:10A9B00001030424E7E795F8D64584F00103082451
:10A9C000E1E795F8D64584F001031024DBE7092A76
:10A9D00015D00B2AE2D180240FE0102A01D0152ACD
:10A9E000DCD1AB684FF4807493F82230CBE70123BD
:10A9F0004FF40054C7E74FF400440523C3E7402455
:10AA0000FBE72846FFF776FFD5F8BC352343C5F8AA
:10AA1000BC35012385F8D435C0E700002DE9F043AB
:10AA200085B002AFC0F8E83597F8283080F8EC35EB
:10AA300090F8F03580F8E025541C83F001035B4268
:10AA4000A40080F8ED350026E31DC0F8DC15C0F841
:10AA5000E4650546914640686A46DB08A2EBC303FD
:10AA60009D46026802AB926A7B60013C8846A4B2B4
:10AA7000904704F1090292B2904218D37B68029683
:10AA8000414603AA08EBC909494504D051F8080B0F
:10AA900042F8040BF8E70134A4B200948B2206219B
:10AAA0002846FFF7ABFE0C37BD46BDE8F0833046C5
:10AAB000F9E7000013B50C230446009309220B4B61
:10AAC0000621FFF79BFE06F0A3FB94F88834C4F838
:10AAD0008404013384F88834E36805491A78062031
:10AAE000013202B0BDE81040F8F764B9BC7E03083B
:10AAF000B47B030810B5002308248278082A0ED8F6
:10AB0000DFE802F00B051217202B37474D006229B2
:10AB100002D10223837002E08370B52901D00020A6
:10AB200042E083780133F5E703238370C17001713C
:10AB3000F5E704238370C37819440379C9B2C1705F
:10AB40001944F4E705238370C378027901700B443C
:10AB5000DBB2C37013440371E1E706238370C3784B
:10AB600019440379C9B2C1701944002301714370BB
:10AB7000D5E7C378027819440379C9B2C170194482
:10AB8000437801710133DBB29A424370C7D1072386
:10AB9000C0E7C27884708A42C1D08370ADE7027981
:10ABA00083708A42A9D1012010BD000007B500239F
:10ABB000009304220A21FFF721FE03B05DF804FB95
:10ABC0001FB5C368044619788068FEF793F901231E
:10ABD000ADF80A3006210023ADF80800ADF80C30BE
:10ABE000009102AB08222046FFF708FE04B010BD1A
:10ABF000B0F87624083201F065BB00002DE9F74F6C
:10AC00000569D0F8BC35044695F9010038B923F43C
:10AC10000023C4F8BC356B7884F8D7352EE013F4E4
:10AC2000002000F08880D4F8F435FBB128460DF1FF
:10AC3000070110F8017F07F0EF0747F021078DF8B3
:10AC40000770FDF7D1FB4FF0000C604666463122DD
:10AC500010214FF028080CF1FF3527FA0CF3052DD1
:10AC600064D8DFE805F00E2C6E6363A2082115207E
:10AC700015F08AF9C4F8F4050028D7D103B0BDE86F
:10AC8000F08FD4F8F4954FF0200A09EBC00509F8CD
:10AC900030A003F001036E70AA70E9706B6000F1E0
:10ACA000010ED4F8F49502305FFA8EFEC0B209EBC3
:10ACB000CE054FF0050A09F83EA06E7033E0D4F8D7
:10ACC000F4E54FF021090EEBC0050EF8309003F0CB
:10ACD00001036E70AA70E9706B60D4F8F49500F10E
:10ACE000010E5FFA8EFE09EBCE054FF0070A09F858
:10ACF0003EA06E70AA70E9706B6000F1020ED4F88D
:10AD0000F49594F8C1A55FFA8EFE4FEACE050330A4
:10AD1000C0B24D44BAF1000F10D14FF00A0B09F840
:10AD20003EB085F801A0AA70E9706B600CF1010CCF
:10AD3000BCF1070F8FD123695B786DE74FF0090AEB
:10AD4000B9E7D4F8F4E54FF022090EEBC0050EF890
:10AD5000309003F001036E70AA70E9706B60D4F854
:10AD6000F49500F1010E5FFA8EFE09EBCE054FF06F
:10AD70000D0A09F83EA06E70AA70E9706B6000F1D0
:10AD8000020ED4F8F49594F8C1A55FFA8EFE4FEA4E
:10AD9000CE050330C0B24D44BAF1000F02D14FF0DE
:10ADA0000E0BBCE709F83E8087E7D4F8F4E54FF0D6
:10ADB00025090EEBC0050EF8309003F001036E700C
:10ADC000AA70E9706B60D4F8F4A500F101095FFA8C
:10ADD00089F90AEBC90E4FF0180B0AF839B08EF852
:10ADE00001608EF802208EF80310CEF8043094F83B
:10ADF000C195851CEDB2B9F1000F12D1D4F8F4A5BC
:10AE00000AEBC50E03304FF01A0B0AF835B0C0B28A
:10AE10008EF801908EF802208EF80310CEF80430E0
:10AE200084E7284682E7000090F8C00500F0FD00A6
:10AE3000A0F1800358425841704700002DE9F04FBF
:10AE400085B002AF06460C4692469B46FFF7ECFFE4
:10AE500020B900200C37BD46BDE8F08F3046FFF723
:10AE600099FC0023C7E90033804600F10F037068A6
:10AE700023F00703ADEB030D03689B6A98471FFAA5
:10AE800088F505F110039BB298420DF10809E0D353
:10AE900001233B707C6087F801B03C4603CC083549
:10AEA000029003914246514604A8ADB217F010FE3D
:10AEB00000954B468A2206213046FFF79FFCC9E7E2
:10AEC0007FB505460E46FFF7AFFF98B10024CDE9E8
:10AED0000244686803689B6A98470F280CD90823C6
:10AEE00000938B226B4406212846ADF80840039658
:10AEF000FFF784FC04B070BD2046FBE72DE9F04F5E
:10AF000087B002AF81460C4690461D46FFF78CFF86
:10AF100020B900201437BD46BDE8F08F0023C7E9F3
:10AF20000233D9F80400531C6A46DE00A2EBC303C7
:10AF30009D4603689B6A98470836B0420DF1080A9F
:10AF4000E7D301233B727D72BB68029303AE04EB2F
:10AF5000C8084FF0040B444515D02346484653F823
:10AF6000042B7B601146FFF715FC46F8042B7B6829
:10AF700005460246194630462E44043517F0A8FD12
:10AF8000AB440834E7E71FFA8BF2009253468A225B
:10AF900006214846FFF732FCBCE7000013B5836882
:10AFA00093F924300446002B5BD0406803689B6A09
:10AFB00098470D2855D9D4F8BC351A0706D594F80A
:10AFC000D6251AB123F00803C4F8BC3594F896349A
:10AFD0005A1C84F89624192B00F21081DFE813F034
:10AFE0001A0063006B002200690067006D002000FA
:10AFF000280035004A004F0041009D006F0071009D
:10B0000074007600820089004100A700AC00CA00ED
:10B01000ED00F900072201212046FFF753FC12E062
:10B020002022F8E7204602B0BDE81040FFF738BC08
:10B0300094F8C035FF2B14D1002300933022012156
:10B040002046FFF7DBFB60B989E0A36893F9203065
:10B05000022B08D000230093162206212046FFF77A
:10B06000CDFB02B010BDD4F8BC3523F48053C4F836
:10B07000BC35F6E70023009324220621E0E72046B2
:10B08000FFF7D2FE034658B1236994F8D72593F908
:10B0900001309A42E5D0D4F8BC3543F40023E6E70A
:10B0A00000903E22E9E7002300930822E5E7022210
:10B0B000B1E70322AFE70622ADE71222ABE7042295
:10B0C000A9E709220A21A7E70B22FBE7A36893F966
:10B0D000223023B9D4F8BC3523F48073C7E710229B
:10B0E000022199E7A36893F92230002BF2D01522B0
:10B0F000F6E794F898345BB9414B1B68DB6A93F828
:10B100009C302BB9204602B0BDE81040FFF74EBD81
:10B11000D4F8BC3523F40073A9E72046FFF784FE7A
:10B1200000289ED037492046FFF7CAFE8BE7D4F8A7
:10B13000BC3523F480239AE794F8C03503F0FD036F
:10B14000802B8ED12046FFF759FD0246002888D07B
:10B15000D4F8F41503232046FFF7D0FE28B994F85D
:10B160009634013B84F896347BE706F051F8C4F836
:10B17000900476E794F8C03503F0FD03802B7FF44C
:10B1800070AF06F045F8D4F89034C01AB0F5FA7FE5
:10B19000E5D30023C4F890342046FFF72FFD024684
:10B1A00000283FF45EAF0323D4F8F41500934FF466
:10B1B00000232046FFF732FC45E794F8C035822B88
:10B1C0007FF44FAF032300930F494FF480130822FD
:10B1D000EFE794F8F135002B3FF443AFA368DB8C25
:10B1E00013F0200F4FF00303009314BF07490849E1
:10B1F0004FF4001314BF02220122DAE70023B1E763
:10B2000030260020010003201C7E0308647E030812
:10B210005C7E030837B5069D0095044600F094FF58
:10B22000124B23604FF47F43A4F8963441F6FF732A
:10B23000C4F8BC35FF2384F8C0359DF81C3084F871
:10B24000D035E168A068012384F8D33584F8D5357A
:10B2500084F8D835002309781A46FDF73BFB2046D1
:10B26000FFF79CFE204603B030BD00BF7C7E030884
:10B270002DE9F04F2DED028B90F87A14052997B047
:10B28000044640F0A08090F87554012D45D190F807
:10B290006230062B03D00A2B2FD000251BE090F83C
:10B2A0006330242B1DD008D8092B0FD0162BF4D1D6
:10B2B000D4F8BC3523F4805317E0312B18D03E2B43
:10B2C000EBD1D4F8BC3523F400630EE080F87B5456
:10B2D000002580F8D455284617B0BDEC028BBDE898
:10B2E000F08FD0F8BC3523F48063C4F8BC35D4E7C4
:10B2F000D0F8BC3523F48043F7E790F86330092B8E
:10B3000006D00B2BC9D1D0F8BC3523F08003ECE775
:10B31000D0F8BC3523F04003E7E7002DBDD190F80D
:10B320006230062BB9D190F863308A2B34D08B2B46
:10B33000B3D1D0F8DC65002EAFD090F9ED2590F8B0
:10B34000E005571C4FF001030DD184F8ED5584F84A
:10B35000F03594F9ED3583429FDA56F833102046E4
:10B36000FFF7AEFD99E7D4F8E45503FA02F1834004
:10B370002943013B9942C4F8E41501D0824207DB1E
:10B38000D4F8BC35D4F8E81523EA0103C4F8BC3579
:10B39000013284F8ED25DCE7D0F8DC35002B3FF4F2
:10B3A0007CAF90F9EE25C44953F832301A0C1204E0
:10B3B0008A427FF472AFC268C04912780420013219
:10B3C000F7F7F8FC87E706290ED190F87524162ABE
:10B3D00000F05B817FD8012A00F08081082A00F00C
:10B3E0009A81002A00F0928194F87A240A2A40F087
:10B3F000898294F8758408F0FD03092B3FF44DAF62
:10B40000B8F1040F40F08B82012304F2B74684F8B0
:10B41000983404F18001304604F2994718F07AF824
:10B4200004F18A051E2204F16201384618F072F810
:10B430004346A34AF021284617F058FB04F2B158BE
:10B44000002800F02482011D0822404618F062F80E
:10B450009C4BE2689C49CDE9016712780132009269
:10B4600006204246F7F7A6FC98490822304618F015
:10B470003DF8002840F0188295490A22384618F015
:10B4800035F8E8B994F8C0359249802B1EBFD4F83E
:10B49000BC3543F48033C4F8BC35802384F8C03510
:10B4A000D4F8BC3523F4006343F40023C4F8BC355E
:10B4B0004046F5F797FF002840F0EB8184F8C1057E
:10B4C00085490A22384618F011F810B9812384F80A
:10B4D000C0350127E9E13E2A41D08B2A00F03281B4
:10B4E000242A81D100238268A0F8623092F91430B6
:10B4F0005D1C08D090F8641099421EBF80F864303B
:10B500000123A0F8623092F92130B4F8625013F1AF
:10B51000640F1BD094F96E209A4217D045F00205B3
:10B5200084F86E30A4F86250242204F16203009281
:10B5300006212046FFF762F9D4F8BC3543F4806356
:10B54000C4F8BC35012384F8D435A6E6002DEBD130
:10B55000D4F8BC3523F48063C4F8BC35BBE6D0F81E
:10B56000108098F90160002E3FF4ABAEFFF75CFC51
:10B57000054600287FF4A5AE04F1620207AF04F18E
:10B580009A091346BE4610685168BC46ACE80300F1
:10B5900008324A456746F6D11068CCF80000002210
:10B5A000114646FA02F0C00703D5012A1CBF01313B
:10B5B000C9B20132072AF4D14A0094F865600592B5
:10B5C000002722464FF0080ABE423FDD92F866C0CF
:10B5D00098F9010040FA0CF010F001004FEAC701A1
:10B5E0002AD0BCF1010F1DD094F863900598A9F101
:10B5F000030B9BFBF0F094F8C0B5C0B2BBF1040F95
:10B6000082F8670002D8BCF1020F12D082F868906D
:10B610002144D1F86A0040F00100C1F86A00013706
:10B620000832D1E74FF0030082F867C082F8680063
:10B63000EEE782F868A0EBE7214482F8670082F821
:10B640006800D1F86A0020F00100E6E719463C22C4
:10B650007046059317F02CFA059B88B1F600043666
:10B6600000963E2206212046FFF7C8F8D4F8BC35E4
:10B6700043F40063C4F8BC35012384F8D4352AE6CA
:10B68000D4F8BC3523F4006366E7836893F920504F
:10B69000022D3FF40DAE90F86230AB423FF408AE9D
:10B6A000034603F8625F08250095FFF7A7F8D4F872
:10B6B000BC3543F4805343E700003110D47B0308CA
:10B6C000FC7B03087CE30308017C03081D7C030862
:10B6D000267C0308317C0308417C0308B0F87634EB
:10B6E000082B10D190F89734052B02D9FFF7D8F822
:10B6F000D3E5034493F8643094F8632094F862101F
:10B70000FFF724F9C9E590F86430F5E790F8623066
:10B7100080F89734C1E50369B0F86220B3F90230CC
:10B720009A4207D1436E012B04D1D0F8BC3523F0E7
:10B730000103DAE52046FFF743FAD4F8BC3543F0BD
:10B740000103FDE6B0F87634DFF838A4043BDBB241
:10B7500000F16607042B7FF647AEB846043B58F865
:10B76000049BDBB2D145059315D13B79002B72D0F8
:10B770004FF000038DF81C3007AA072351462046DE
:10B78000FFF75CFB012384F8D435D4F8BC3543F4CF
:10B790008033C4F8BC3549462046FFF707F8054614
:10B7A0002046FEF7F7FF002D06464BDBD4F8DC25DC
:10B7B0002BB202EBC303059A824203F1040B0DD3B3
:10B7C000012804D15B683A795340D90706D4324640
:10B7D0004146584617F06CF9002841D094F8EC35F2
:10B7E0005A4649462046FFF729FBD4F8BC35D4F821
:10B7F000E82584F8EE551343C4F8BC350122D4F88B
:10B80000E43584F8D42502FA05F123EA0103C4F8EB
:10B81000E43594F9ED35002B14DB94F8E0158B42F8
:10B8200010DAD4F8DC2552F8330048450AD1013348
:10B830005BB2994284F8ED3504DD52F833102046AE
:10B84000FFF73EFB002E3FF428AD059B9B1BDBB2B0
:10B8500008EB06077EE7D4F8BC3523F4803398E77D
:10B8600094F8E025D4F8E405012303FA05F59340A4
:10B87000013B05439D4204BFD4F8BC35D4F8E8250C
:10B88000C4F8E45504BF9343C4F8BC35C1E7B84BD2
:10B89000DFE5B8494046F5F7A5FD00287FF410AE76
:10B8A000012384F8C1350BE60027B349082230464E
:10B8B00017F01CFE10BB822384F8C035D4F8BC35C9
:10B8C00023F4006343F48013C4F8BC35012384F8E7
:10B8D000F035AA4A0423F021284617F007F900287A
:10B8E0003FF4DBAC012384F8F135A5490620F7F7D6
:10B8F00061FAD4F8BC3543F40013F6E4002F3FF4AA
:10B90000CCACE6E7022A0ED194F87534102B04D1A2
:10B91000A36893F9223013B1BFE4152BF8D0204669
:10B92000FFF706F8B9E4012AF9D194F87524122A30
:10B9300017D8012A1BD9931E102B18D8DFE813F053
:10B940002600AA00CE001700DF002F011700170005
:10B95000170017001700170017001700170017002F
:10B960003702202A00F01882302A00F08B8294F8E7
:10B97000D2550135EDB284F8D255002D7FF48DAC4F
:10B980002B4601212046FEF7B5FFA4E494F8D635F6
:10B9900033B1D4F8BC3543F00203C4F8BC3552E0EF
:10B9A000D4F862109FED788A2046FFF721F9D4F889
:10B9B0006230C4F88034E368D4F866209A61E368A2
:10B9C000D4F86A205A61E368012583F85C50D4F802
:10B9D0006E10D4F87230E2685B1A07EE903AF8EE17
:10B9E000E77A0A2367EE887A2046C2ED167AD4F801
:10B9F0007220E16892FBF3F200F0EEFCE36894F849
:10BA0000D3255A70D4F8762094F8D13507EE102A51
:10BA1000B8EE477A2B4384F8D13527EE087AE368ED
:10BA200083ED117AD4F87A20E36807EE902AF8EED5
:10BA3000677A67EE887AC3ED127AE36883F852502A
:10BA4000E36883F85350E36893F8543063B105F02A
:10BA5000DFFBD4F8CC35C01AB0F5C87F40F23E8287
:10BA6000E368002283F8542094F8D135D9077FF594
:10BA700014AC9A07C3F340057FF50FACD4F87C14DF
:10BA8000D4F8802491427FF408AC23F0030384F8B7
:10BA9000D13520E4D4F862102046FFF7A9F894F8D5
:10BAA000D63523B1D4F8BC3543F0040375E794F8D8
:10BAB0006710E26811F0010F0BD094F86630032B89
:10BAC00005D18A0700D5042384F8D335BBE7022BC0
:10BAD000FAD0012384F8D3355370B4E7002384F8F7
:10BAE000D535D4F862102046FFF782F8E368B4F841
:10BAF0006E20DA85E368B4F86C201A86A3E7D4F8E0
:10BB000062102046FFF774F894F8D635E2681BB14E
:10BB1000B4F86A30138196E794F86D10CB0739D5E5
:10BB200094F86C30032B33D18F0700D5042384F8AD
:10BB3000D33594F8D5351BB1E368B4F88E20DA8597
:10BB4000E36894F8912083F8322094F8D335012BE0
:10BB50007FF679AFE56805F05BFB2866E368D4F80B
:10BB600062205A60E368B4F86A201A816BE700BF6C
:10BB7000AE710308397C03084C7C0308557C03082C
:10BB80005A7C0308010003206F12833AACC52737A3
:10BB9000022BCCD0012384F8D3355370C9E701259B
:10BBA000D4F8621084F8D6552046FFF721F8D4F86F
:10BBB0006230C4F8C435C4F88034E368D4F87A201D
:10BBC0009A61E368D4F87E205A61E3681FED128A17
:10BBD00083F85C50D4F88210D4F88630E2685B1A9F
:10BBE00007EE903AF8EEE77A0A2367EE887A204665
:10BBF000C2ED167AD4F88620E16892FBF3F200F0E9
:10BC0000EBFB94F87630052B00F2C380DFE803F0FD
:10BC1000C1C1039FB8C1E36802225A70E2681FEDF8
:10BC2000250A537884F8D33594F8D13543F00103CD
:10BC300084F8D135D4F88A3007EE903AF8EE677A76
:10BC4000012567EE887AC2ED117AD4F88E20E36878
:10BC500007EE902AF8EE677A67EE887AC3ED127ADB
:10BC6000E36883F85250E36883F85350E36894F82C
:10BC7000792083F83220D4F89E20D4F86230C4F8BA
:10BC80007C3407EE902AF8EEE77AE36867EE887A6C
:10BC9000C3ED077AD4F8A230E66807EE903AF8EEE2
:10BCA000E77A27EE800AF9F7AFFF86ED080AE36826
:10BCB00083F85050D4F89220E36807EE902AF8EE0B
:10BCC000E77A67EE887AC3ED0D7AD4F89620E368B8
:10BCD00007EE902AF8EEE77A67EE887AC3ED0E7ADF
:10BCE000D4F89A20E36807EE902AF8EEE77A67EE38
:10BCF000887AC3ED0F7AE36883F85150D4F8A62010
:10BD0000E36807EE902AF8EE677A27EE888A83EDDB
:10BD1000108A94F8D13543F0020384F8D13594F8B1
:10BD2000D5353BB1E368B4F8AE20DA85E368B4F802
:10BD3000AE201A8694F87630012B03D9E56805F019
:10BD400067FA2866E368D4F862205A607BE6E36805
:10BD500003225A7094F877309E0742BFE3680422AA
:10BD60005A7094F877305D0642BFE36805225A7036
:10BD700094F97730002BBFF651AFE36806224CE709
:10BD800094F8772059490620F7F714F8E36803225E
:10BD900043E7E3685D7041E72046D4F86210FEF7A0
:10BDA00027FF94F86D3098077FF54DAEDAE694F8EA
:10BDB000D63523B1D4F8BC3543F01003EDE5D4F803
:10BDC00062109FED4B8A2046FEF712FFD4F87620D2
:10BDD000D4F86230C4F87C3407EE902AF8EE677A23
:10BDE000E3689FED440A67EE887AC3ED077AD4F8DA
:10BDF0007A30E56807EE903AF8EEE77A27EE800AA7
:10BE0000F9F702FF85ED080AE368012583F8505031
:10BE1000D4F86620E36807EE902AF8EEE77A204629
:10BE200067EE887AC3ED0D7AD4F86A20E36807EEEE
:10BE3000902AF8EEE77A67EE887AC3ED0E7AD4F8A6
:10BE40006E20E36807EE902AF8EEE77A67EE887ACC
:10BE5000C3ED0F7AE16800F0D5F9E36883F851503B
:10BE6000D4F87E20E36807EE902AF8EE677A67EE52
:10BE7000887AC3ED107A94F8D13543F0020384F840
:10BE8000D135E0E5D4F862102046FEF7B1FE94F813
:10BE9000672002F00702022A84F8C02513D8AAB14D
:10BEA000D4F8BC3523F40063C4F8BC35D4F8BC35F1
:10BEB00023F40073C4F8BC3530220023012120464E
:10BEC000FEF718FDBFE5D31E012BEFD90A4B0B4936
:10BED0001B68986903681B689847E7E7D4F8C8258A
:10BEE000D4F8C4359A427FF4D8A9BDE5727C030822
:10BEF0000AD7233CACC5273730260020867C0308B0
:10BF00002DE9F743044605F083F9D4F88C34B4F8EE
:10BF10009424C31A9342054662D32046FFF73EF8A5
:10BF2000D4F8BC35C4F88C547BB3C823A4F894343B
:10BF3000606803685B699847B0F5005F28BF4FF4FD
:10BF40000050002785B2B8460826BBB29D4240F299
:10BF5000DC80606803680DF10701DB699847002801
:10BF600000F0D3809DF80730002019464FEA032CDB
:10BF70004FF0060E94F87424082A3BD8DFE802F04C
:10BF80003F35454F607192AFB6004FF4FA63A4F8A5
:10BF90009434A36893F92330002BC9D094F87B2400
:10BFA000002AC5D194F88824042AC1D8D4F884047E
:10BFB00041F288322D1A9542BAD9564A1268D26A8D
:10BFC00092F89C20002AB3D1012B05D0022BAFD1CF
:10BFD00094F8D435002BABD02046FEF76BFDA7E7D5
:10BFE000D4F8BC35002BA3D1D3E7622B04D10223B4
:10BFF00084F874340137A8E7002284F87424B52B40
:10C00000F8D194F874340133F2E7032284F87424ED
:10C0100084F87A3484F8723484F87334EAE70422BA
:10C0200084F8742494F8722494F8731484F87534A2
:10C030001A44D2B284F872240A4484F87324D9E7EB
:10C04000052284F8742494F87224A4F87614134416
:10C0500094F87324DBB284F87234134484F8733494
:10C06000C8E794F8722494F8739484F874E41A443A
:10C07000D2B284F872244A4484F87324B4F8762443
:10C08000624492B2B2F5826FA4F8762404D9A4F87F
:10C09000760484F874046DE7A4F87804002AA9D122
:10C0A0000723A5E794F8722494F873141A44D2B2C3
:10C0B00084F872240A4484F87324B4F87824B2F51E
:10C0C000826F3CBF121982F86230B4F87834B4F849
:10C0D000762401339BB2A4F878349A4290E794F81E
:10C0E000722484F874649A42D3D183E7002284F8DE
:10C0F000742494F873249A427FF47CAF2046FFF7AF
:10C10000B7F8002818BF804674E7404603B0BDE882
:10C11000F08300BF302600200320704737B5054666
:10C1200040680191144668B103689B6A9847A04231
:10C1300008D9686801990368DB68224603B0BDE846
:10C140003040184703B030BD10B504460C4820609D
:10C150000298C4E90332C4E9010164224FF4FA7180
:10C1600004F1200000F084FCE268002382F85130E2
:10C17000E26882F85230E26882F85330204610BDFF
:10C180000C7F030810B590F8443013B9C3685868A1
:10C1900010BD046D0CB9006CFAE7D0E912014FF440
:10C1A0007A720023F4F7A8FE2044F1E738B52DEDAC
:10C1B000028BC568DFED127A95ED088A28EE278A92
:10C1C0000446B0EE480A14F0CDFCD5ED077A27EE10
:10C1D000800A85ED0D0AE568B0EE480A14F0B2FD5C
:10C1E000D5ED077A27EE800A002285ED0E0AE36876
:10C1F000DA63E368002283F85020BDEC028B38BD7F
:10C2000035FA8E3C10B5D1ED0D0A91ED0E0A0C46B3
:10C2100014F0D2FDDFED077A20EE270AF9F7F4FCDF
:10C2200004F1340084ED080A05F042FB84ED070AAE
:10C2300010BD00BFE02E6542F0B5C468164E2578EB
:10C24000846836680368F66A9B6A4FF0140C0CFB2E
:10C25000054E87B09EF820E1CDE904126F1CBEF1B7
:10C26000000F0FD00CFB0544D4F81C419847DDE9C2
:10C270000412CDE90104094B00973046F8F77EFE21
:10C2800007B0F0BD9847DDE90412CDE90070044B1A
:10C290003046F8F773FEF3E730260020C87E030827
:10C2A000EA7E030800B58FB001A93322FFF7C4FF6F
:10C2B000034901AA0620F6F77DFD0FB05DF804FBE7
:10C2C0001A7C03082DE9F341036C8B42044688462F
:10C2D00075D0D0E90676012380F8443057EA06038A
:10C2E000016420D0C3685B78012B1CD90022002395
:10C2F000C0E9062304F08CFF656DA26D60653223F2
:10C30000C5F119050544B5FBF3F55D43E36DAB429B
:10C3100019D1B4F86030042B11D80133A4F860307F
:10C32000A36D0BBB15E0606830B1036891B29B6DE3
:10C33000984707460E46DDE704F06CFFF9E79542A3
:10C34000EED0A565ECE70023A4F86030E565002A8F
:10C3500038D1E368A0681978FCF7CCFDC8223221F7
:10C3600000B2F9F79DFCA065A36D05EB5302B2FB8B
:10C37000F3F25A43D4E912134FF47A756A43521810
:10C3800043F10003C4E91223CDE9007604F1200053
:10C3900000F072FBE368C3E91A01E368012283F845
:10C3A0007020E3685B78934209D9D4E912014FF415
:10C3B0007A720023F4F7A0FDA8EB0000206502B01C
:10C3C000BDE8F08123684FF47A71DB6BB1FBF2F1C9
:10C3D0002046C9B29847A3E78368DB8CDB0607EEEB
:10C3E000902A0CD591F85C304BB1D1ED166A9FEDD7
:10C3F000057AF8EEE77AE6EEC77AFDEEE77AC1ED68
:10C40000047A70470000C842006800BA7047000014
:10C4100007B5036842681BBA12BA6846CDE9002323
:10C42000F9F762FC51EC100B03B05DF804FB00005F
:10C4300007B5FFF7E9FF019001A8F9F751FC03B038
:10C440005DF804FB00F1730208B503465018FFF7CE
:10C45000DBFF1860081D1044FFF7D6FF19449880D1
:10C4600091F87920DA8091F87A201A7291F87B207D
:10C470005A7208BD70B500F17306044656FA81F091
:10C48000CDB2FFF7C5FFC4F80B0005F10800C4F8F2
:10C490000F1056FA80F0FFF7BBFFC4F8130005F148
:10C4A0001000C4F8171056FA80F0FFF7B1FFC4F877
:10C4B0001B00C4F81F1070BDF8B54318044693F86C
:10C4C000733080F82330DA070D4611D5CFB200F172
:10C4D0007306781C56FA80F0FFF7AAFF07F10900EF
:10C4E00084ED090A56FA80F0FFF7A2FF84ED0B0AEB
:10C4F00094F823305B0708D504F17300053550FA32
:10C5000085F0FFF795FF84ED0A0AF8BD10B50431F8
:10C510000446733050FA81F0FFF78AFF84ED0E0A6B
:10C5200010BD000070B5CCB2054600F17306201DA9
:10C5300056FA80F0FFF77CFF04F1080056FA80F00D
:10C5400085ED120AFFF774FF103485ED130A56FAD1
:10C5500084F0FFF76DFF85ED150A70BD2DE9F843F6
:10C5600090F87130402B05460F4646D103244FF01A
:10C57000010895F87230A34242D905EB040999F8F5
:10C580007360462E14D901F0B5FCA2224FF400319D
:10C5900001F09CFC013E99F8749002340B2E16D8E1
:10C5A000DFE806F0111715151515151C21151526B0
:10C5B000730906F01F0208FA02F157F823200A4314
:10C5C00047F82320E6E721462846FFF73BFF4C4487
:10C5D000CFE721462846FFF74DFFF8E721462846DA
:10C5E000FFF76AFFF3E721462846FFF78FFFEEE7E4
:10C5F00021462846FFF796FFE9E70020BDE8F883CB
:10C600000120FBE710B5C46E013C0B461146052C1A
:10C6100004D8DFE804F0101A1E223843022B01D0A0
:10C62000002010BD0123C366002380F8753180F817
:10C6300076311846F5E780F87030022290F87611CE
:10C64000C2660B4480F87631EAE780F87130032245
:10C65000F4E780F872300422F0E790F87521811831
:10C66000013281F8733090F876110B4480F87631FE
:10C6700090F87230D2B2934298BF052380F87521AA
:10C6800098BFC366CCE70622C26690F8762180F890
:10C6900073319A42C4D1FFF761FFC2E780F8743169
:10C6A0000023C366C5E7000010B5044B04491860B9
:10C6B0000446FBF7AFFB204610BD00BFD43A002074
:10C6C000BC7F030890F8233063B9012380F823303E
:10C6D000054800684FF40073006C80224FF46141FC
:10C6E000F8F778BB704700BF30260020002850DDE7
:10C6F0006F2846D01BDC132845D00EDC431E082BC8
:10C7000011D8082B33D8DFE803F041053236323236
:10C71000323239004FF416607047392839D0642816
:10C720003AD026283AD04FF47A7358437047B0F580
:10C73000FA7F36D010DCB0F5807F34D006DC732869
:10C7400034D0E628EFD14FF461307047B0F5E67F82
:10C75000E9D14FF4E120704740F2DC53984228D0F1
:10C76000B0F5FA6F27D040F29933984225D0B0F552
:10C77000FA6FD8DD70474FF4965070474FF416505B
:10C7800070470F4870474FF4964070474FF49660DB
:10C7900070474FF4614070470A4870474FF41640A5
:10C7A0007047094870474FF47A3070474FF4E130D2
:10C7B000704706487047064870474FF46120D9E734
:10C7C000FCB10100A086010020A1070060E3160073
:10C7D00080841E000068FFF789BF0000914215D0D9
:10C7E000CBB2581E012801D92B2905D1511EC9B23F
:10C7F00001290BD92B2A09D0053B012B08D8501F42
:10C80000C0B201288CBF0020012070470120704772
:10C81000002070472DE9F843002504468946174655
:10C820002E4600F1060818F9352049462046FFF744
:10C83000D5FF38B1B74203D104EBC500BDE8F8839A
:10C840000136F6B20135042DEDD10020F6E70000E7
:10C8500010B5FFF7DFFF78B1C379092B0CD8074A71
:10C860001033126852F8234024B1236881885B6B2F
:10C8700020469847204610BD0024FBE730260020C4
:10C880000E4B70B51D68CBB2092B0C4612D8103375
:10C8900055F8232000EBC103116810464E6B9988B0
:10C8A000B04750B9A8690649036822461B68BDE82D
:10C8B0007040184700231B68FFDE70BD3026002043
:10C8C0004C7F03082DE9FF41FF23804603A9213057
:10C8D0008DF80C30FBF7A2FD4046FFF7F3FE564BF8
:10C8E0001B68019308F1080401267327019A06F1D9
:10C8F000100352F82350E6717DB3B1B24046FFF702
:10C90000BFFF94F906300133332B00F28C80DFE84F
:10C9100003F0241A1A1A2C3335353D478A338A52CC
:10C920008A8A245A8A8A698A8A4C8A7D8A8A8A8A69
:10C930008A248A8A8A8A8A8A8A8A8A8A8A8A1A8A2D
:10C940008A8A8A8A8A242046FFF744FF4FF480733C
:10C95000014680222846F8F73DFA0136042E04F1FC
:10C960000804C3D104B0BDE8F081092303A920461F
:10C970000393FBF7A9FDF0E73923F7E72046FFF71C
:10C9800029FF102301464FF48072E3E703A92046F4
:10C990000397FBF799FD80231A464FF4E131D9E75D
:10C9A00003A920460397FBF78FFD2046FFF712FFF0
:10C9B00080230146CDE7092303A9A01D8DF80C3083
:10C9C000FBF712FDC9E703A920460397FBF77CFD9F
:10C9D0002046FFF7FFFE1E2301461A462846F8F7B9
:10C9E000F9F90DE02046FFF7F5FE802301461A46CF
:10C9F0002846F8F7EFF92B680121DB6C28469847A9
:10CA00002B680021DB6B28469847A6E703A9204640
:10CA10000397FBF74FFD2046FFF7DCFE102301468E
:10CA20004FF40072DAE72046FFF7D4FE01462846AD
:10CA3000F8F7DAF991E700BF30260020032973B533
:10CA400005461E460CD8CC00A01D01A928448DF82F
:10CA50000420FBF7BBFC01A928190196FBF734FD64
:10CA600002B070BD014B1868704700BFD43A002077
:10CA700001804280704700002DE9F043DDE9074C5A
:10CA8000017EA71A6CEB030629B1D0E90251AF422F
:10CA900076EB010103DAC0E9027601210176D0E9E3
:10CAA0000251B0F800E04FF47A78551908FB0EFEF9
:10CAB00043EB01011EEB050941F10008A14578EBAC
:10CAC0000C0809DAB4EB0E046CF10001A21A61EB58
:10CAD0000303C0E902232546438B0BB9C0E9047662
:10CAE000D0E90442A74276EB0202B8BFC0E904765F
:10CAF000428801339BB29A42438301BFD0E90423A9
:10CB0000C0E90223002343832846BDE8F0830000E8
:10CB100037B504460846089D11461A460368019534
:10CB20009DF81C5000951D68069BA8472060204674
:10CB300003B030BD4FF0FF33002110B50022436138
:10CB40000446417200F12003E830D9709A60DA603F
:10CB50001A615A629A62DA621A635A639A63DA63F2
:10CB60001A645A645A659A65DA6564338342ECD173
:10CB7000044B1A6822B904491C602046FBF74AF9A5
:10CB8000204610BDD83A00208480030890F8221077
:10CB900029B901234384117083711846704700201E
:10CBA000704700004FF000007047000041B103796A
:10CBB000012B05D05A1C027140F823100120704748
:10CBC0000020704738B5054690F8220058B1002380
:10CBD000012004F0CFFC00210446A86B04F0DAFC2D
:10CBE000231A5842584138BD11B990F821007047B6
:10CBF0000020704738B590F90530044633B390F8FB
:10CC000003311BB300252279EBB29A4206D954F8BE
:10CC1000230003689B6898470135F4E704F0F8FAAD
:10CC2000A36EC01AB0F5FA7F94F9E8302CBF00204B
:10CC3000012084F8210013B1002384F8053194F811
:10CC400005112046BDE83840FFF7CEBF002038BDB3
:10CC5000024690F90500B0B192F8030198B1D2ED07
:10CC60000D7A9FED097AF4EEC77AF1EE10FA09D445
:10CC7000B7EE087AF4EEC77AF1EE10FAD4BF0120CD
:10CC80000020704700207047ABAA2A3F014B18686C
:10CC9000704700BFD83A002010B50446006810B1B4
:10CCA00003685B689847204610BD000010B5044635
:10CCB000006810B103685B689847204610BD00000B
:10CCC00070B5D0F8F46016F0800688B004461ED126
:10CCD0000E223146FFF776FF0546002836D0CDE913
:10CCE0000566069B00210A2207A8CDE9061300F07D
:10CCF0003DFB01462046FFF759FF07A8FFF7CCFF91
:10CD000006A8FFF7C9FF15B105A8FFF7C5FFD4F8BE
:10CD1000F41011F4803517D1134B14491B6898682F
:10CD200003681B6898470C22CDE90650294607A8DE
:10CD300000F0DCFC01462046FFF738FF07A8FFF7AC
:10CD4000B5FF06A8FFF7B2FF08B070BD042306497F
:10CD5000CDE901030968064B0093024649680E239A
:10CD600006A8FFF7D5FEBCE7302600204C8003085C
:10CD7000801A060010B50446FFF7A2FF23790BB115
:10CD8000A37943B9044B05491B6898690368BDE85A
:10CD900010401B68184710BD30260020548003083F
:10CDA00010B590F9053004461BB3012380F8043117
:10CDB000836B13B1002280F804212364A37923B983
:10CDC0002046FFF7D7FFA3794BB10A4B1B68986A3F
:10CDD000036864215B6898472046FFF70BFF94F8CF
:10CDE000223003B9A363012384F80331002384F8BC
:10CDF000043110BD30260020064B10B503600446F8
